:020000000C945E
:10000200DA0B0C9400000C9400000C9400000C9489
:1000120000000C9400000C9400000C942C600C94D2
:1000220000000C9400000C94C6130C9400000C9475
:1000320000000C9400000C9400000C9400000C943E
:1000420078130C9400000C94DE5C0C9400000C9469
:100052001A5D0C9400000C9400000C9400000C94A7
:1000620000000C9400000C9400000C9400000C940E
:1000720000000C9400000C94875E0C9400000C9419
:10008200CA5F0C9400000C94000000000100020002
:10009200040008001000200040008000000100025F
:1000A200000400080010002000400080000102044B
:1000B200081020408000B803C20B80100000BC036F
:1000C200C20B821F0000C603C20B81030000CE03D5
:1000D200C20B01040300D803C30B01060500E203AF
:1000E200C50B01800000EE03CC0B020F0000F603EB
:1000F200C60B020F0000FE03C80B020FD01206044B
:10010200CA0B0110000010041A0C011000001A049E
:10011200CB0B000100002204CE0B010801002C04CD
:10012200CF0B030801003A04D00B0307000042047E
:10013200E60B017F3F004C04E50B0105000056046D
:10014200D10B030400005E04E40B01641E006A0488
:10015200D20B000100007604D30B000100008204E0
:10016200E30B010200008E04D40B000100009C048A
:10017200D50B020F0000A804D70B020FE703B2044D
:10018200190C0163000010051B0C011000001A0578
:100192001C0C01020200BE04D90B03080100C404B6
:1001A200DA0B03080000CA04DB0B03080000D004CA
:1001B200DC0B03080000D604DD0B03080000DC049E
:1001C200DE0B03080000E204DF0B03080000E80472
:1001D200E70B040A2E00F004F10B040A2E00F804C7
:1001E200FB0B040A2E000005050C040A2E0008056C
:1001F2000F0C040A2E0000000000FF000000220580
:1002020000022A0504043005080736050C053605E8
:100212008C063C0580094405100B4C05500C560514
:1002220040035E05140A6805180870051C010000E9
:100232000002280060009800D00008014001210C53
:1002420058002D0B2D002B0B2B004D0A4D008081E9
:1002520082838400002188898A8B8C8D8E8F310B5A
:10026200312041424300320B322044454600330BD9
:100272003320474849004D0A4D0000000000340B6E
:1002820034204A4B4C00350B35204D4E4F00360B77
:100292003620505152002B0A2B0000000000370B71
:1002A200372053545500380B382056575800390B15
:1002B2003920595A2F002D0A2D0000000000430C4E
:1002C200430000000000300B3020202E2C002C0AAE
:1002D2002C00000000003D0A435200000000000014
:1002E2004A01460032002100004B004A014600321A
:1002F200004D000096004A0146003200540000E121
:10030200004A01460032003D0000F00000003200C9
:1003120050002D0000F00050003200500047000055
:10032200F000A000320050004B0000F000F000325C
:100332000050002B00005800B400040038003800C0
:10034200213803006A6100008700C800640032009F
:100352003D4603006E65696E00000800C800640037
:100362003200215603004B004A01460032004D0084
:10037200000001000100E60063004D0000000000E3
:10038200A0001B00007105D700A0001A0200710531
:1003920069000000180400730569001E01190600B7
:1003A200730550726F64756B742000005370617234
:1003B2007465202000005F4944005F52733233327B
:1003C200494400005F526F74617465005F54617349
:1003D20074656E5800005F54617374656E59000055
:1003E2005F44656661756C744B6579002A436F647E
:1003F200653000002A436F64653100002A436F6450
:10040200653200002A4D61784D6F64756C005F455E
:1004120072774D6F64756C002A5469736368450086
:100422005F4D795465726D4E72005F4D61737465F4
:10043200725465726D7300005F454D6F6465000014
:100442005F4543726564577472005F5273304D6F3B
:10045200646500005F5634756E6435005F50756CDC
:10046200736554696D6500005F41736B4372656427
:10047200697400005F53656E6444656269740000CC
:100482005F4372656469744D6F6465005F437265B2
:100492006469744D6173746572002A5461626C659B
:1004A2005374617274002A5461626C65456E640013
:1004B2002A4669727374426F6E5000002A4A6F6254
:1004C20031002A4A6F6232002A4A6F6233002A4A96
:1004D2006F6234002A4A6F6235002A4A6F62360020
:1004E2002A4A6F6237005F4572726F7231005F4550
:1004F20072726F7232005F4572726F7233005F45C3
:1005020072726F7234005F4572726F7235005F46AD
:1005120072656967616265005F4B6F6D6D610000B6
:1005220054617374657200004C69745A00004C6522
:100532006974540050756C730000546173742030F8
:10054200000073657269656C6C0073657269656C35
:1005520020320000546173742032000054617374BD
:10056200207061720000466F6C676554000053771B
:10057200697463680000706F7274696F6E69657286
:10058200656E00002E666F6C67650000506F7274B6
:10059200696F6E656E207369636865726E00436889
:1005A20065662D4D656E75004B206C697374656EC2
:1005B20000004B206C6F65736368656E00004B2012
:1005C200647275636B656E0054206C697374656E3A
:1005D200000054206C6F65736368656E00005420E0
:1005E200647275636B656E0053797374656D000098
:1005F200506F7274696F6E004B7265646974650046
:100602004B7265642E436C7200006D616E2E506FEA
:100612007274696F6E005465737400005061726188
:100622006D657465720050726F64756B746500005D
:100632004B656C6C6E65720056656E74696C650014
:1006420030A00531AA0532B40533C00534CA0535D8
:10065200D40536E00546EA0541F20543FA054402AF
:10066200064A0C060000000030EA05371806391E5B
:1006720006382806423206453A0600000000457256
:10068200726F72004F70742E0000496D70756C733A
:10069200000054696D656F7574008006300C0005AA
:1006A20000008606330C000300008C06310C0005A6
:1006B20000009406320C001400002E202C3041421F
:1006C200433144454632474849334A4B4C344D4EF8
:1006D2004F35505152365354553756575838595A48
:1006E2002F390500C11100000300D90B00000300DF
:1006F200C1110300170E0300D90B00000500E0082A
:1007020000000A00C1110A00170E0A00D90B0A00E4
:10071200C1110A00170E2800D90B000000000000CA
:1007220000000000000000000000000000000000C7
:1007320000000000070C182022204D994D40114066
:1007420048914720222018C007000000070C1F3FD5
:10075200EE3F7277727FFF7F777F783FEE3F1FC059
:1007620007000000000000000C183DEE3F3FEE3F86
:100772001FC80F0700020000000000000000000078
:10078200000207080F1FCE3F1FC80F07000200001C
:100792000000000000000007080F0F880F376F7F6E
:1007A2007FFF7F3260070F80000000000000000220
:1007B200000207080F1FCE3F3FEE3F1AC0070F800F
:1007C2000000000000000000000000000006000F12
:1007D2000F0006000000000000000000FFFFFFFF06
:1007E200FFFFFFFFFFF9FFF0F0FFF9FFFFFFFFFF41
:1007F200FFFFFFFF00000000000006000910881044
:10080200108810090006000000000000FFFFFFFF33
:10081200FFFFF9FFF6EF77EFEF77EFF6FFF9FFFF54
:10082200FFFFFFFF000000000E01006A1E33286177
:1008320061886133001E0000000000000000000714
:100842008C0C186618186C0C078003030C0F03003D
:1008520003000000020003038C0302CC02028002A8
:1008620002000E1E001E0C00000000000C000E0B09
:1008720008090CC40E0B4C0938C478784C3103CCEF
:10088200030180000000020202271FCC18306770AB
:10089200306C181FC2270200020000000000001086
:1008A20000181C001E1F081F1F001E1C001810002D
:1008B200000000000000000088010388070F881F65
:1008C2000F88070388010080000000000000020773
:1008D200080F1FC0020200020200021FC80F070019
:1008E20002000000000819198819198819198819B5
:1008F200198819198000198819000000000E1F3686
:10090200CC6666CC6636CC1E06CC0606CC0606CC79
:100912000600000000081F30C03030081F30CC3005
:100922001F8C0000CC301F8000000000000000007F
:100932000000000000000000000000000E1F1FEE7B
:100942001F0000000200070F8C1F020002020002BB
:100952000200021FC80F0700021FC00000000207AA
:10096200080F1FC00202000202000202000202007F
:100972000200000000000202000202000202000265
:100982000200021FC80F0700020000000000000062
:10099200000001080101CE3F01C801010000000072
:1009A2000000000000000000000004000C1C0E3FCC
:1009B2001C000C0400000000000000000000000009
:1009C2000000000000000000400040400040400ED7
:1009D2007F000000000000000000088C1838EF7F44
:1009E20038EC180880000000000000000000000041
:1009F200000000000207080F1FCE3F7FF00000003A
:100A020000000000000000000000000F7F3FEC1F0C
:100A12000F8007020000000000000000000000003C
:100A220000000000000000000000000000000000C4
:100A3200000000000600060F000F0F000F0F000657
:100A42000600060000000600060000000000001973
:100A52008819198819000000000000000000000039
:100A6200000000000006060666063FFC0C0CC819D2
:100A7200198C7F3300333300000000000600061F8C
:100A82008C3F3600363F8C1F06CC063FC81F06003F
:100A920006000000000000001338387E3801C80349
:100AA20007000E1C0E3870EE600000000000070DFB
:100AB200881919801B0E001E3E063333C8313BC60F
:100AC2001E0000000E000E0E000606000C000000C4
:100AD2000000000000000000000000000380060E7D
:100AE200000C1C001C1C001C1C001C0C000E060828
:100AF200030000001C0006070003038803038803A9
:100B020003880303000706001C0000000000000029
:100B12000C3636C81F0F0C3F0F081F36CC360000AC
:100B220000000000000000000000060006060C3F66
:100B32003FC00606000600000000000000000000A2
:100B4200000000000000000000000000000E0E0087
:100B52000E06000C000000000000000000000C3F28
:100B62003FC0000000000000000000000000000084
:100B7200000000000000000000000000000E0E0057
:100B82000E00000000010000370000EC01038007A6
:100B92000E001C3800706000000000000F8E3F3015
:100BA200676060FB616333666C33787036303FE8B0
:100BB2000F0000000300071F001F030003030003D0
:100BC2000300030300031FEE1F0000001FCE3F704F
:100BD2007360607E0001C80307000E1C00387FFFAF
:100BE2007F0000001FCE3F7073600037000FEC0FD4
:100BF2000063006037703FEC1F00000001CC030768
:100C0200CC0E1CCC3870CC607FFF7F00CC0000CCB7
:100C1200000000007FFF7F600060600C7F3FE70004
:100C22000033006037703FEC1F00000003CC070E5A
:100C3200001C3800307FCE7F7073606037703FECED
:100C42001F0000007FFF7F00660000CC00018801CA
:100C52000300030600060C000C0000000F8C1F3876
:100C6200E630306E381FCE3F7073606037703FECF5
:100C72001F0000001FCE3F7073606037703FFF1F80
:100C8200006E0001C8031F001E00000000000000EB
:100C920000000E000E0E00000000000E000E0E00FE
:100CA200000000000000000000000E000E0E000018
:100CB2000000000E000E0E000606000C00CC010320
:100CC20080070E001C3800381C000E07080301CCF8
:100CD20000000000000000000000000E3F3FE000A6
:100CE200000E3F3FE0000000000000003000381C12
:100CF200000E07080301CC010380070E001C380018
:100D0200300000001F8C3F70E66060EC010380073A
:100D12000600060600000600060000001FCE3F3057
:100D22006B676FBB6D6DBB6D6DBE6F67C0703FCC87
:100D32000F0000000600060F000F0F08191988198E
:100D420030CC3F3FC6606066600000007F087F6174
:100D5200CC6060CC617F8C7F60E660606E607FC833
:100D62007F0000000F8C1F38E6306000606000607A
:100D7200600060306E381FC80F0000007F087F617E
:100D8200CC6060666060666060666060CC617F8037
:100D92007F0000007FEE7F6000606000607F887FE0
:100DA2006000606000607FEE7F0000007FEE7F6089
:100DB20000606000607F887F6000606000606000AB
:100DC200600000000FCE1F38603060006063EE6389
:100DD2006066603066381FEE0F000000606660607B
:100DE20066606066607FEE7F606660606660606617
:100DF200600000001F881F060006060006060006A7
:100E02000600060600061F881F000000006600009C
:100E12006600006600006600006660606C703FC895
:100E22001F000000606E6061C86367006E7C007C1A
:100E32006E0067638C6160E66000000060006060C5
:100E420000606000606000606000606000607FEED3
:100E52007F000000606E7070EE7979E66F6F6666F3
:100E62006666606066606066600000006066707062
:100E720066786C666C66666663666361EE6060E601
:100E8200600000000F081F39CC3060666060666049
:100E920060666030CC391F800F0000007F8C7F605D
:100EA200E66060666060EC7F7F806060006060008A
:100EB200600000000F081F39CC3060666060666019
:100EC20060666333CC391FE60F0000007F8C7F60C1
:100ED200E66060666060EC7F7F8067638C6160E6DD
:100EE200600000001F8C3F70E6606000703F8C1F46
:100EF20000E600606E703FC81F0000003FCC3F0656
:100F020000060600060600060600060600060600A3
:100F12000600000060666060666060666060666031
:100F2200606660606C303FC81F00000060666060F1
:100F32006C3030CC3019881919800F0F000F060061
:100F420006000000606660606660606660606666FB
:100F520066666F79EE7070E6600000006066603071
:100F6200CC3019800F0600060F081930CC306066AD
:100F72006000000060666030CC301988190F000FE5
:100F82000600060600060600060000007FEE7F004F
:100F9200CC000180030600060C00183000307FEE02
:100FA2007F0000001F881F1800181800181800186A
:100FB2001800181800181F881F0000000000406069
:100FC200007038001C0E0007038C0100E70000309F
:100FD200000000001F881F018801018801018801AB
:100FE2000188010188011F881F0000000200070F0D
:100FF2008C1D38E770603000000000000000000027
:1010020000000000000000000000000000000000DE
:101012000000000000000000007FFF7F00000707C3
:1010220000070600060300000000000000000000A8
:1010320000000000000000000000000C1F3FE6005E
:101042001FEE3F6066607FEE3F0000006000606060
:10105200006060086F7FCE70606660606E607FC8FF
:101062007F00000000000000000000081F3FC67063
:101072006000606006703FC81F000000006600004C
:10108200660000661F3FEE716066606066703FEE4C
:101092001F00000000000000000000081F3FC67093
:1010A2007FEC7F6000703FC81F00000007880F1CA4
:1010B20000181800187F007F180018180018180070
:1010C20018000000000000000000000E1F3FE67044
:1010D200606E703FE61F006E003FC83F60006060B8
:1010E200006060006F7F8C7160CC6060CC6060CC0F
:1010F2006000000000000006000600000E0E000660
:101102000600060600061F881F00000000000001FE
:101112008801000803038801018801018801018810
:10112200191F800F300030300030300831338037E3
:101132003E003E37083331CC300000000E000E0670
:1011420000060600060600060600060600061F88C0
:101152001F0000000000000000000008597FCE7F41
:1011620066666666666666666600000000000000E7
:10117200000000083F3FCE303066303066303066C7
:101182003000000000000000000000081F3FCE7089
:10119200606660606E703FC81F00000000000000C3
:1011A200000000087F7FCE6060666070EC7F6F8019
:1011B20060600060000000000000000E1F3FE6704B
:1011C20060666070EE3F1F6600006600000000006F
:1011D2000000000C373FE63830003030003030007D
:1011E2003000000000000000000000003F7F80602F
:1011F2007F083F0188017F803F000000000018182F
:10120200001818007F7F00181800181800181F888F
:101212000F00000000000000000000066060666031
:10122200606660606E703FE61F0000000000000014
:101232000000000660606C3030C81919800F0F0082
:1012420006000000000000000000000666666666F8
:101252006666666F6C3F39C810000000000000002F
:101262000000000C6071C83B1F000E1F083B71CCD0
:1012720060000000000000000000000C3030C819BF
:1012820019800F0F000606000C0C00180000000069
:101292000000000C7F7F800306000C1800307FCC1A
:1012A2007F00000003CC070E000C0C000C1C003861
:1012B2001C000C0C000C0E0C0703C00006000606F6
:1012C20000060600060000060600060600060600E6
:1012D200060000003C003E070003030003038C01EC
:1012E20003800303000307003E3C00000000001CD3
:1012F2006C36638000000000000000000000000067
:101302000000000000000000000006000F198C30F1
:101312006066607FEE7F00000000000000001E009B
:1013220060077E0700F01EF060F77EF7FBDE1F000D
:10133200E007FF0700F81FF8E0FFFFFF00000F00C3
:10134200E002EF0200780F78E07AEF7AF7BD1F0033
:10135200E007FF0700F81FF8E0FFFFFF230000028D
:101362000000100000050000FE0500182800FE0421
:1013720000182400F90F00F80F0070001F7180237D
:1013820072802A73111574111C75151B76151A7744
:10139200181C781521050100FF000000013F2B02F7
:1013A2000010072100000100072300100000FD309B
:1013B20000073300113068FF0000E50080000100E3
:1013C20001000102000403301004000008020209B7
:1013D20000000A00000C00000D00000F00001000C9
:1013E20000110700120000130000FD500010B01B96
:1013F200110700FD5000121E01FD500013001F29AD
:101402001F00FD5000200000210000FE01002B0CF7
:1014120000FE00002B2000300000310603320002E3
:101422003507013604043706063805013907073C3B
:1014320000063D070850000051EF00520000533FE4
:1014420001FE01006000A7FE0000600027610100AC
:101452006A00008000008100008200008300008496
:101462000000850000901000920007930700953F4E
:1014720003970000980000070100FD5000072100BB
:10148200072300FD5000077301FF00000000000069
:101492002564002B003E3E006B65696E204B726531
:1014A20064697400436F6C6F72546F756368205681
:1014B2007320312E35340049443D00202047433DFE
:1014C20000202036346B004B653A00496E3A0043E7
:1014D200616C6962726174696F6E004F4B00546F88
:1014E20074616C20002D2D2D2D0054696E79200021
:1014F20054696E792062616400204C006B65696EEC
:1015020020454570726F6D004D4F44554C20535429
:101512004F5000446174612000696E697400533F4A
:10152200000066616C736368657220546973636856
:101532002000546973636820766F6E204B2000464A
:1015420065686C6572200056656E74696C20616B0B
:101552007469760054696D656F7574004353492050
:101562004E722000436F646520006B65696E204BEC
:1015720072656469740066616C7363686572205495
:101582006973636800546973636820766F6E204BD9
:10159200005831393931303000504C5520203A0052
:1015A200436F6465203A005469736368203A004DC2
:1015B20042005053004D31004F3100535000435010
:1015C2000044590062757379004D500020676573BD
:1015D200706572727400256400004162726563680E
:1015E2006E756E67004B656C6C6E65722000546F91
:1015F20074616C004D6F64756C2000202000433FC5
:101602000073656300496D7000504C553A200053D9
:1016120070617274653A20005072313A2000507243
:10162200323A200046756E6374203A200054797075
:101632003A20003A20563A2020302B2030003A003F
:101642003A20544F3A20003A2050733A2000537007
:101652003A004B204D6F6465204A6F62204A6F62E8
:10166200466C616773004B20004D6F646520004A31
:101672006F62202000562020204572722050676C35
:1016820020496D7020544F005620005061757365DB
:10169200004B656C6C6E65723A004D49004D42001C
:1016A2004D43004D50004D4C0074657374202E2E36
:1016B200004F4E0025303258002530345800253670
:1016C20064002533642E25303264002535640025FC
:1016D20064002532640025336400444400004B2337
:1016E20000425300422100424600542300544F005E
:1016F2004952004D5A004251004252004353005693
:101702005300564300494C00426600004B230054EC
:1017120023004245004345004241004453004342F6
:101722000023502241534349492D492F4F222C2255
:10173200312E3030222C323030382D30312D3031B4
:101742003B0023482245636F222C22312E30302267
:101752002C323030382D30312D30313B00235322A2
:1017620045636F222C22312E3030222C3230303819
:101772002D30312D30313B00504F00504632333B3B
:101782005055002564002B302B303B00256400258A
:10179200303258002E3030004F4E000077616C6CB2
:1017A200610001002D4E414E00000100E10EA41720
:1017B2000000F894EE27ECBBF1E0F5BFE5BFE09343
:1017C2006C00F8E1F1BDE1BD8DE0A2E0BB27ED9335
:1017D2008A95E9F780E090E1A0E0B1E0ED9301970E
:1017E200E9F7ECEAF7E185919591009761F0A5910F
:1017F200B59105901590BF01F00105900D920197EA
:10180200E1F7FB01F0CFEFEFEDBFE0E1EEBFC0E0AB
:10181200D3E00C943D150A9902C0E1E00895E0E09E
:101822000895A0913E0CA13031F40E94276B0E94D2
:1018320044660E94386B0895A0913E0CA13031F4A9
:101842000E94276B0E94426B0E94386B0895E881C8
:10185200E03011F01C9A01C01C982FC00E94466B08
:101862000E94466B0E944B6BEFE3F0E00E94506BCC
:1018720008951A93A0910403A43081F4E0910F0417
:10188200E093100410E0183048F4ABE01A9FF00126
:10189200E052FD4F0E94566B1F5FF5CF3CC0A091F6
:1018A2000403A43039F4E881E0931004E0E0E0930B
:1018B2000F0403C0E8810E945A6B219608951A937F
:1018C200A0910403A43019F110E0143000F50E9435
:1018D200606B3196E491EA93E2DFE0E0E09310047A
:1018E2000E94696BEBE0F1E00E94736B0E94736BE4
:1018F200FA93EA930E94606BE491EA930E94606B10
:1019020032960E94786B0E94BB421F5FDECF0E941C
:101912007B6B0E94806B199108952A970E94BB7C71
:1019220030E010E000E047ED50E028E0E0911A0CD2
:10193200E03019F020E149E650E0321710F00C9443
:10194200DF0C0E94846BE13090F10E94846BE038DE
:1019520070F0EEE00E948A6BE2E9F4E1FA93EA9316
:101962000E94846BEF70EF5F0E94926B07C0ECE005
:10197200EA9395DFE8E5EE83E0E0EF830E94696B8E
:10198200A02FB0E0E7E3F0E00E94357AE40FF51F04
:101992000E94736BFA93EA93EDE2F0E0FA93EA9312
:1019A2000E94846BEA930E94466B0E949C6B1F5FAD
:1019B200143011F410E00F5F3F5FBFCF0E947B6BCA
:1019C2000E944A480E94C27C619608950E94A26BBE
:1019D200ECE0EA9364DFEAE3F3E00E94566BEBE0AB
:1019E200EA935DDF0E94A66B0E94AB6BEAEAF0E02D
:1019F2000E94B06BE0913B0CF0913C0CE491EA93B5
:101A0200E0913B0CF0913C0C31960E94B76B0E9426
:101A1200BB4201E00E94BA6B0E94BD6B11F00F5FE6
:101A2200F9CF0E94CB6B031718F4E0E0E093C005F6
:101A32000E94CB6B11E00E94D26B0E94BD6B11F031
:101A4200153008F021C00E94A66B0E94D56BE0E41D
:101A5200F0E00E94357A3496FA93EA93E2EEF0E0EF
:101A62000E94B06B0E94D26B0E94D86BE491EA9301
:101A72000E94D26B0E94D86B31960E94B76B0E9473
:101A8200BB423F5F1F5FD7CF0E94806B0E94C47C26
:101A920036C427970E94BB7C22E354E0A091040342
:101AA200A43011F426E453E010E0143010F00C944A
:101AB200A50D00E0051710F00C94A30DE12FEE0F19
:101AC200EE0FE00F3E2F0E94D26B0E94E46B319624
:101AD200E4910E948A6B0E94D26B0E94E46B329660
:101AE200FA93EA930E942468ED85E03039F4AF81DD
:101AF200A13210F4E0E0EF83E0E0E887A02FBB27FB
:101B0200E22FE85FF0E00E94357A3896FA93EA9382
:101B12000E94D56BEAE3F0E00E94357AE55BFF4F65
:101B22000E94E96B0E94736BFA93EA930E94D26B54
:101B32000E94E46BE491EA930E94466B0E949C6BC4
:101B42000F5FB8CF1F5FB1CF0E94806B0E94C27C33
:101B52002E96089522970E94EE6BA13059F40E94AE
:101B6200F36BABE2B1E00E94607A2E2F57E1E2EC18
:101B7200F0E008C00E94F36B0E94F76B2E2F53E037
:101B8200E7EEF0E0EE83FF830E94FC6BA091190860
:101B9200A13081F4E9ECF0E00E94136C0E941A6C0F
:101BA2000E941F6CEBE2EA93E5E9F4E10E94786B94
:101BB2000E94BB42E3E0F0E00E94136C0E94256C9D
:101BC2000E941F6C0E942A6C0E942E6C3F5FE09163
:101BD200C20BAFEE0E943F7AF0E0EE83FF8311E08A
:101BE200E091C30B1E17C0F500E0E091C20B0E1787
:101BF20088F50E94346C59F10E943B6CE09310040A
:101C02000E94BA6BAE81BF810E94357A33960E94E0
:101C1200E96B0E94D56B0E94357ADF010E94456C08
:101C22000E94486CEA85FB853497FA93EA930E94F6
:101C32001F6C0E942A6C0E942E6C3A930E94C71F4E
:101C4200EF3F29F0ADE05A9FF0010E944D6C3F5FDB
:101C52000F5FCBCF1F5FC4CF0E947B6B0E94806B54
:101C6200CBC022970E94BB7CE2E5F7E0EE83FF83C4
:101C720040E0443190F4AE81BF8111960E94556CD0
:101C82001396EFEFEC93AE81BF81EC93EE81FF816F
:101C92003496EE83FF834F5FECCFE091C20BA0EF4F
:101CA2000E943F7A2E2F0E94F36BA0E4B1E00E94C3
:101CB200607A5E2F0E94FC6B21FE24C00E945A6C47
:101CC2000E945A6CEFEAF0E0FA93EA930E945F6C8A
:101CD2000E942A6C0E942E6CEFE00E945A6BE6EB87
:101CE200F0E0FA93EA930E945A6C0E941A6C0E94E6
:101CF2005F6CEFE7EA93E7E9F4E1FA93EA93E0E055
:101D0200F0E011C00E945A6C0E945A6CE8EEF0E0BA
:101D1200FA93EA93E52F0E94656CFA93EA930E9484
:101D22002A6CEBE8FBE0FA93EA930E94BB423F5F26
:101D320011E0E091C30B1E1710F00C94F70E00E0B7
:101D4200E091C20B0E1710F00C94F50E0E94346C49
:101D520011F40C94F20EA0919B0BE0E8EA23E03818
:101D620021F0A091E30BA23019F40E943B6C0AC04F
:101D72000E94686CE03011F4E0E001C0E8E0E0931A
:101D82000F04E7E0E0931004A02FBB27E22FF0E05E
:101D92000E94357A3396FA93EA930E94456C0E9428
:101DA200D56B0E94357A3396FA93EA930E941F6CA0
:101DB2000E945F6C0E942A6C0E942E6C4E2FA09192
:101DC2001E08E32F0E946D6CEA0FFB1F43833A93B8
:101DD2000E94C71FEF3F29F0ADE04A9FF0010E9429
:101DE2004D6C3F5F0F5FACCF1F5FA3CF0E947B6B39
:101DF2000E94806B0E94CF340E94C27C2896089574
:101E0200E1E0E0930D04E2E0E0930E04E0E0E09311
:101E12001004ECE0E0930F04ECE5F3E00E94566B53
:101E2200EAE0E0930F04EAE4F3E00E94566B0E94BA
:101E32004A4808951A93A981A43029F4A0E021FC0C
:101E4200A1E0A03009F427C0E9810E94746C0490DB
:101E5200E9810E947A6CE491A02DAE1BA2501A2F48
:101E6200EFE00E945A6BE4EBF0E0FA93EA93EB8125
:101E72000E947A6C0E94E87A3296FA93EA93EAE335
:101E8200F0E00E94826CEFE7EA93E7E9F4E10E9456
:101E9200786B0E94BB421881229608951A930A9386
:101EA2000E94896C0E94B4170E94686C0E2FE4E3B2
:101EB200F2E00E94E87A33971E2F0E94466B0E943E
:101EC200466B0E944B6B0E948E6C0A930E94B24A30
:101ED200ECE3F0E00E94936C0E94B745E2E0E093ED
:101EE2000E04E091990BEF70E09310040E949A6C3B
:101EF200E0E0E0931004AA81A13051F40E94A26CA8
:101F02000E94AB6B0E949C45EAE9F4E10E94A76C37
:101F120021FE0DC0E4E0EA938DDFECE3F2E00E94E3
:101F2200AB6CEEE3F2E00E94AB6C0E946548A1DC70
:101F320080C0E8810E947A6C0E94AB6CEA810E94A8
:101F4200746C0E94AB6C0E94F445E881EA9372DFE4
:101F5200C4C11A930A93EC81EA93EBDF1AEEEC8187
:101F62000E94746C0490EC810E947A6CE491A02D22
:101F7200AE1BA2500A2FAC81A43029F4A0E021FCB0
:101F8200A1E0A03009F409C01EEAAA81BB811B9618
:101F9200E0E0EC93EC81EA934DDF0E943B6CE0932E
:101FA2001004EC810E94B06CFF93EF930E945A6C74
:101FB200EE810E947A6C0E94E87A31960E94826CCD
:101FC2000E94BA6BFA93EA93EC85E058EA930E9476
:101FD200466B0E94B66C0E94BB42AF91BF91EC93DC
:101FE200EC810E947A6C0E94AB6CEE810E94746C50
:101FF2000E94AB6C0E94654819810881259608955C
:102002000E94BB6C0E94F76B8F010E94466B0E947C
:10201200466B0E944B6B0E94BE6C0E94A26C0E9497
:102022009C45EA81EA930E94B4170E949A6C0E942E
:10203200C56C19810881239608950E94BB6C0E9489
:10204200F76B8F010E94466B0E94466B0E944B6B9E
:102052000E94BE6C0E94A26C0E949C45EC81FD8194
:102062000E94A76CAA81BB810E94B17C24F4A0309B
:10207200E0E1BE070CF006C0EA81FB81FA93EA9325
:102082000E945740AA81BB81A130E0E1BE0724F043
:10209200A030E1E1BE070CF00AC0A7EEBBE0EA8186
:1020A200FB81E150F0410E94CF6C0E94D76C0E94EC
:1020B200C56C19810881269608950E94BB6C0E9406
:1020C200F76B8F010E94466B1A930A930E94654830
:1020D200E0E0E0933D0C099119910895E881EA93BB
:1020E2000E94B4170E94941EE03051F10E94DD6CF0
:1020F2000E94466B0E94E16C0E949A6C0E94E56C01
:10210200E881EA930E941420E8830E94E96C3B97DD
:1021120034F00E94E96C0E94F46CE9E40BC0A3EE77
:10212200B6E00E94F86C0E94FB6C0E94006D0E9457
:10213200056DE3E7EA930E943645E2E0E0930E0480
:10214200CCC00E948467E0E0E0930F04A0910403F6
:10215200A43019F4E8E6F3E002C0E4E7F3E0FA930E
:10216200EA930E949B4208950E94C3450E9484679D
:102172000E94E867E1E0E0930D040E94DD6CE6E076
:10218200F0E00E94096DE6EAF4E10E94A76C0E9469
:10219200466BE7E0F0E00E94096DE9EBF4E10E9492
:1021A200A76C0E940D6DEA930E946440EDEBF4E18E
:1021B2000E94A76CE0910403EA930E946440E3EC5E
:1021C200F4E10E94A76C08952A971A930A930E9439
:1021D200466B0E94466B0E944B6BE4E6F0E00E9465
:1021E200506B00E010E01530B0F4053020F40E948E
:1021F200126DE03009F40DC00E94466B0E94BA6B6A
:102202000E94096D0E94196D0E94126D0E941E6D3E
:102212000F5F1F5FE8CF0E94206D0E949C45E9EC92
:10222200F4E10E94A76CE091420CEA930E946440A0
:10223200E091410CEA930E946A400E94A66B0E94C0
:10224200A26C0E949C45EDECF4E10E94A76CE09127
:102252002306EA93E5E0EA930E941A40E0911A0C01
:10226200E03079F10E94A66BE2E0F0E00E94096D95
:10227200E09128060E94236D0E945A6C0E949C45A0
:10228200E0912806E295EF70E695E695AE2FE09193
:102292002906EE0FEE0FEA0F0E94236D0E94AB6B30
:1022A2000E949C45E0912906E295EF70AE2FE091E5
:1022B2002A06E295E07FEA0FEA93E6E0EA930E94BB
:1022C2001A40198108817DC1E881E064E7B9369A34
:1022D200349BFECF349AE4B1F5B121960895E8819A
:1022E200F981AA81BB81AE17BF071CF4EA1BFB0B65
:1022F20006C0A881B981EA81FB81EA1BFB0B249607
:10230200089528970E94BD7CEFE0E0936100E1E030
:102312000E94296DE5E00E94306D0E94376DE093C6
:102322006F05F0937005E0917B05F0917C05E093D9
:102332006D05F0936E05E1E0EA93C6DFE0937B055D
:10234200F0937C05EFE0E0936100E8E00E94296DE4
:10235200EAE00E94306D0E943C6DE0936B05F093C1
:102362006C05E0917905F0917A05E0936905F093A7
:102372006A05E0E0EA93A8DFE0937905F0937A0535
:102382000E943C6DA0916B05B0916C05EA0FFB1F9A
:10239200A0917905B0917A050E94416D8F010E944A
:1023A200376DA0916F05B0917005EA0FFB1FA091E8
:1023B2007B05B0917C050E94416D9F01E0916B0508
:1023C200F0916C050E94486DFF93EF930E943C6D63
:1023D2000E94486DAF91BF91EA0FFB1FFF93EF93ED
:1023E200E0917905F0917A050E94486DAF91BF9115
:1023F200EA0FFB1FE0937505F0937605E0916F05F8
:10240200F09170050E944E6DFF93EF930E94376D1D
:102412000E944E6DAF91BF91EA0FFB1FFF93EF93A6
:10242200E0917B05F0917C050E944E6DAF91BF91CA
:10243200EA0FFB1FE0937705F0937805A0917505ED
:10244200B0917605E4E1F0E00E94077A0E2EA091A9
:102452007705B0917805E4E1F0E00E94077AE0297F
:1024620019F00E946B44ABC0009371051093720582
:102472002093730530937405A0916405A63428F463
:10248200E0916405EF5FE09364050E94546D9897B4
:1024920024F40E94596D98970CF00EC0A091640527
:1024A200AA3019F4E1E0E0936105A0916405A83235
:1024B20019F4E2E0E09361050E94546D999724F0CB
:1024C2000E94596D99970CF47AC0E0916705EF5F0D
:1024D200E09367050E945E6D0E94546D0E94636DD9
:1024E2000E946A6D0E946F6D0E943A7A7F936F9389
:1024F200FF93EF93A2E0B0E00E94037B0F010E94E2
:102502005E6DDF01F001EA1BFB0BAF91BF918F9172
:102512009F910E94786D0E946A6D0E947D6D0E945B
:10252200596D0E94636D0E94826DAC81BD818E8166
:102532009F81EFE3F1E060E070E00E943A7A7F93DE
:102542006F93FF93EF93A6E0B0E00E94037B0F012D
:102552000E947D6DDF01F001EA1BFB0BAF91BF9181
:102562008F919F910E94786D0E94826DE09112047A
:10257200E03049F4E885F985E0935905F0935A056E
:10258200EC81FD810AC0EC81FD81E0935905F09355
:102592005A050E946F6D0E94CF79E0935B05F0931C
:1025A2005C05E0915905F0915A05FA93EA93E0919E
:1025B2005B05F0915C05FA93EA930E94F3430E9453
:1025C200C47C2C9608951A930E94C345E2E0E093DE
:1025D2000E04E2E3F0E00E94736B0E94876DE1ED6E
:1025E200F4E10E94A76CE4E1EA930E94C33FE0E9B0
:1025F200F1E00E948B6DE4E1EA930E94C33FA09157
:102602006705A13010F0A895FACF10E0143010F051
:102612000C946513E2E0E0930D040E948F6DDF01DC
:102622000E94AB6CFD0132960E94AB6C0E94B745D2
:102632000E948F6D3496E491EA930E943645E1E060
:10264200E0930D04A0916705AF3110F4A895FACF7D
:10265200EAE0EA930E94C33F0E948F6DDF01359644
:102662000E94E87ABF01FD010E94956DDB010E9484
:10267200137BE2E3F0E0FA93EA930E94D56BE8E27F
:10268200F0E00E94357AE65AFF4F0E94876D0E9461
:102692008F6D0E94956D0E94F46CA0916705AE311A
:1026A20010F0A895FACF0E948F6DDF010E94AB6CEB
:1026B200FD0132960E94AB6CE8E1F0E00E949C6D55
:1026C2000E94506B1F5FA2CFE2E3F0E0FA93EA931D
:1026D200EAEFF0E00E94876DEDEDF4E10E94A76C55
:1026E200E0EDF7E00E948B6D0E94C3455FC10E943E
:1026F200A16D0A93E4E6E2BF78940E94B54301DE3D
:10270200E6B3AFEFEA27E093420CE091410CE030F0
:1027120009F002C0E091420CE0933108A3E6BBE06D
:102722000E94B06DE091630BE77031F4A0910A044E
:10273200E0E4EA27E0930A04E091630BEF7131F4DD
:10274200A0910A04E3E8EA27E0930A040E942465C0
:102752000E94B320E2B3EF700E2EA0911408B09144
:102762001508EFE0F0E0AE27BF27EA23FB230E9423
:10277200E879E029E2BBE0911408E07111F41D9AB6
:1027820001C01D980991199114C00E94A16DE6E043
:10279200E4BDE0B1E295EF70AE2FE0916300E0712D
:1027A200EA2B1E2F0E948E6C0E948A200E94FE64D9
:1027B2001991E991EFBFF991E991B991A991999193
:1027C200899179916991F9901990099018950E94CF
:1027D20028640E94AE640E94B14F0E94D01D0895E9
:1027E2001A93A8950E94C941E13011F00C94521439
:1027F200E091C605E1501E2FA091C505A13021F43C
:102802000E94B66DE03009F40CC0ADE01A9FF001F1
:10281200E15FFC4FBF01E081E260DB01EC930E94CB
:10282200BD6DA091C505A23011F0A43089F40E94BB
:10283200B66DE093DB050E94C26D31F0FD01E15FF0
:10284200FC4FE081E27009F403C01A930E94CB6D41
:10285200A091C505A33019F41A930E948226A09173
:10286200C505A53029F4E091C605EA930E94AF267A
:10287200A091C505A830A9F4E0E0EA93E091C6056D
:10288200EF77EA930E9487171E2F1F3F51F0E0E077
:10289200EA930E94C33FE12FE058E093DB05E09307
:1028A2002D06E0910A04E07821F1E0910A04EF7725
:1028B200E0930A040E948E48E0910A04E07131F02C
:1028C200E0910A04E270EA930E949D44E4EEEA93E6
:1028D2000E946A65A0913E0CA13021F4A0911908D2
:1028E200A43009F406C0E0EBEA930E946A65E09323
:1028F200410CA0913D0CA13039F4E0913F0CF091D4
:10290200400C0E94CF6D09F401C0D7DB60DF4EC0DE
:102912001A930E94C345E1E0F0E00E94786B0E94A6
:102922009C4510E00E94D96D0E94466B0E948E6CFD
:102932000E949C45E0912108E03049F4E0EEF4E188
:102942000E94A76C0E94DF6D0E94056D1E5FA09120
:102952002108A130F0F0E0912108E150EA930E94B1
:10296200E317A091B40BAD3229F40E94E86D0E94E6
:10297200AD7C79F0E4EBFBE00E94D76CE6E0F0E09E
:10298200FA93EA930E94F56D0E94E86D0E94056D2C
:102992001E5FE0912108EF5FE09321081C3020F4D4
:1029A200A0912108AB3008F001C0BECF1991089563
:1029B2001A930E94C345E981E03019F4E0E0E09304
:1029C2001E08A981A230A9F410E0A0911E08A1302E
:1029D20010F01C3008F00DC0E0911E08E150E093A9
:1029E2001E080E94F96D19F40E94076E09F01F5F1C
:1029F200ECCF0E94D96D10E00E94466B0E948E6C53
:102A02000E949C45A0911E08A03408F50E94F96D11
:102A120019F40E94076ED1F0E0911E08EA930E9419
:102A2200B4170E949A6C0E94466B0E94F56D0E9438
:102A3200126E0E94F46CE8E7EA930E9436450E9407
:102A4200E56C0E94176E0E94056D1E5F05C0E7EEE1
:102A5200F4E10E94A76C1E5FE0911E08EF5FE09315
:102A62001E081C3020F4A0911E08A13408F001C0F9
:102A7200C3CF188122960895E0E0E5BFE0936D0090
:102A8200E0936C00EBBBEFEFEABBE0E0E8BBE7BB37
:102A9200E5BBEFEFE4BBE0EFE2BBE1BBE0E2E3B9B1
:102AA200ECEBE2B9E0E0E0936200E0936100EFE07A
:102AB200E0936500E0936400E0E0E0BFE7E0E3BF9D
:102AC200E4E6E2BFE0E0E1BFEFBDEEBDEDBDECBD8F
:102AD200E7BDE6BDEBBDEABDE9BDE8BDE093790027
:102AE200E0937800E3E0E5BDE6E0E4BDE0E0E3BDCD
:102AF200E0938B00EAE0E0938A00E0E0E093890053
:102B0200E0938800E0938100E0938000E2E1E093AB
:102B12008700E4E3E0938600E0E0E0938500E09341
:102B22008400E0938300E0938200E0936A00E0E394
:102B3200EABFE0E4E9BFE8BFE1E4E7BFE0E0E09339
:102B42007D00EBB9E8EDEAB9E6E0E0939500E0E05C
:102B5200E0939000E3E3E9B9E0E0E0939B00E8ED65
:102B6200E0939A00E6E0E0939D00E0E0E0939800B5
:102B7200E3E3E0939900E0E8E8B9E0E0E0BDE0E4F7
:102B8200E7B9E7E8E6B9E0B5EF7EE0BDE0E2E09361
:102B92007000E0E0E0937200E4E4E0937400EFE19F
:102BA200E1BDEFE0E1BD0E94BB5C0E944D4A0E9484
:102BB2008E447894E1E0EA930E94280C0E940D6D05
:102BC200E53128F0A9E0B0E0E0E00E941B7BCCDA1E
:102BD20021E030E0E0EEEA930E946A65E093320879
:102BE2000E94206E3F5FA0913208A43511F03A3066
:102BF20008F001C0EFCF30E0E0EBEA930E946A6593
:102C0200EF3F19F0E1E0E0933E0C0E94206E3F5F3F
:102C1200A0913E0CA03011F43A3008F001C0ECCF84
:102C22000E94A26C0E94A66B0E949C45A091320851
:102C3200A43581F4E2EEEA930E946A65E0933208D9
:102C4200ECEEF4E10E94A76CE0913208EA930E9454
:102C5200364508C0E0E0E093320820E0E2EFF4E11C
:102C62000E94A76CA0913E0CA13021F4EBEFF4E19D
:102C72000E94A76C92D0E03059F40E94A26CE9E065
:102C8200F0E00E94096DEEEFF4E10E94A76C20E0F3
:102C92000E945E6D0F01A2E0B0E00E94037B0E165F
:102CA2001F0654F40E947D6D0F01A6E0B0E00E9461
:102CB200037B0E161F060CF086DC203071F40E9496
:102CC200A26CEAE0F0E00E94096DEAE0F5E10E9400
:102CD200A76CA8950E94236EFCCF0E94B6350E9475
:102CE200A26CE9E0F0E00E94096DE5E1F5E10E94E5
:102CF200A76C0E94571AE03019F0EBE1F5E102C02F
:102D0200EDEDF4E1FA93EA930E944D450E94366597
:102D1200E1E0EA930E94C33F00E010E00436E0E005
:102D22001E0724F40E94AE64E03009F005C00E9440
:102D3200206E0F5F1F4FF2CF0436E0E01E072CF02B
:102D4200A0916705AF3108F03EDC4ADD0E942131D7
:102D52000E94871CFACFFFCF0E94266E17FD02C089
:102D6200103011F4E0E05DC3E12F5BC30E94266ED8
:102D720017FD10E01A3008F41F5F0E94336E51C332
:102D82000E94266E17FD02C0103011F4E0E049C324
:102D920011500E94336EE1E044C31A930A9310E08B
:102DA200E4E6F0E00E948B6DA8950E948465E03015
:102DB20021F4E0EA0E943E6E09F002C001E001C087
:102DC20000E00E9495651F5F003011F4153008F095
:102DD20001C0E6CFE02F0991199108950E94436E38
:102DE2003DC40E94436E0E94506E0895A881B9812D
:102DF2000E94B17C24F4A83EE3E0BE070CF005C0BB
:102E02000E94536E0E94F7650DC3E0E00BC3EA8196
:102E1200E03011F4EFEFEA83A881B9810E94B17C1E
:102E220024F4A83EE3E0BE070CF006C00E94536EF5
:102E3200ED81EA930E9423665AC10E94BD7C20E084
:102E420030E0283EE3E03E077CF4A8953A932A93CB
:102E5200CDDF1E2F1F3F29F0EFEFEA933A932A931B
:102E6200D6DF2F5F3F4FEDCF0E94C47C4DC01A9337
:102E72000A93E0E0F0E0E093430CF093440CAA8163
:102E8200A03458F40E945C6EE55FFB4F8F010E94F4
:102E9200636EE3E4FCE00E946C6EE091430CF091FF
:102EA200440C23C11A931FEF1F5F1A93E0DFA9811D
:102EB200BA81EA17FB0711F0113408F001C0F4CF10
:102EC200E12F188114C11A930A93A091C20BE091C9
:102ED200C30BEA9FF001A0911E08EA0F0E2F0134E6
:102EE20008F00FE310911E08101758F41A93BFDF71
:102EF200AA81BB81EA17FB0711F4E12F03C01F5F10
:102F0200F3CFEFEF19810881249608950E94BB7CCC
:102F120010E0103418F50E94D56BE8E2F0E00E9450
:102F2200357AE050FC4FAF01E0EAEA93FA0170967D
:102F32000E94706EEC713E2FE0EAEA93FA013F962E
:102F42000E94706E0E2FEF81E31719F4EE81E017E5
:102F520009F002C0E12F03C01F5FDBCFEFEF0E9439
:102F6200C27C289608951A930A93E0918A0BAA814B
:102F7200EA17C1F0A03468F40E945C6EE050FC4F86
:102F82008F010E94746E0E946C6EEA81E0938A0B3C
:102F920009C0EFEFE0938A0B0E947F6E0E94846E5D
:102FA200E093950BA2C01A930A930E945C6EE050C4
:102FB200FC4F8F01AA81A03420F40E94746E0E94FB
:102FC200506E93C01A930A93E091B30BAA81EA1749
:102FD200A1F00E948E6E40F40E949A6E0E946C6E66
:102FE200EA81E093B30B09C0EFEFE093B30B0E94C9
:102FF200A56E0E94846EE093BE0B77C01A930A936B
:103002000E948E6E20F40E949A6E0E94506E6DC0D5
:103012001A930A93E091340CAA81EA1751F10E94A3
:10302200AA6E08F50E94636EE5E3FCE00E946C6EF6
:10303200EA81E093340CE0E0E0932B06A091360C99
:10304200A13020F0A091360CA83008F00BC0A9EDF9
:10305200BBE0E091360C0E94B46EAE0FBF1FEC9144
:10306200E0932B0606C0EFEFE093340CE0E0E09330
:10307200350C3BC01A930A930E94AA6E30F40E9448
:10308200636EE5E3FCE00E94506E2FC01A930A9330
:10309200E0912F0CAA81EA17C1F00E94B76E70F47A
:1030A200E0EAEA930E94AB6B1A930A93E0E3FCE036
:1030B2000E946C6EEA81E0932F0C07C0EFEFE09361
:1030C2002F0C0E94C16E0E94F9670FC01A930A93D7
:1030D2000E94B76E50F4E0EAEA930E94AB6B1A9337
:1030E2000A93E0E3FCE00E94506E19810881239666
:1030F20008950E94C16E0E94F967E881EF5FE09334
:10310200310CD2C124970E94BB7C0E94C86E0E94DF
:10311200F967AA85A03478F5AB85A13010F0A63006
:1031220008F007C0EB850E94B46E0E94CF6E0E9429
:10313200E26EEB85E030F9F4E0E0EE83EF83E887BE
:10314200E98740E050E020E030E02530E0E03E0753
:1031520084F4F9010E94CF6E0E94E26E0E94126E08
:103162004E0F5F1F0E94176E0E94E76E2F5F3F4F48
:10317200ECCF0E94F26E3FC11A930A93AB81A13049
:1031820010F0A63008F01CC0EB810E94B46E0E94C1
:10319200EC790E94E879DF01EA810E94036FE8E09E
:1031A200F0E00E94357AE050FA4E8F01E0EAEA93AD
:1031B2000E94A66B1A930A93EDE1FCE00E94506E06
:1031C200198108810C94CE1D0E94BD7CEC810E9465
:1031D200076FE83109F459C00E940C6F309729F04B
:1031E2000E940C6F0E94116FEC830E94881E0E2FAA
:1031F20010E0101710F00C9446190E94156F82DF30
:10320200AFE1BCE00E94B06DA091210CB091220C04
:103212008091230C9091240C0E941A6F0E94CA790B
:10322200E093210CF093220C6093230C7093240CF6
:103232000E94156FA1DFE0EAEA93EE810E94B46E6C
:10324200EE0FFF1FE050F04F0E94706EE270D9F453
:10325200ED81E093250C0E940C6F309751F40E948F
:103262000D6D0E94216FEF5EF84DDF010E94276F06
:1032720002C00E940C6FE093260CF093270C0E9470
:103282002C6F0E94316F1F5FB4CF0E94C47C2696C0
:1032920008951A930A930E94376FECE2F0E00E94BD
:1032A2003E6F0E94426F0E94476F10E01034D8F4C4
:1032B2001A9359DEE0912208EA931A9323DF0E94BF
:1032C200506FEA0FFB1F0F010E94506F0E94586F50
:1032D200DF01CB010E94176E0E94CA79D0010E94C1
:1032E200E37A1F5FE3CFA0911908A330B9F500E09C
:1032F2000031A0F50E94BA6B0E945D6F69F510E083
:103302001A3050F5E02FE05DEA93E0E2F5E10E9429
:10331200626FE12FE05D0E94696FE1F40E946E6FBF
:103322000E94756FEA0FFB1FFF93EF930E94756F68
:103332000E94586F7F936F93FF93EF930E940C61EB
:10334200AF91BF918F919F910E94CA79AF91BF9126
:103352000E94E37A1F5FD4CF0F5FCACF10E01A300A
:1033620090F40E94756F0E94586FA0912908B09145
:103372002A0880912B0890912C080E94CA790E94F9
:10338200476F1F5FECCF0C94161E24970E94BB7CE4
:10339200EA85EA936CDD9F01022E032A39F13A9302
:1033A2002A9380DD1E2F40E050E0E0E0EE83EF83C1
:1033B200E887E987AA851A17B1F4012F003498F437
:1033C2000A9355DD2E173F0761F4EB85EA930A93C2
:1033D20099DE0E94126E4E0F5F1F0E94176E0E94AE
:1033E200E76E0F5FEBCF0E94F26E05C0EB85EA93AA
:1033F200EB85EA9387DE0E94C27C2C9608951A938D
:10340200A895A981A63068F40E94C86E0E94F96747
:1034120010E0103430F4E981EA931A93ADDE1F5FB5
:10342200F8CF1881229608951A9311E0163020F4ED
:103432001A93E5DF1F5FFACF6AC3E1E0E093350C30
:10344200E093360C31C0A8950E94A56EEEEAF3E037
:10345200FA93EA930E94A66B0E947C6FE093BC0BE6
:103462000E94856FE093BD0BE0E0E093BE0B1CC0B1
:10347200A895EAE8FBE00E948C6FE9E2F0E00E9486
:103482003E6F0E947F6EE4EAF3E0FA93EA930E94B1
:10349200A66B0E947C6FE093930B0E94856FE09372
:1034A200940BE0EBE093990B219608950E94BB7C6C
:1034B2000E94916FE03228F0AAE0B0E0E0E00E94C2
:1034C2001B7B00E08BDCA091BF0BB091C00BA6333D
:1034D200E2E1BE0741F110E01A3030F41A93B3DF93
:1034E2001A938CDD1F5FF8CF10E0103430F41A937A
:1034F200BFDF1A9358DD1F5FF8CF10E0103830F4A9
:103502001A939BDF1A93B6DD1F5FF8CF8DDFA9E018
:10351200B0E0E0E00E941B7BE6E3F2E1E093BF0B48
:10352200F093C00B01E010E0183210F00C94EA1A8C
:103532000E94966F9F010E94966FAF010E94A06F3A
:103542003496E491E03011F0E13069F4D901AC91A4
:103552000E94A06F3596E491EA1720F40E94A06FB2
:103562000E94A76F34C0E23091F4DA010E94D97A46
:10357200E031A7E2FA0714F4FF2342F40E94A06F9D
:1035820036960E94E87ADA01ED93FC9320C0E3308C
:1035920049F4D901AC91AF3F21F40E94A06F0E947F
:1035A200A76F15C0E43099F4D901AC91AF3F79F41B
:1035B20000E00E94A06F3596E4910E1740F40E943D
:1035C200A06F0E94A76F2F5F3F4F0F5FF2CF1F5F69
:1035D200ABCF07DC10E0153060F41A9357DDA091F1
:1035E200300CA63020F01A9384DD1A936FDD1F5F32
:1035F200F2CFE02F0C94AD1FE881EF5FE883A88142
:10360200A43610F0E0E0E883E8810C942A200E94BE
:10361200F86CA5E0B0E00E94357A30960C942A202E
:10362200A091380CBB27E091370CA6C0F9DF329786
:1036320074F00E94AC6FE091370C0E94B36F0E944D
:10364200506EE091370CEA93D7DFE093370C089580
:103652000E94AC6FE091380C0E94B36FFA93EA9328
:103662000E9444660895E5E2FCE00E94BB6F0E945E
:10367200AC6FE091380C0E94B36F0E94506EE091E3
:10368200380CEA93B9DFE093380C08950E94BD7CB0
:10369200E0E0E093370CE093380C10E030E0343691
:1036A20080F5A8950E94AC6F3A93B1DFFA93EA9342
:1036B200E5E2FCE00E946C6E00E0A091250CA130D6
:1036C20010F0A03808F001C001E0E12FE03041F431
:1036D200013029F43093380C3093370C11E00FC0CD
:1036E200E13031F4003019F43093370C12E007C0A6
:1036F200E23029F4013019F43093380C13E03F5FC3
:10370200CECF49C21A93A091D00BA870B9F010E0A5
:10371200E981FA810E94D56BAE17BF077CF4ED8177
:10372200E093250CEB81FC81E851FC4F0E94C26FB3
:10373200E0E0F0E00E94316F1F5FEACF18810C9445
:10374200AF1FE881EF5FE883A881A43610F0E0E0C4
:10375200E883E8810C942A20E881E150E883A8817B
:10376200A43610F0E3E6E883E8810C942A20A091C5
:103772003A0CBB27E091390CF0E031960E94C76FFA
:10378200EC59FF4FDF01E4E6F0E00E94927A0895DF
:103792000E94F86CA5E0B0E00E94357AE050FE4F3E
:1037A2000C942A200E94CC6FE881EA93C0D10C9439
:1037B2002A201A9342DBE1E0E093870BA8C1A89587
:1037C20010E0143680F41A93ABD1A0912A0CAF3FCB
:1037D20031F40E94CF6FAF3FEFEFBE0711F01A93A3
:1037E200E1DF1F5FEECF0E94D46F689420F88FC193
:1037F2000E94BD7C10913A0CAD81AA23CAF5E091DA
:10380200390CE11719F0AD81AA230AF030C01A93DE
:1038120087D10E94CF6FEE81FF81EA17FB0729F45F
:10382200E885A0912A0CEA1709F01EC00E94DA6FFF
:10383200EC81FD810E94D479EA17FB0744F40E94CF
:10384200DF6F0E94E86FE0E0EC83ED830BC00E9423
:10385200DF6FEC83FD83E0E0F0E00E94E86FE0E0E0
:10386200E0932A0C1A9363D10E94ED6FC8CF46C031
:10387200E091390CE11729F0AC81BD810E94B17C45
:103882000CF01BC01A934CD10E94CF6FEE81FF81C6
:10389200EA17FB0729F4E885A0912A0CEA1709F038
:1038A20009C00E94DF6F0E94E86F1A9340D1E0E0E6
:1038B200EC83ED830E94ED6FDBCFAC81BD810E9472
:1038C200B17C1CF454DF33970CF418C0E885E09304
:1038D2002A0CEE81FF810E94F26FEC81FD810E9431
:1038E200E86FE091390CEA9322D1E091390CEA9326
:1038F20028DFE093390CE0E0EC83ED83689420F854
:10390200EC81FD810E94C47C299608951A93A091AE
:10391200450CA03059F4E091480CF091490CFA930F
:10392200EA93E8EBFBE00E94F76F09F40BC0E1E0D9
:10393200E093450CE091390CE093470CE091390C8F
:10394200E093460CA091450CA13011F00C940A1D95
:10395200E0913A0CA091470CEA1711F40C94FB1C6D
:10396200E091470CEA93F8DEE093470CEA93D8D053
:10397200A0912A0CA13010F0A03808F034C0E091D8
:10398200460CEA93E9DEE093460CA091470CEA1755
:1039920049F1EA93CCD0E091E30BE030E9F410E096
:1039A2001530D0F4ABE01A9FF001DF01E352FA4F79
:1039B200E081E03049F0FD01E452FA4FE081AE2FA0
:1039C200E091470CEA1709F005C00E94FD6FA09133
:1039D200460CA0831F5FE4CF0E94CC6FE091470C9E
:1039E200EA93A5D006C00E94CC6FE091470CEA93FF
:1039F2009ED00FC0E091460CE0933A0CE0E0E093D9
:103A0200450C689420F80E945E67E093480CF0939E
:103A1200490C7DC01A93A89510913A0CE091390C8B
:103A2200E117C1F00E9403700E94B17C64F4EB8143
:103A3200A0912A0CEA1739F40E94CF6FE981FA812A
:103A4200EA17FB0709F003C0E12F1881A6C00E9404
:103A5200ED6FE4CFEFEF1881A0C00E94DA6F0E94F1
:103A6200B17C84F4E0912B06E87031F4E0912F08E8
:103A7200A0912A0CEA1731F40E9407700E94116F7C
:103A8200E03408F001C05CC10C948820A895E09154
:103A9200390CA881EA1761F0E8810E940C7019F0D4
:103AA200E8810C942A20E881EA934BDEE883EFCF89
:103AB200EFEF0C942A201A93A89510913A0CE091FA
:103AC200390CE117E1F00E9403700E94B17C8CF482
:103AD200E0912B06E87031F4E0912F08A0912A0CB6
:103AE200EA1739F40E94CF6FE981FA81EA17FB07DE
:103AF20009F002C00C946F200E94ED6FE0CFEFEF4F
:103B02000C9470201A9310913A0C1A93BFDF1991FA
:103B12000895E881EA9315DEE883EA93B7DF99C254
:103B22000E94AC6F0E9413700E946C6E92C20E943F
:103B3200AC6F0E9413700E94506E8BC20E94BD7CBB
:103B42000E94D46F10E030E0343628F5A8953A93FD
:103B5200E7DF00E0A0912A0CA03808F401E0E12F91
:103B6200E03041F4013029F430933A0C3093390CAF
:103B720011E00FC0E13031F4003019F43093390C08
:103B820012E007C0E23029F4013019F430933A0C04
:103B920013E03F5FD9CF0E94C47C249608951A9304
:103BA2000A93A0911908A43009F43FC010912F087C
:103BB2000091540CE0913108E03059F0E0932F0865
:103BC200689424F80E941C70E0E0E0933008E0E57D
:103BD20020C0E0913008E03021F0E0932F08E2E5C8
:103BE20018C0E0E0E0932F08E093540CE091C50B7D
:103BF200E03031F0E091C50BE150EA930E940918E0
:103C0200A091350CA17039F0E091C50BE0932F081B
:103C1200E4E4E093540CA0912F081A1721F4A09128
:103C2200540C0A1711F0689423F809911991089518
:103C32000E942270EBE0EC93EC81D8011696EC9393
:103C4200EB81D8011796EC93D8011896E0E0F0E0EA
:103C5200ED93FC93D80112960E942F70D80114960E
:103C62000E942F700E94347001C10E942270ECE009
:103C7200EC930E94347034C21A9318E0113108F5A3
:103C8200E0911408F0911508A981BA81EA27FB276F
:103C9200BF010E944070E623F723309781F00E9413
:103CA2004070A981BA81EA23FB23309731F01A933D
:103CB200E0E0EA931A93BCDF02C01A93D6DF1F5FDB
:103CC200DDCF0DC2A0911B0CA93030F0E0915C0C4D
:103CD200A0915B0CEA1709F414C0E0915C0CE0308F
:103CE20021F4E3E6EA93C1DF08C0E0911B0CEA93FA
:103CF200E0E0EA93E3E6EA939BDFE0915C0CE09379
:103D02005B0C0895A0919B0BECE1EA230895A0912E
:103D12009B0BA07411F0E2E00895A0919B0BA07898
:103D220009F0F5C10DC0A0918A0BAF3F09F4EFC1B4
:103D3200E9DFE43009F4EBC1E5DFE03109F4E7C182
:103D4200E1E008950895A881AF3F11F4E0E081C158
:103D5200D9DFE43011F4E1E07CC1E0E07AC1A8816E
:103D6200A23019F4CFDFE83011F0E1E072C1E0E0F7
:103D720070C1A881B981AC91A130A8F0A881B981A4
:103D8200AC91A43180F4A881B981EC910E944B706E
:103D9200EB5FFC4FE081EF770E2EA881B98112967E
:103DA200EC91E01509F002C0E1E011C1E0E00FC1C1
:103DB200A881A13118F0E881E051E883E8810E94EE
:103DC20050700E945A70A091D10BA13018F0A881B6
:103DD200A43009F006C0E6E9F0E00E94E87A0E9409
:103DE2005A7037C1A881A13010F0A63008F006C081
:103DF200E8810E946570E15CF94F2AC1E0E029C1C7
:103E0200A881A13010F0A63008F006C0E8810E9417
:103E12006570EC5BF94F1CC1E0E01BC10E94BD7CE8
:103E2200EC81EA93EDDFEF731E2F1030E1F0EC81AD
:103E3200EA93E6DFE0743E2FE12FE150A1E00E9419
:103E4200E079A0912306EA230E2F303011F40030DE
:103E520009F002C0E1E008C0303011F0003009F48E
:103E620002C0E1E001C0E0E00E94C47C2596089512
:103E72000E94BB7C00E00530A0F50A930E9447181F
:103E82000E946A70A7E10A9FF001EE5CF94F0E945E
:103E92008C6FE4E1F0E00E943E6FE091310CDA01B8
:103EA2005096EC93A091300CEFE3EA23AE2FE09111
:103EB200330CE295E07FEE0FEE0FEA0FDA01559632
:103EC200EC93E091310CE1503E2F3F3F41F0E09105
:103ED200320C0E94216FDA015196ED93FC930F5F31
:103EE200CACF10E01034C0F51A930E94B4171A9387
:103EF2002ADFE13079F5E0919E0BEA9373DFE1501E
:103F02000E2F0F3F39F10E946A70E12FDA011396EA
:103F1200EC93E0919E0BDA011496EC93E091A40BE2
:103F2200F091A50BDA011696ED93FC930E941A6F9D
:103F3200A4E6B0E080E090E00E943A7ADF01CB0193
:103F4200E091A40BF091A50B0E94786DDA011A960C
:103F5200ED93FC931F5FC6CF0E94C27C2696089504
:103F6200A0911908A23031F0A83021F0A73011F049
:103F7200A53009F40AC00E94376FEFEFF0E00E940B
:103F82003E6F76DFE0E0E093A20608951A93E9819E
:103F9200E058E98310E01530C0F4A3E21A9FF00163
:103FA200EB55F94FE081AE2FE981EA1749F4F001B0
:103FB200EC55F94FE081AE2FE0912F08EA1709F096
:103FC20002C0E12F03C01F5FE6CFEFEF18812296F8
:103FD20008950E94BD7CED81EA93D8DF1E2F1F3F1A
:103FE200F1F0A3E21A9FF001ED55F94F9F01D901BB
:103FF2001296EC91EF77EC93EC81D901EC930E944D
:104002004B70EF5EFC4FBF01E081EF77DB01EC9379
:10401200EC810E944B70E15FFC4FA1E0A083E12F95
:104022000E94C47CE4C40E94F86C0E94717061F426
:10403200E0914E0CEF5FE0934E0C0E94F86CED5550
:10404200F94FA0914E0CA0830E94F86CED55F94FE8
:10405200E081219608951A931FEFE091D50BF0911C
:10406200D60BA981BA81AE17BF073CF0E091D70BFE
:10407200F091D80BEA17FB070CF412C00E9476707D
:104082000E94F7161E2F103031F01F3F21F0E091F1
:104092002F08E11729F4E1E0E0935C0CE0E01FC097
:1040A200E0E0E0935C0C1AC01A930E947670D3DFB2
:1040B2001E2F103099F01F3F39F4E4E2F5E1FA9334
:1040C200EA93EB81FC8106C0E4E3F5E1FA93EA931B
:1040D2000E947B70FA93EA930E941E10E12F1881CE
:1040E20023960895E0916505E03009F00895E09186
:1040F2002C06E03009F008950AC0E0916605E03030
:1041020009F00895E0912D06E03009F00895E0E00D
:1041120008950E94BD7CE0912606F0912706AC81AD
:10412200BD81EA27FB279F0110E0153090F4F901C9
:10413200E17049F0A7E11A9FF001EF5CF94FDF014E
:10414200EC91EF5FEC93D9010E947E709F011F5F9B
:10415200ECCFEC81FD81E0932606F09327060E94C6
:10416200C47C45C428970E94BB7C3091260610E08F
:104172001530B8F5A7E11A9FF001EB5BF94F00810A
:10418200E12FA1E00E94E0792E2FE22FE32391F0AC
:10419200003810F0003C08F001C00F5F003C31F421
:1041A200E22FA0912306EA2BE0932306003808F4BD
:1041B20000E80FC0003408F40F5F003439F4EFEF69
:1041C200E227A0912306EA23E0932306003808F0B1
:1041D20000E0A7E11A9FF001EB5BF94F00831F5F3C
:1041E200C7CFE0E0E0932C06E0E0F0E0E0931608B1
:1041F200F0931708E0915C0CE03021F0E0911B0C89
:10420200EA93D6DDE0911D08EF5FE0931D08E0918F
:10421200E40BA0911D08EA1751F4E091E40BF0E0E1
:10422200A0E0B1E00E94FC7AEA1BE0931D08A09195
:104232001908A13019F0A93009F096C0A091630BBA
:10424200B091640BE4E1F0E00E94927A309719F4A5
:10425200E1E0E0931F0846DFE03019F04EDFE0783E
:1042620009F462C04ADFEF775E2F5A930E94B417B7
:104272000E94456CED55F94F5081503011F40C9469
:10428200952151DDE13031F4E0911A08EA9367DDBE
:10429200E03009F449C00E9483700E94036FEC91E0
:1042A200EC71EC3021F4E0911D08E07851F40E94A9
:1042B2008870EC91EA937CDD0E948D70EC91EA9318
:1042C20077DD0E948870AC91A63070F5A3EEB6E05F
:1042D2000E94456C0E94FB6C0E94B06D0E94887027
:1042E200EC91EA937FDD1E2F1130F0F00E94927064
:1042F2000E949570CF010E9492700E94FB6C6D919A
:104302007C91E12F0E946570EF5CF94F0E949A70D8
:10431200E60FF71FDC01ED93FC93E12F0E9465701D
:10432200EF5CF94FA0E0A08310E01530E8F40E94A2
:104332009D7013965C915F3FA9F05A9374DE5E2FD5
:104342000E94A7700E9492700E949570BF010E9405
:1043520092700E94FB6C0E94AD70AE81BF8112967A
:10436200E0E0EC931F5FE1CFA0911908A23039F091
:10437200A83029F0A53019F0A73009F0EAC1E0E031
:10438200E093200800E0053010F00C94AA23A3E289
:104392000A9FF001ED55F94FEA87FB87AA85BB8595
:1043A200AC91A03019F0A281A07809F0D0C1E091BF
:1043B2002008EF5FE0932008AA85BB8513960E9430
:1043C200D97A309771F0AA85BB8513960E94BA708C
:1043D2000E94C07029F4AA85BB8513960E942F7093
:1043E200B6C18BDEE03021F00E94C07009F4AFC18B
:1043F20020E030E0333010F00C9455230E94CA7054
:10440200DF010E94D26B0E94CF6CE887F987A181FD
:10441200A27021F4A481B581109709F410C1E88536
:10442200F985A181A47011F40C947722A181A8705E
:1044320021F40E949132E03009F457C00E94D070FA
:10444200EBE0EC93A885B9850E94DD70A885B9855B
:104452001396EC91AC85BD851796EC93EC85FD85A2
:1044620038960F01E885F985A181E1E0EA230E94EF
:10447200E470ED93FC93A885B98514960E94D97ACD
:10448200AC85BD851296ED93FC930E94E770AC85D6
:10449200BD851496ED93FC93A02FEAE0EA9FF0010C
:1044A200E30FEF5F0E94ED70E885F985A085B18585
:1044B200E2E0F0E00E94357AA885B9851896ED937E
:1044C200FC930E94E770309739F4A885B985189655
:1044D200E8EEF3E0ED93FC93E885F985A181E8E04D
:1044E200EA2BA885B9851196EC936EC0E885F9850B
:1044F200A181A17031F4A885B98514960E94BA7081
:1045020043C00E94F6706EDCE1501E2F0E949D7027
:104512001296EC91E03001F5AE81BF8153960E9474
:10452200B06DEE81FF81A189B289109751F00388A5
:104532001488AE81BF8151960E94D97AE015F105A7
:104542000CF009C00E94256C14DCE03011F00E94CE
:10455200FB700E9403710EC0E885F98534960E94B3
:104562000B710E94E4700E94C76F0E9413715396F0
:104572000E942F70E885F985A581AA232AF4A885CF
:10458200B98514960E942F70A885B985EC91EC71BB
:10459200EC3021F4E0911D08E078B1F4E885F9856A
:1045A200A481B5815E971CF4A181A07209F404C0B4
:1045B200E885F985A28106C00E94F670F9DBE885DC
:1045C200F985A381AA93F4DB0E94E770309791F0FA
:1045D200A885B98518960E94BA700E94E770309734
:1045E20049F40E94256CC5DBE03011F00E94FB709B
:1045F2000E9403710E94F67011DCE03001F10E940A
:10460200256CB7DBE03049F00E94FB70AA85BB85C0
:10461200EC910E944B700E944D6CAA85BB8512964C
:10462200EC91E058AA85BB851296EC93E3E0E09307
:1046320024060E94F670E4DBEF73E0932506A8855A
:10464200B98514960E94D97A309761F52F5F32307E
:1046520048F5A885B98516960E94D97A309789F0CF
:10466200E885F985A681B7810E941A71AA85BB8562
:104672001396ED93FC93A885B98516960E942F7028
:1046820011C00E94CA70DF01E32FEF5FF0E00E94C9
:10469200CF6CE887F987A181EDEFEA23A885B98578
:1046A2001196EC933F5FA6CE233011F00C94A82311
:1046B2000E949132E03069F00E94D070E8E0EC9301
:1046C200AA85BB850E94DD70AA85BB85EC910E94FC
:1046D200ED700E94256C4DDBE03011F00E94FB7002
:1046E200AA85BB85E0E0EC93EA85FB85A581ECE138
:1046F200EA23E83061F50E940D6DAE2FEA85FB8555
:10470200E38DEA1741F4EA85FB85E48DE150EA93F3
:104712000E94B7161CC00E949132E030C1F00E9484
:10472200D070E3E0EC93AC85BD85EFEFEC93189687
:10473200EA85FB85E38D0E941F71AC85BD851296CB
:10474200EA85FB85E48D0E941F710E9423710F5F31
:104752001ACE0E94297149F4A0911908A23021F0C1
:10476200A83011F0A53009F401C050C010E0153096
:1047720010F00C9407240E949D7013965C915F3F89
:1047820011F40C9405240E94A770AE81BF81BD0173
:104792000E94AD70EE81FF8138960E940B710E94DB
:1047A2002F710E9413710E94D97ADF010E94B17C9D
:1047B200B4F4EE81FF81A681B7810E94B17C7CF4C2
:1047C200AE81BF810D901C90AE81BF8116960E9472
:1047D200D97AD001AE1BBF0B0E94B17C0CF014C081
:1047E200AE81BF81BD010D901C90EE81FF81A6813B
:1047F200B781F001EA1BFB0BDB01ED93FC935A93AB
:10480200E5E0EA930E94E7411F5FB1CFE0911C0807
:10481200E03041F4E0911608F0911708E093140893
:10482200F09315080E94C27C2E9608950E94BD7CCA
:10483200A091C20BE091C30BE150EA9FF001EF5F40
:104842001E2F2FE330E000911E08A091190CA13019
:1048520080F0E091190CE150A0911E08AE1728F0EB
:10486200E091190CE1503E2F04C0E091190CE25086
:104872002E2FEC81E03049F1EF3F51F4A0911E0858
:10488200A11BA31720F0E0911E08E11B0E2F1DC0F3
:10489200EE3F59F4E12FA0911E08AE0FA21720F4AB
:1048A200A0911E08EA0F0E2F10C0EC3F49F4A09110
:1048B200190CA13020F0E091190CE1500E2F05C027
:1048C200AC81A1501A9FF0010E2FE0911E08E01753
:1048D20051F00A930E94B417A0918B0BAD3209F4E8
:1048E200032F00931E080E94C345A0911908A83007
:1048F20019F40E94320E02C00E94AB0D0E94C47CC9
:10490200259608950E94BB7CFDD9E03111F40C94E8
:10491200F52420E030E040E050E010E0133060F594
:104922000E9433710E94FB6C0E94D97A309711F178
:104932000E9436710E9450702E2B3F2B0E943671BE
:10494200EA936CDAE03029F0E3E0E0932406E0E059
:104952004CC00E943D710E9450702E2B3F2B0E9432
:104962003D71EA935BDAE03029F0E3E0E09324065C
:10497200E0E03BC01F5FD2CF00E0053058F5A3E274
:104982000A9FF0010E94717019F110E0133000F5D6
:104992000E94CA70DF010E947B700E944471AE0FB8
:1049A200BF1F1296EC910E9450704E2B5F2B0E94FB
:1049B200CA70DF010E947B700E944471AE0FBF1F5C
:1049C2001396EC910E9450704E2B5F2B1F5FDECF2F
:1049D2000F5FD3CFF901E423F523309729F0E1E00B
:1049E200E0932406E0E001C0E1E00E94C27C26964A
:1049F20008951A93E091520CE03011F40C944F2573
:104A0200E091E50BE13059F4A091520CA13311F47D
:104A1200EFE001C0E0E0EA930E94535D3FC0E23064
:104A220059F4A091520CA13311F4E6E001C0E5E182
:104A3200EA930E94535D32C0E53061F4A091520CBA
:104A4200A13319F4E0919A0B01C0E0E0EA930E94CD
:104A5200535D24C0E330B1F410E0173040F40E94FB
:104A62007B70E05CF64F0E944B711F5FF6CFA09106
:104A7200520CA13311F4E1E301C0E0E3EA930E9496
:104A8200535D0CC00E944F71E9E4EA930E94AF614A
:104A9200E091520C0E9456710E945B718FC4229762
:104AA2000E94BB7C30E0A0911908A23029F0A83006
:104AB20019F0A53009F021C1A985A03410F00C9499
:104AC2007D26E0912F08E03009F417C1E9850E94A4
:104AD200076FE03131F4E1E3E093520C8ADFE1E069
:104AE2000CC121D9E03009F408C110E01530A0F45E
:104AF200A3E21A9FF001DF010E94717041F0FD01F3
:104B0200EB55F94FE081AE2FE985EA1709F002C0B3
:104B1200E0E0F3C01F5FEACFF5DEE03011F40C9461
:104B22007D2610E0A3E21A9FF001ED55F94FEE83C6
:104B3200FF83AE81BF81EC91E03011F00C947626B8
:104B420013960E942F7000E0033010F00C9445265B
:104B5200A3E21A9FF001E855F94FDF010E94BA6BF8
:104B62000E94CF6CAF01DA0116960E942F700E944C
:104B72006071DA011296EC930E946771DA01139662
:104B8200EC93A0919B0BEEEFEA23DA01EC930E94E7
:104B92006E71DA011196EC93B5D8E43139F0FA016D
:104BA200A181E2E0EA2BDA011196EC930A93D7D8BD
:104BB200E03011F40C942726FA01A281AA9312D9AB
:104BC200E1502E2F2F3F81F0A7E12A9FF001EF5CE9
:104BD200F94FA0E0A083A7E12A9FF001EE5BF94F15
:104BE200A0E0B0E0A083B1830E9476710E94FB6CCA
:104BF2000E94D97ADA011496ED93FC93013040F0C9
:104C02000E9476710E94FB6C0E94D97A309709F05B
:104C12000EC0AE81BF811596E02F0E94B46E0E9435
:104C22004471AE0FBF1F1196EC91E062EC93AE811E
:104C3200BF815A96EC91E062EC93023030F40E940C
:104C42007971DA0116960E941F7104C0DA01149676
:104C52000E942F7057D8EC3019F4E0E0E0931D0861
:104C62000E9480710E94216FDA011896ED93FC93E5
:104C7200FA01A281A63030F0A181E4E0EA2BDA0148
:104C82001196EC930F5F60CFA0911908A23011F03A
:104C9200A53019F4A885AF3F08F007C0E0912F08AE
:104CA200EA93EA85EA930E94E518E885AE81BF811E
:104CB200EC93E0912F08AE81BF811196EC93E985C8
:104CC200AE81BF811296EC93A885A43138F4E885B1
:104CD2000E944B70E15FFC4FA1E0A083AE81BF81D7
:104CE2001696EC91ED7FEC9331E01F5F303011F4BA
:104CF200153008F001C016CFE32F0E94C27C2A961D
:104D020008951A930A93A0911908A23011F0A530C0
:104D120021F40E9487710E94CB6DA0911908A830DE
:104D2200C9F40E948771E1E0EA930E942546E0916E
:104D3200E30BE03069F4EA810E949271E081EF773F
:104D42001E2FABE01A9FF001EA51FA4FA0E0A083B8
:104D5200689420F8198108812396089564970E9427
:104D6200EE6BA23039F4E0912F08EA93EB8DEA93CF
:104D72000E94E518A0911908A83011F00C9425277B
:104D82000FEF20E0253050F4A7E12A9FF001EE5CFE
:104D9200F94FE081AE2FEA8DEA1709F402C02F5FC6
:104DA200F1CFA7E12A9FF001E15DF94FAF01DA01EE
:104DB20015960C910F3F11F40C9425270E949871BF
:104DC20010810E9403700E94B17CECF4ADE2BCE061
:104DD2000E94BA700E949E710E94DA6FA083B18312
:104DE2001A930E94981DABE00A9FF001E252FA4F1B
:104DF20030810A93FE0137960E94A4713A93FE0114
:104E020037960E94A8710E94AE71F1F40E949871C7
:104E1200AFEFA083DA011396EFEFEC93DA01159668
:104E2200EC930E949E710E94B471E0E0F0E00E9457
:104E3200E86FE0E0E0932A0C1A930E94981D0A930F
:104E42000E949A0F689420F80E94C27C6B96089583
:104E52001A9310E01031B0F4A7E11A9FF001EC5B55
:104E6200F94FE081EF73AE2FE981EA1729F41A9323
:104E72000E940F1FE03009F403C0E1E01881E0C096
:104E82001F5FE8CFE0E01881DBC01A93E091550C78
:104E9200F091560CFA93EA93E4EFF1E00E94F76F77
:104EA200F9F00E94B97110E01530D0F4A091590CBC
:104EB200AF5FE5E00E948F7AE093590CEF5FEA93CF
:104EC200C7DFE03059F0E3E0E0932406E091590CAB
:104ED200F0E0EF5FFF4EE093250670C21F5FE4CF64
:104EE2006DC21A93E0912306E093510CE8E7F0E0DB
:104EF200FA93EA93ECEDF0E0FA93EA930E94F44518
:104F020010E01530D8F4E12FEF5FEA93A1DFE03033
:104F120099F00E94466BE12FEA5FF0E00E94096D72
:104F2200E1E4F5E10E94A76CA7EEBBE00E947B7072
:104F32000E94CF6C0E94D76C1F5FE3CF3FC2A5DFF8
:104F4200E0912406E13029F4E9E4F5E10E94C07120
:104F52003CC0E23029F4E6E5F5E10E94C07135C0BB
:104F6200E33051F4E1E4F5E1FA93EA93E0912506A6
:104F7200F0E0E050F04F29C0E43019F4EEE5F5E13D
:104F82001FC0E53031F4E0912506EA930E9401103A
:104F920020C0E63019F4E6E6F5E112C0E73029F464
:104FA200ECE6F5E10E94C07110C0E83029F4E8E7B0
:104FB200F5E10E94C07109C0E93059F4E7E8F5E172
:104FC200FA93EA93E0912506F0E0FA93EA930E94BD
:104FD2001E10E0E0E09324060895A881B98111969D
:104FE200E1E0EC930E940770A881B9811296ED93DB
:104FF200FC930E94881EA881B9811796EC930E94A7
:105002000D6DA881B98118960E941F71E091C605A5
:10501200A881B981EC93E0912A0CA881B9811696F6
:10502200EC93E0918A0BA881B9811A96EC93E091F6
:10503200AD0BF091AE0BA881B9811496ED93FC9360
:105042002296089564970E94BD7CA091E30BA23042
:10505200E1F4EB8DEA930E94B4170E94881EADE240
:10506200BCE00E941F71ABE2BCE0EB8D0E941F719D
:10507200E0912F08E0932A0C0E940C6F309721F0E8
:105082000E940C6F0E94F26F14C0AA8DAF3F09F408
:10509200CAC0EA8DEA930E94911DAB8DAF3F29F4FD
:1050A2000E9407700E94116FEB8FEB8DEA930E94B2
:1050B200B4170E94881E0E2FA98DAF3F21F00E94C7
:1050C200941EE03009F001C0AEC00E94DA6F0E9467
:1050D200BA6BAE17BF071CF015DCE13009F0A3C0B4
:1050E200A091D20BA03021F4A091E30BA23011F5D4
:1050F2000E940D6DE13041F00E949132E03021F0CA
:105102000E94A732E03009F002C00E94C5710E94DD
:105112000D6DE13021F40E949732E03009F409C0AC
:105122000E94D171EE55F84FFA93EA9356DF0E942E
:10513200D77177C0EB8DEA93EA8DEA93B0DC1E2F2C
:10514200113011F00C941229A091D40BA13059F412
:10515200E0912F08EA930E940770FA93EA93EFEF27
:10516200FFEF0E94DD710E94DA6F0E94BA6B0E940B
:10517200C76F0E94E86F689420F8A091E30BA030FB
:1051820019F4A88DAF3F09F437C00E94E171EE51C6
:10519200FA4F0E94DA6FA083B183E88D0E94B06C4F
:1051A2003081E88DEA93FE0135960E94A471E88D64
:1051B2000E94B06CE081EA93FE0135960E94A871CC
:1051C2000E94831EE03131F00E94E171EA51FA4FF0
:1051D200A1E005C00E94E171EA51FA4FA2E0A0836A
:1051E2000E94E171EC51FA4FFF93EF930E945E67C8
:1051F200AF91BF91ED93FC930E94AE7119F4E0E080
:10520200E0932A0CEA8DEA930E94981DE0912F0800
:10521200EA930E940C6F0E94E671FA93EA930E944D
:10522200831BE1E001C0E0E00E94C47C6C9608951B
:1052320069DBE13041F40E949132E03021F00E94BA
:10524200A732E03009F007C00E940C6F0E94F26F93
:105252000E94C5712FC337C30E94BD7C0E94E971B1
:105262001F3F11F40C948429E091520CE03011F0AC
:105272000C9483291A930E94B417E5E0E093240664
:1052820010932506A0911908A23031F40E94F27100
:105292000E945520E03009F010C0A091530CA133B8
:1052A20031F4E0912F08EA931A930E94E518E1E3A2
:1052B200E093520C0E94C47CEBC2A0911908A83062
:1052C200A1F40E940C6F0E94F6710E2F0A930E94A5
:1052D20009333E2F1A930A93EFEFEA933A93B2DE21
:1052E200E03019F00E94C47CD3C2A0911908A53005
:1052F20031F49EDFE03019F00E94C47CC9C2E0E3C1
:10530200E093520C06C0E0E3E093520CE4E0E09339
:1053120024060E94C47CBCC2E09140090E94FA713A
:1053220008951A93E6E0EA930E94535D0E944F713A
:10533200A0914009A83539F4E3E9F5E10E9406722B
:10534200E0E00E945B71A0914009A33509F510E0ED
:10535200A0911908A83021F0A23011F0A53009F46B
:1053620011E3E3E5EA930E94AF611A930E94AF61F1
:10537200E0E8EA930E94AF61E0E8EA930E94AF613D
:10538200E0E80E945671E093520CE0E00E945B71EB
:10539200A0914009A93491F4A091E50BA43019F42D
:1053A200E0E0E093520C0E940A72E09325060E940C
:1053B2001472EC91E093530C4FDF1BDB19910895AB
:1053C2000E94BD7CA0913F09A53411F00C94282ABB
:1053D2000E941972E2E3F0E0E0934C0CF0934D0C62
:1053E200A0914009A73741F4E4E4F9E00E94207259
:1053F2000E9425720E94FA71A0914009A03310F018
:10540200AA3308F023C02091270830912808E0E44D
:10541200F9E00E942072E2E0EA930E9456610E2FA8
:105422000E942572E09325060E9425720E9429722D
:105432000E94E9710A931A930E94E51820932708A3
:1054420030932808E2E5EA930E94535D1CC0E09184
:105452004A0CF0914B0CFA93EA93E0914C0CF091C8
:105462004D0C0E94F76F79F0E0E0E0933A09E5E431
:10547200EA930E94535D0E941972E8ECF0E0E09317
:105482004C0CF0934D0C0E94C47C02C20E94896CA9
:105492000E944A0D0E942E720E94466B0E94466B29
:1054A2000E949C45A0911B08A23021F4EBE9F5E192
:1054B2000E94A76CA0911B08A13021F4E2EAF5E159
:1054C2000E94A76CE0911B08E03021F4E9EAF5E1C3
:1054D2000E94A76C0E9438720E94786B0E949C45C1
:1054E2000E943B720E944072FA93EA93E0915F0538
:1054F200F09160050E9446720895E1E003C0E0E089
:1055020001C0E2E0E0931B08C1DF08950E94831E00
:10551200EC3109F0D8C1E0919A0BE33631F4A09155
:105522001908A23009F4EBDF17C0E23631F4A0917A
:105532001908A23009F4E5DF0FC0A091C505A23019
:1055420011F0A63021F4E0919A0BEA936FD9A09161
:10555200C505A43009F4D1DFADC10E94DD6C0E9403
:10556200466B0E94E16C0E94466B0E94466B0E9451
:105572009C45E8E7F5E00E94A76CE0911A080E94BA
:105582004A72E6E8F5E00E94A76CE2E0E0930E04BE
:1055920008950E94376FE0ECF0E00E943E6FE881D0
:1055A200E03009F406C0A0911A08AF5FE3E00E9460
:1055B2008F7AE0931A08E1E0E0934E0C0E94391FC3
:1055C2006FC20E94BD7C10E0103410F00C942F2B9F
:1055D2000E947B70ED55F94F30813F3FE9F11A93FC
:1055E2000E94B41700E00E944E720E94FB6C0E945F
:1055F200D97A3B9794F00E9451720F010E944E7229
:105602000E94FB6C0E9457720E945D720E94036F9F
:10561200EC91EE7FD001EC9301E00E9462720E9455
:10562200FB6C0E94D97A759794F00E9451720F0117
:105632000E9462720E94FB6C0E9457720E945D720D
:105642000E94036FEC91E160D001EC9301E0013024
:1056520019F41A930E94D4171F5FB6CF0E94C47C1C
:1056620017C11A930A9323FE03C00E9465722CD7B6
:105672000E94F741E030C1F1E0E00E946C72103804
:1056820020F5113219F40E9465721ED71D3439F4C7
:105692000E9473720E94D462E3E0E09318081B3206
:1056A20071F40E947872EAE2EA93E4EBF5E1FA938C
:1056B200EA93E0911A08E05DEA930E94D4621F32F5
:1056C20019F4E1E0EA93B2D848DF103868F00E949A
:1056D2007E721A930E94142019DFE03011F4103206
:1056E20008F002C0E0E5F5E20E947E200E2F0038AD
:1056F200C8F10F770034A8F5E0911F08E03031F0CF
:105702000A930E946F10E0E0E0931F08E0915A0CA8
:10571200E01739F10A930E94B4170E948870AC9185
:10572200A83028F40E948D70AC91A830A8F0E02F28
:10573200EF5FE093A2060A930E9414200E948870F1
:10574200EC91EA930E948D70EC91EA93E091A206AB
:10575200EA930E94191E03C0E0E0E093A2060093C0
:105762005A0C0EC0A0915A0CAF3F51F0E091A20624
:10577200E03019F0EA930E94361EEFEFE0935A0CE4
:10578200099119910895A881A03310F0AA3308F065
:105792001DC00E9482720E948772AAE0B0E00E943D
:1057A200357ADF01E8810E948C72EA0FFB1FE093D9
:1057B2002508F0932608E2E0E0930E040E94387276
:1057C2000E94786B0E94E16C0E943B72A881A33414
:1057D20051F40E942E720E9438720E94786B0E94CD
:1057E200E16C0E943B725CC11A930A93A0E023FC15
:1057F200A1E0A03019F0AA81A03009F016C0E89407
:1058020023F8E7E0E09318080E94DF44A0913108F2
:10581200A03019F40E948F7209F407C0E7E0EA93FE
:105822000E94947251D6E89424F824FE24C00E9467
:105832009772EAE5F0E00E949E7219F0AA81A13007
:10584200C9F46ED6E030B1F00E94A4720FEF1FEFE0
:105852000E94F2710E942C20E03021F4009127086E
:1058620010912808EB81EA93E0912F08EA931A93AA
:105872000A932AD60BC00E949772ECE2F1E00E94D2
:105882009E7221F40E94AB72E09330081981088164
:1058920024960895E091C80BF091C90B0E94AF7253
:1058A20011F4E2E00895E091C60BF091C70B0E945B
:1058B200AF7211F4E1E00895E091CC0BF091CD0BC1
:1058C2000E94AF7211F4E0E00895EFEF0895E0E076
:1058D200E0931B08A0911908A23021F40E94C3454D
:1058E2000E94AB0DA0911908A83009F44CD6A091E2
:1058F2001908A53009F443D10895E2E0EA930E9421
:10590200C33FE2E0E0930E04E881EA933CDFA88122
:10591200AF3721F4E0912B06E37009F403C0E2E013
:10592200E0931808A881A13239F0A33421F40E942F
:105932008272109709F004C0A0911908A23009F0F0
:105942000FC0A0911B08A33009F4DBDDA0911B0856
:10595200A23009F4BCDFE0911B08E03009F4CFDD8E
:10596200A881AD3311F00C940D2D0E94DF44E0911B
:105972001B08E030A1F4E0912508F0912608FA9383
:10598200EA930E945520E03041F4E0912508F0911D
:1059920026080E9429729BDF01C0B1DD3DC0E130C3
:1059A20069F478DFEF3F41F0E3E00E94B3720E94B6
:1059B20073720E94B97201C08ADF2EC0E230F1F424
:1059C2000E948272A034E0E0BE07B4F4E0912508A0
:1059D200EA930E94C072E2E0E0930E040E94466BDA
:1059E2000E94466B0E949C450E949A6C0E94010F85
:1059F200E3E0E0931B0801C084DD0EC0E33061F4F4
:105A0200E0912508EA930E94B417E0912508EA93F1
:105A1200EEEFEA9344D875DDA881AD3409F46DDD6B
:105A2200A881A43521F4A0911908A23009F001C07F
:105A320066DDA881AB3221F4EEEFEA930E941724CF
:105A4200A881AD3221F4EFEFEA930E941724A881D6
:105A5200A73421F4E1E0EA930E941724A881AB3431
:105A620021F4ECEFEA930E9417241AC00E94B11F9E
:105A72000E94C345E0E0E0931B08A881A13039F4FD
:105A82000E948F7221F0A091CB0BA03009F402C0CA
:105A920036DD06C00E94AB0D0E94F2710E942C20DE
:105AA200219608951A930A930E94C4720E94631E5B
:105AB2000E94F741E03091F10E94CD7278F10E948C
:105AC2007E7224DDE03051F50E94D5720E94EA1FF9
:105AD200EF3F09F0F6C40E94F2710E945520E030B7
:105AE20021F40E94941EE13009F018C00E94831E26
:105AF200E83119F40E94DA7209F001C0E2C40E948E
:105B0200D5720E9450250E2F013021F4A0919A0BDC
:105B1200A03009F403C01A930E940110A0912E062E
:105B2200AF3F61F110912E06EFEFE0932E061A932C
:105B32000E94B4170E94F2710E945520E03021F4B5
:105B42000E94941EE13009F019C00E94831EE831C0
:105B520019F40E94DA7209F001C0B3C41A93EEEF8D
:105B6200EA930E9450250E2F013021F4A0919A0B46
:105B7200A03009F403C01A930E940110A2C40E942B
:105B8200B11F0E94391FE89421F8E0E0E0931E085B
:105B92000E94E1720E94C3450E94466B0E94466BBE
:105BA2000E949C45E09132060E941E6DE0913306F0
:105BB2000E941E6D0E94466B0E94A26C0E949C4530
:105BC200E0913F060E941E6DE0913906F0913A067F
:105BD2000E94F46C08950E94BD7C0E94C4720E94CF
:105BE200F741E03049F00E94CD7230F00E947E729F
:105BF2008DDCE03009F41CDBE091570CF091580C7D
:105C02000E94CF6D11F40C94662E0E94E1720E94E4
:105C1200466BE2E0F0E00E94E872E0913706F09114
:105C220038060E94F46CE0913B06F0913C060E941B
:105C3200F46C00E0053010F00C94662EA7E10A9F88
:105C4200F001E15DF94F9F01F901A381AF3FD9F165
:105C5200D9011A960E94006D7F936F93FF93EF9381
:105C62000E94EB72AF91BF918F919F910E94F77941
:105C72000E943A7ADF01CB010E94F072D9011C9690
:105C8200ED93FC93F90104841584D9011E960E94B8
:105C9200D97AE015F105B9F0F90104841584A685D5
:105CA200B785F001EA1BFB0BE093AD0BF093AE0B53
:105CB200BFDAE13041F4D9011C960E94D97AD901A8
:105CC2001E96ED93FC930F5FB5CF0E94C47C1AC45D
:105CD2000E94BD7C0E94C4720E94631E0E94F74112
:105CE200E03011F40C94FF2E0E94FA410E2F0A9319
:105CF20004DE003820F0A091C605A03808F429C0BF
:105D02000F770A930E94F7720E94F6711E2FA091DC
:105D1200E30BA03011F41F3F09F416C030E0353018
:105D220098F4ABE03A9FF001E452FA4FE081E117B8
:105D320049F43A9FF001E252FA4FE081EF5FE093BB
:105D4200C605232F3F5FEBCF0A930E94D5722A9399
:105D520054C0A091E30BA03021F4003810F00538B4
:105D620008F00AC00F770E9498711081EFEFEA9352
:105D72000E94D5720A9366D9A091E30BA03011F06C
:105D8200003808F43BC00F770A930E94B417BEDBB9
:105D9200E030A1F50E94FA720E94EA1FEF3F19F06B
:105DA2000E94C47CAFC30E94941EE13039F50E9468
:105DB200881EE03049F40E94FA720E945025E030B9
:105DC20011F00E94FF721AC00E94831EE83141F452
:105DD2000E94DA7221F00E94FA720E9450250EC0CF
:105DE200A0911E08E02F0E946D6CAE0FBF1F1C9188
:105DF2000A930E94D572EFEFEA9324D9A0912E065E
:105E0200AF3FF9F000912E06EFEFE0932E060A93D2
:105E12000E94F7720E94F6711E2F0A931A93EEEFF8
:105E2200EA93EFEFEA930ED91F3F41F4A0919E0B44
:105E3200A03021F4A091A10BA03009F002C00E9471
:105E4200FF7220FE0AC0E89420F8E091E30BE030F4
:105E520019F4F1D342D501C0A1D530E0353080F537
:105E6200ABE03A9FF001DF01EA51FA4FE081E03006
:105E720049F0AC51BA4F0E940573E8EEF3E00E947C
:105E8200F76F99F4ABE03A9FF001EA51FA4FE081E3
:105E9200E23051F43A9FF001EC51FA4FDF010E94D7
:105EA200D97A0E94CF6D09F409C0ABE03A9FF001A4
:105EB200EA51FA4FA0E0A083689420F83F5FCECF6A
:105EC2000E94C47C1FC30E94EE6BA33011F40C9499
:105ED2001D31E0913A08ED3411F00C944630E09116
:105EE2003B08EA3511F00C94FB2F24FC83C0E091AF
:105EF2003C08E0532E2FE0913D08E0533E2FEEE3A5
:105F0200F8E00E9420720E941472AC91AB3429F422
:105F12000E940A730E94E2600E2F0E941472AC91DA
:105F2200A43529F40E940A730E94E260AF01E09155
:105F3200CE0BE31731F5E0E0E093500C0E94A4721F
:105F42004093270850932808A09130080A1759F067
:105F5200E7E0E09318080093300820934F0CE0E04C
:105F6200E0932F080DC0A0914F0C2A1721F0A091A9
:105F72002E08A03009F004C02093180820934F0C7B
:105F820035C0A0913008A03049F4A091CF0B0E94F7
:105F9200D26BE255FF4FE491EA2309F40CC0E7E02B
:105FA200E093180820934F0CE0E0E0932F08E09173
:105FB2003908E093500CE0913908A091500CEA178F
:105FC200A9F44093270850932808009330080E94B0
:105FD200A472A0914F0C2A1721F0A0912E08A03094
:105FE20009F004C02093180820934F0C273011F4B5
:105FF2000E941C70E0913B08E93439F4E7E00E940A
:10600200B3720E94AB72E0932F08E0913B08E23436
:1060120039F4E4E00E94B3720E94AB72E0932F085D
:10602200E0913B08E03519F4E1E0E0931808E091D3
:106032003B08EC3449F4E4E0E0931808E0913C08B2
:10604200E053EA930E94D914E0913B08E334E9F467
:10605200A0913C08A13320F0A0913C08A93308F09C
:1060620014C00E940D73E0912208EA930E94001A64
:10607200E0913908EA93E7EBF5E1FA93EA930E949B
:10608200426F0E94EC7A0E94C762E0913A08E035C2
:1060920021F4A0911908A13009F003C00E9478727E
:1060A2005CDAE0913A08EF3459F4E0913B08EE34BF
:1060B20039F4E0913908EA93EAEBF5E10E941373AF
:1060C200E0913A08E33569F5E0913B08EF3349F591
:1060D200A0913C08A03320F0A0913D08A03308F421
:1060E20020C00E940D73E0913D08E0531E2FA09145
:1060F2002208A63010F41A3008F013C0103011F440
:106102000E944A19E0913908EA93EDEBF5E1FA931E
:10611200EA930E94756F0E94586F0E94EC7A0E9467
:10612200C762E0913A08E33411F00C94E530E09153
:106132003B08EF3311F00C94E530E0913D08E03379
:1061420019F4EFEFE0932308A0913C08A033F8F094
:106152000E940D73A0912208A630C8F4E091230892
:10616200EF5FE0932308E0912208EA93E09123088D
:10617200EA930E94C619A0911F0CB091200C1097AF
:1061820021F4A0912308A03408F001C0E7CFE091E8
:106192002308EA930E94B4170E941973E0ECF5E118
:1061A2000E9406720E94126E0E941E730E94237346
:1061B2000E94176E0E94EC7A0E9423730E947F6EE7
:1061C2000E944C620E949962E0913A08E434A1F57F
:1061D200E0913B08E43481F514E0E1E0E093390911
:1061E200103538F40E947B70E85CF74FE081E032B2
:1061F20008F41AC00E947B70E85CF74FE081E3323A
:1062020059F40E947B70E75CF74FE081E053EA9318
:106212000E94535D1F5F06C00E947B70E85CF74FCF
:106222000E944B711F5FDCCF0E941973E3ECF5E112
:106232000E9406720E9499620E94C27C269608956C
:106242001A930A930E94297111F40C948F31E0E0A1
:10625200E0935C0CE0911808EF770E2F009318087A
:106262000E94C3450E94A26C0E94AB6B0E949C4597
:10627200013021F0A0911908A13009F00DC0EEE81B
:10628200F5E00E94A76C9DD9E4EFF1E0FA93EA935E
:106292000E9415420E94C345073049F40E94B11F73
:1062A200E0E0E0931B080E94A2100E9472270430D3
:1062B20031F4E6ECF5E10E94A76C0E94600C083014
:1062C20019F40E9429735FD1053019F40E942973D1
:1062D20056DC013039F40E943673009319083DD917
:1062E2000E94AB0D093059F40E9436730E94AB0D27
:1062F2000A93E1E0EA9378DAE1E0E0935C0C0230A1
:1063020029F40E942973E1E0EA93B0DB033011F42F
:106312000E94753F009319080E94631EA0911908FC
:10632200A73011F00C943B32E091550CF091560CD1
:106332000E94CF6D21F0A0911B08A03009F00AC085
:106342000E94B971E091510CA0912306EA1711F055
:106352000E9472270E94F741E030E9F0E2E00E94D9
:106362006C721A9310DA1D3409F4C7D81D3399F4EC
:106372000E94DF448FDAEF3F41F0E3E0E093180838
:106382000E9473720E94B97206C0E7E8E09318088F
:10639200E0E0E0931B08A0912F08A03031F0E091DB
:1063A2002F08A0912E08EA1709F455C0E0912F0892
:1063B200E150EA930E940918A091350CE1E0EA232A
:1063C200E13021F4E0912B06EF7C09F429C0E0E0F2
:1063D200E0932E08E0914F0CE03019F0E09318089A
:1063E2001EC012E0E0912B06EC7009F018E0E0917B
:1063F200C50BA0912F08EA1781F0E0912B06E074FB
:1064020039F011E0EAE2EA93EBECF5E10E94137352
:10641200E0912B06E07809F019E0109318081BC0F0
:106422000E94C3450E94A2100E94A26C0E94AB6B04
:106432000E949C45EBE4EA930E943645E0912F08C6
:10644200EA930E946440EEECF5E10E94A76CE091B1
:106452002F08E0932E08A0912F08A03021F4A091DC
:106462002E08A03009F406C0E0E0E0932E08E7E829
:10647200E0931808A0911908A33011F40E94753D09
:10648200A0911908A13009F4ECD8A0911908A23002
:1064920009F408DBA0911908A83009F419DCA091CD
:1064A2001908A53009F497DBA0911908A93049F41D
:1064B200E0E0E0932008E0911908EA93E0E0EA9333
:1064C20093D90991199108950E944173E652F84FA8
:1064D200A6E0A0830E944173E752F84FAB81A083EC
:1064E2000E944173E152F84FAA81A0830E94417336
:1064F200E552F84FA881B981A083B1830E9423712C
:106502000E94B14F249608950E944773A881B981D1
:10651200AC91A53020F0A881B981E0E0EC9389C06C
:10652200A0911308BB27E091120805C0A0911108A1
:10653200BB27E0911008F0E031960E94C76F3596B4
:10654200DF01E5E0F0E00E94927A08951A9310913B
:106552001308E0911208E117A1F0ABE01A9FF001D5
:10656200E652F84FE081E13011F0E23011F4E1E05F
:106572004DC0EDB7FEB7FA93EA931F93C5DF1F91A3
:10658200E8CFE0E043C01A930E94B11FECEDF5E0C2
:106592000E948C6F0E941A6C0E94F96710E01530FD
:1065A20068F40E94FD6FAFEFA083ABE01A9FF00189
:1065B200EE51FA4F0E94B4711F5FF1CF10E0153017
:1065C20048F4A7E11A9FF001EC5CF94FAFEFA0830A
:1065D2001F5FF5CFE0912B06E37019F00E948F72D6
:1065E20009F402C0689401C0E89421F8EFEFE09347
:1065F2002D08E091E30BE03029F41DD06ED1E89430
:1066020020F804C00E94C3450E94320E19910895D9
:106612001A9310E0153058F40E94FD6FE081AE2FFE
:10662200E981EA1711F4E12F03C01F5FF3CFEFEF07
:1066320018812296089522970E94BB7C00E00530C3
:1066420058F40E944D73A0E00E945373E152FA4F36
:10665200A0E0A0830F5FF3CF00E00530C0F50E94F9
:106662009871E081EF3F89F10E949871E0810E9468
:106672000C70B9F00E949E71DF010E94D97A0E94CB
:10668200DA6FEA17FB0751F00E949E710E94DA6FDF
:10669200A083B1830E945873A1E0A0830E944D732E
:1066A20012C0ABE00A9FF001EA51FA4FE081E030FC
:1066B20061F40E949871AFEFA0830E949E710E94C4
:1066C200B4710E945873A1E0A0830F5FC6CF0E94ED
:1066D200831D1E2F1F3F11F0E1E001C0E0E0E093B7
:1066E2005C0C1F3F11F40C94C83350E000E00530FD
:1066F20048F40E949871E0811E1711F451E002C023
:106702000F5FF5CF5030E1F500E00530C8F50E948B
:106712009871E081EF3F91F50E94987110830E9479
:106722009E710E94DA6FA083B183ABE00A9FF001F1
:10673200E052FA4FA0912A0C0E945373EF51FA4F84
:10674200FF93EF930E9407700E94116FAF91BF9168
:10675200EC930E945873A1E0A0830E944D73A1E0C4
:106762000E945373EC51FA4FFF93EF930E945E67BE
:10677200AF91BF91ED93FC9351E002C00F5FC5CF83
:10678200503029F01A930E948A1D1E2FAACF30E0A2
:10679200353010F00C940E34A7E13A9FF001E15D20
:1067A200F94FEE83FF8350E000E0053048F55030AA
:1067B20029F5ABE00A9FF001EF51FA4F20812A93AD
:1067C2000E94B4170E944D73E081E13059F42A937C
:1067D2000E94A41EE13031F4A32FAF5FE0919E0B23
:1067E200EA1709F00BC0E22FAE81BF811396EC933A
:1067F200E02FAE81BF811596EC9351E00F5FD5CFAC
:10680200503049F4AE81BF811396EFEFEC93AE8125
:10681200BF811596EC933F5FBBCF0E94C27C0C9464
:10682200B6360E94BD7CAC81BD81EBE4EC93EC8179
:10683200FD813196FA93EA930E945E73E052FA4F19
:10684200E0810E94926B00E00E946773EC91E0305D
:1068520011F00F5FF9CF0E946773E0E2EC930F5FD4
:106862000E946D730E94486C0E945E73EE51FA4F53
:10687200DF010E94006D0E947273EE81ABE0EA9F1D
:10688200F001EF51FA4F10811A930E94B41700E001
:106892000E946773EC91E03011F00F5FF9CF0E9414
:1068A2006773E8E7EC930F5F0E946773E0E2EC9393
:1068B2000F5F30E03A3060F40E946D73EA0FFB1F05
:1068C2000F01ABE8BBE00E9479730F5F3F5FF2CF2D
:1068D2000E946773EC930C94FB3664970E94BD7C14
:1068E20000E010E0153040F40E94FD6FE081EF3FC0
:1068F20009F40F5F1F5FF6CF053021F0A0912D083C
:10690200A03009F406C0E0E0E0932D08EA930E946B
:106912004F0F10E0153088F5ABE01A9FF001E152FD
:10692200FA4FE081E03039F11A9FF001E352FA4F59
:10693200E081E030B1F01A93FE0135960E94A47115
:10694200ABE01A9FF001EF51FA4F30813A930E9467
:10695200B4171A93FE013596FA93EA930E94AA0F8E
:106962000AC01A930E949A0FABE01A9FF001E152FB
:10697200FA4FA0E0A0831F5FCDCF053021F4A09194
:106982002D08A13009F406C0E1E0E0932D08EA9356
:106992000E944F0F0E94C47C689608950E94BB7C9F
:1069A200A091E30BA23011F40C94953830E034310D
:1069B20068F40E9480730E948473DA011296E0E008
:1069C200EC93DA01EFEFEC933F5FF1CF0E94831D6E
:1069D2000E2F0F3F11F0E1E001C0E0E0E0935C0C0C
:1069E2000F3FA1F10E940770FA93EA930E94641785
:1069F2001E2F1F3F31F1A0911E08E12FEA1B3E2FEF
:106A02003431F8F40E9480730E948473FA01329642
:106A12000F01E081AE2F0E948A73B0E0EA0FFB1FE4
:106A2200D001EC93FA01A281A43620F0DA01129689
:106A3200E3E6EC93DA01AC91AF3F19F4E02FDA010F
:106A4200EC930A930E948A1D0E2FCACF0E94E8136C
:106A520030E0343110F00C94B4350E9480730E94FF
:106A62008473FA01A381AF3F11F40C94B2350E94F2
:106A72008F730E94076FE83139F40E948F73EA9393
:106A82000E94AD16E03009F408C00E948F73EA93A9
:106A92000E94AD16DA011296EC93A0919B0BA0789E
:106AA20039F4FA010280DA011196EC91E01509F449
:106AB20058C0DA0113962C91ADE02A9FF001EF5EE7
:106AC200FC4F0F01DA011296EC91D001EC930E9477
:106AD2008F73EA930E94C71FEF3F29F0ADE02A9F10
:106AE200F0010E944D6CDA011296EC91E03089F0CF
:106AF2000E949473DF010E94686CEC93ADE02A9FC0
:106B0200F001E25FFC4FDF01E091990BEF70EC9333
:106B120013C00E94686CE03021F40E949473A0E0DC
:106B220003C00E949473A8E0A083ADE02A9FF00105
:106B3200E25FFC4FA7E0A0830E948F73EA930E945A
:106B4200C71FEF3F19F0ECE0E0930F04DA01129651
:106B5200EC91DA011196EC932A93E1E0EA930E9418
:106B620025463F5F76CF0C949538E7E0E09318080E
:106B72000E94EF16A8950E94471BA8950E949F1D90
:106B8200A895EFEFE093B30BE0938A0BE093340CFC
:106B9200E0932F0CE0932E060E949A73EC7F29F06B
:106BA200A8E0B0E0E0E00E941B7B089524970E94D9
:106BB200BD7C0E941241ECEDF5E10E948C6F0E94B7
:106BC2009E410E943A41E0912208E03061F0E7EEF6
:106BD200F5E10E948C6F0E949E41E09122080E9482
:106BE2009F730E94A3730E943A410E944A1900E0D7
:106BF2000A30A0F40A930E94E3170E94A56EEFE008
:106C0200EA930E947841E02FA3EAB6E00E94A773BC
:106C12000E94586F0E94AB730F5FEACF0E944C41F3
:106C2200E0EFF5E1FA93EA93EFE0EA930E949E41E6
:106C32000E94DF6D0E94AB730E944E410E943A4156
:106C420010E0103110F00C94B2360E940D6DE11775
:106C5200E1F5E6EFF5E10E948C6F0E949E410E94F1
:106C62008E6C0E94A373E0E0E0931E08A0911E08C0
:106C7200A03448F5E0912208EA93E0911E08EA93D5
:106C82000E94C6190E94126E3097B9F0E0911E0858
:106C9200EA930E94B4170E94126EFA93EA930E943A
:106CA200B1730E949E410E947F6EEAE0EA930E94C5
:106CB20078410E94176E0E94AB73E0911E08EF5F4D
:106CC200E0931E08D3CF0E94B6730E947B700E948D
:106CD2005D6F11F00C94B036E6EFF5E10E948C6F17
:106CE2000E949E410E948E6C0E94A3730E94BA73FE
:106CF200E0E30E94696F29F40E946E6F0E94E260D5
:106D02009F0100240216030644F50E940A730E94A2
:106D12000C610E94826D0E940A730E94C2733A93B0
:106D22002A930E94B1730E949E410E94C673EAE0B8
:106D3200EA930E947841EC81FD816E817F810E94FD
:106D4200AB730E94BA73E1E30E94696F29F40E9457
:106D52006E6F0E94E2609F01D4CF0E94B6731F5FE4
:106D620070CF0E9413410E94C47C289608950E940D
:106D7200BD7CAD81BE812C910E94CB730E948E6C32
:106D82000E94BA6B0E94096DECE3EA930E943645B9
:106D9200EC81EA930E948E452A93ED81EA930E9448
:106DA2000440EEE3EA930E9436450E9440720E943C
:106DB200E6710E9446720E94D073333409F431E2C4
:106DC200313320F0EC81E05DE31708F407C0E32FD4
:106DD2000E948C72E255FF4FE4912E273D3311F051
:106DE200313209F401C0CACF3D3319F4AD81BE81FD
:106DF2002C93E32F0E94C47C279608950E94BB7CAB
:106E020020E0AF81B8855C910E94CB730E948E6CAA
:106E12000E94BA6B0E94096DE2E0EA930E948E45DD
:106E22005A930E9464400E9440720E94E6710E943E
:106E320046720E94D073303310F03A3308F00EC01D
:106E4200203009F450E021E0A52FEAE00E948F7A79
:106E5200AAE0EA9FF001E30FE0535E2F3B3211F408
:106E6200533608F001C05F5F3D3211F4513008F42F
:106E720001C05150333429F4203009F431E250E09A
:106E820020E03D3319F4EE81E51708F005C0AF812B
:106E9200B8855C9130E020E03D3311F0313209F4E5
:106EA20001C0B4CF3D3319F4AF81B8855C93D0C033
:106EB2000E94BB7C20E0AF81B8854D915C910E941D
:106EC200CB730E948E6C0E94BA6B0E94096DAE81D8
:106ED200A23051F4E6E0EA930E948E45FA010E9444
:106EE2001E730E94434008C0E5E0EA930E948E456B
:106EF2005A934A930E944E400E9440720E94E67149
:106F02000E9446720E94D073303310F03A3308F078
:106F12001EC0203011F440E050E021E04031E7E2B1
:106F22005E0734F0DA01E0E1F7E20E94927AAF0103
:106F3200493BEBE05E0724F0DA010E948772AF0161
:106F4200DA010E94D5730E94DA73D097AD013B3209
:106F520021F44033E5E75E070CF002C04F5F5F4F5C
:106F62003D3221F40024041605060CF002C0415003
:106F72005040333431F4203009F431E240E050E043
:106F820020E03D3311F0313209F401C09ACF3D3394
:106F920021F4AF81B8854D935C935AC00E94BB7CAB
:106FA2000E94CB7320E050E04FEF0E948E6C0E9453
:106FB200BA6B0E94E8720E94DF73E885EA930E942E
:106FC2006445E52FE10FF0E00E94E6710E944672EF
:106FD2000E94D073303310F03A3308F021C030539E
:106FE200431729F04F3F09F05F5F20E005C0A22F51
:106FF200AF5FEA2FE3702E2FE52FAF81B8850E9495
:10700200E4730F01E32FACEBB6E00E94A773AE0F5F
:10701200BF1FE22F0E94E473E491D001EC93432F4F
:107022003B3219F4EE815E1708F002C05F5F4FEF4A
:107032003D3211F4513008F402C051504FEFEE814D
:107042005E1720F4313211F03D3309F401C0ADCFA7
:10705200E32F0E94C27C299608951A930A93A09165
:107062009B0BECEDEA231E2F00E00D3040F40E9452
:10707200E8730E94EC73E11711F00F5FF6CF0E94E4
:10708200E873EA0FFB1F0E94E87A0E94A76CE02FC8
:1070920045C4ABE9BBE00E94F86CAE0FBF1FEC9198
:1070A200E17011F4E3E701C0E9E4EA930E94364596
:1070B200219608950E94BB7C0E94CB730E948E6C25
:1070C2000E94BA6B0E94E872C8DF5E2F0E94407273
:1070D2000E94E6710E9446720E94D0733D3211F006
:1070E200363311F4503009F401C051503B3211F0E3
:1070F200333311F45C3008F001C05F5FA0919B0B49
:10710200E1E0EA232E2FE52FA0E0B2E00E94A77370
:107112000E94EC73E20FE0939B0B3D3311F031328E
:1071220009F401C0CBCFE32F0E94C27C26960895BA
:107132000E94BD7C0E94CB730E948E6C0E94BA6B2F
:107142000E94E872ABE9BBE0EC810E94036FEC9114
:10715200E17019F4E3E0F6E102C0E7E0F6E1FA9348
:10716200EA930E944D450E9440720E94E6710E947D
:1071720046720E94D073303310F03A3308F00FC0D9
:10718200ABE9BBE00E94276F0F01ABE9BBE0EC81EA
:107192000E94036FAC91E1E0EA27D001EC933D330A
:1071A20011F0313209F401C0C7CFE32F0E94C47C31
:1071B200259608950E94A26BE1E0EA930E944A0D8F
:1071C2000E94466B0E94466B0E949C450E947F6E05
:1071D200EAE0EA93E3DEE13209F469C40E94466B15
:1071E2000E94466B0E94E16CEBE0F6E10E94A76C04
:1071F200E6E9FBE00E948C6F5BDEE13209F457C4E2
:107202000E94466B0E94466B0E94E16CE1E1F6E14E
:107212000E94A76CE091980BEF5F0E2FEDB7FEB7BF
:10722200FA93EA930F93EAE0EA93E8DD0F91E132F1
:1072320009F43DC400240216030624F4E02FE150B1
:10724200E093980B0E94466B0E94466B0E94E16C91
:10725200EAE1F6E10E94A76CEDEAFBE00E94F1731D
:1072620009F425C40E94466B0E94466B0E94E16CA1
:10727200E0E2F6E10E94A76CEFEAFBE00E94F17304
:1072820009F415C40E94466B0E94466B0E94E16C91
:10729200E6E2F6E10E94A76CEAE9FBE0FA93EA93E0
:1072A200E3E60E94FA7309F402C40E94466B0E944C
:1072B200466B0E94E16CEFE2F6E10E94A76CFADEF7
:1072C200E13209F4F4C310E0133010F00C94203AC8
:1072D2000E94466B0E94466B0E94E16CE12F0E9465
:1072E2004A72E5E3F6E10E94A76C0E94FF730E94D6
:1072F2009C45AEE9BBE00E947B700E94486CE0E1D5
:107302000E94FA7309F4D3C3E9E0F0E00E94786BBB
:107312000E949C45A1EABBE00E947B700E94486CDF
:10732200E0E10E94FA7309F4C2C30E94466B0E9414
:10733200466B0E94E16CE12F0E944A72E0E4F6E1A2
:107342000E94A76C1A93F4DEE13209F4B0C30E94E2
:10735200FF730E94037451F40E9433710E940D74F2
:10736200E2E00E94117409F4A2C309C00E943371C1
:107372000E940D74E0E00E94117409F498C30E9407
:10738200466B0E94466B0E94E16CE12F0E944A729A
:10739200E2E4F6E10E94A76C0E94FF730E949C4502
:1073A200AAEABBE0EE27A10FBE1F2C913327EDB74F
:1073B200FEB73197FA93EA933F932F93E0E0EA9373
:1073C20077DD2F913F91E13209F471C3AAEABBE064
:1073D2000E947B70EA0FFB1F2083123070F50E941F
:1073E200466B0E94466B0E94E16CE12F0E944A723A
:1073F200E9E4F6E10E94A76C0E94FF730E949C459B
:10740200A1EBBBE0EE27A10FBE1F2C913327EDB7F6
:10741200FEB73197FA93EA933F932F93E0E0EA9312
:1074220047DD2F913F91E13209F441C3A1EBBBE06B
:107432000E947B70EA0FFB1F20831F5F45CF37C37B
:107442000E94BD7C10E01A930E94C0720E941674C2
:107452000E94466B0E949C450E94196D0E941A74FC
:107462000E949A6C0E940C6F0E94F46C0E94466B00
:107472000E94A26C0E949C450E941A6F0E94056D98
:10748200E7E0F0E0FA93EA930E94A26C0E949C4526
:10749200E091AF0BF091B00B0E94F7790E94056D5D
:1074A2000E94466BE2E0F0E00E94096DE0E5F6E141
:1074B2000E94A76CE091980BEF5FEA930E946440F0
:1074C200E7E0F0E00E94936C0E949C45C6DD0E94BA
:1074D200E56CE0919A0BE03029F0E0919A0BEA9387
:1074E2000E94644000E00330D8F50E94466BE02F12
:1074F200ED5FF0E00E94096D0E946071EA930E94C4
:107502006440EBE2EA930E9436450E946771EA9377
:107512000E9464400E94E56C0E946E7151F40E94C8
:1075220076710E94FB6C0E94006D0E941E74E3E75C
:1075320009C00E9476710E94FB6C0E94D97A0E9457
:10754200F46CE9E4EA930E9436450E94E56C0E94DD
:107552008071EA930E946A400E9422740F5FC3CF37
:107562000E94FA413E2F3B3211F4103408F001C060
:107572001F5F3D3211F4113008F401C011503D3447
:1075820039F41A930E94B41715DE1A930E94D41785
:10759200313209F058CF8BC20E94BD7C10E00E94AC
:1075A200C345012F0E94466B0E94466B0E949C4578
:1075B200E4E5F6E10E94A76C31E03C3018F51038A2
:1075C200F8F40E94466B0E94D26B0E94096D1A93D6
:1075D2000E9409180E94196D0E94E56CA091350C59
:1075E200E3E00E942674A091360CE7E00E94267424
:1075F200E0912B06EA93E8E0EA930E940440139597
:107602003F5FDBCF0E94600C0E94FA413E2F3D3467
:1076120011F00C944B3B0E94896C0E944A0D102F72
:107622001038C0F51A930E9409180E94466B0E94F6
:10763200466B0E94E16CE8E6F6E10E94A76C0E94AC
:10764200196D0E941A740E94206D0E949C45EBE6FF
:10765200F6E10E94A76CE5E3FCE0FA93EA93E3E02B
:107662000E94FA7309F423C20E94206D0E94E16C09
:10767200E1E7F6E10E94A76CE6E3FCE0FA93EA9305
:10768200E7E00E94FA7309F412C21A930E943B18AF
:107692001F5FC6CF313211F0103808F001C07FCF22
:1076A20006C20E94A26B0E9416740E94466B0E9440
:1076B2009C45E7E7F6E10E94A76C10E01530F0F474
:1076C2001A930E9447180E94466B0E94F56D0E9411
:1076D200196D0E941A74E091300C0E942B74E09193
:1076E200330C0E942B74E091310C0E942B74E091B8
:1076F200320CEA930E946A401F5FE0CF0E94FA4177
:107702000E2F0D3411F00C94C53B0E94896C0E941F
:107712004A0D10E01530C0F51A930E9447180E94D6
:10772200466B0E94466B0E94E16CEAE8F6E10E9419
:10773200A76C0E94196D0E941A7430E03430F8F47C
:107742000E94206D0E94E16C0E94D26B0E94EA7935
:10775200E456F94F0E94E87A0E94A76C0E94D26B0D
:107762000E94EA79E456F94F0E942F74FD01359682
:10777200E4910E94FA7309F49AC13F5FDFCF1A9332
:107782000E9467181F5FC6CF92C11A930A930E9484
:10779200C345E1E0EA930E944A0D00E0083210F08E
:1077A2000C948F3C0E942F0C0E94466B0E94466BE9
:1077B2000E949C450E94BA6B0E9432740E94E87A31
:1077C20031960E94A76C0E94E56C0E94BA6B0E94DF
:1077D20032743496E491E038A9F40E940D6D1E2FA4
:1077E200EDB7FEB7FA93EA931F93E0E1EA9306DB63
:1077F2001F91E13209F492C0E12FA9E0B0E00E94AA
:107802001B7B88C0E238A9F40E94916F1E2FEDB74E
:10781200FEB7FA93EA931F93E0E1EA93EFDA1F913E
:10782200E13209F47BC0E12FAAE0B0E00E941B7BA9
:1078320071C0E138E1F40E949A731E2FEDB7FEB7D2
:10784200FA93EA931F93E3E0EA93D8DA1F91E132C5
:1078520009F464C00E942F0C0E949A73E11731F060
:10786200E12FA8E0B0E00E941B7BFFCF53C0E030C5
:1078720069F40E94BA6B0E94327432960E94AB6C19
:10788200E1E00E94FA7309F449C044C0E13069F4AE
:107892000E94BA6B0E9432740E942F74FD013596C9
:1078A200E4910E94FA73D1F135C0E23061F40E9492
:1078B200BA6B0E94327432960E94AB6CEFE00E9467
:1078C200117461F127C0E33071F40E94BA6B0E9417
:1078D20032740E942F74FD013596E491EA9347DADF
:1078E200E132E1F017C0E430A9F40E94BA6B0E94C1
:1078F200327432960E94E87AE0935D0CF0935E0C4B
:107902000E94E6710E9432743596E491EA9346DB56
:10791200E13221F00E94F2160F5F40CF09911991D6
:107922000895E8810E944A72EEE0F6E10E94A76C97
:107932000C9410411A930E94896C0E944A0D10E027
:10794200133010F00C94F63C0E94466B0E94466B7A
:107952000E94E16C1A93E5DFECE0F0E00E94786BA4
:107962000E949C451A9395DB0E94FF730E94037448
:1079720051F40E9433710E940D74E2E00E9411746E
:1079820009F4FEC209C00E9433710E940D74E0E046
:107992000E94117409F4F4C2123028F50E94466B59
:1079A2000E94466B0E94E16C1A93BBDFEDE8F6E1A0
:1079B2000E94A76CECE0F0E00E94786B0E949C456C
:1079C2000E942274EAE0F0E00E94786B0E949C45DB
:1079D200A1EBBBE00E947B700E94486CE3E60E9430
:1079E200FA7309F4CDC21F5FABCFCAC20E94BD7C3D
:1079F20010E01A930E94C0720E9416740E94466B95
:107A02000E949C450E94196D0E941A740E949A6CF1
:107A120021E000E0033080F5E3E0F0E00E94E96B52
:107A22000E94096D0A937DDF0E946E7149F40E94E3
:107A320076710E94FB6C0E94006D0E941E7408C049
:107A42000E9476710E94FB6C0E94D97A0E94F46CAB
:107A52000A931FDB2F5F023068F4E7E0F0E00E9438
:107A6200E96B0E94096D0E9479710E941E6D0E944D
:107A720022742F5F0F5FCECF0E94FA413E2F3B321E
:107A820011F4103408F001C01F5F3D3211F41130BF
:107A920008F401C011503D3439F41A930E94B4170E
:107AA20049DF1A930E94D417313209F0A2CF0E9403
:107AB200C47C249608950E94896C0E944A0D0E94FB
:107AC200466B0E94466B0E949C45E3E9F6E10E94E8
:107AD200A76CE1E0E0932208E2E2F8E0FA93EA938D
:107AE200E5E0EA938BD9089522970E94BB7C0E941D
:107AF200FA410E2FE0911B08E03011F00C94233F65
:107B02000132D1F4E2E4F6E0A0913B0CB0913C0CDE
:107B1200EA17FB0761F4E7E0E0931808EAE2EA9368
:107B2200ECE9F6E10E948C6F0E94D462A9C0E0E009
:107B3200E093C0050E9437740D3331F4E091C00523
:107B4200F0E00E94D86B04910D3441F4EAE2EA932A
:107B5200EFE9F6E10E948C6F0E94D462063449F488
:107B6200EAE6F6E0E0933B0CF0933C0CE0E0E093B5
:107B7200C005003311F00B3229F4E091C005EF5F2C
:107B8200E093C0050D3229F4E091C005E150E09385
:107B9200C005013329F48FDFED3311F40E943E74E6
:107BA200033329F488DFED3311F40E94D73506330D
:107BB20029F4E0E0E09322080E94D735043329F447
:107BC200E0E0E09322080E943E74A0912408A130D4
:107BD20010F40C94BD3E023301F56DDFED33E9F490
:107BE2000E944B74D1F4E0912208EA930E94001A99
:107BF20030E0303190F40E94D26B0E945D6F59F4F4
:107C0200E32FE05DEA93E2EAF6E10E94626FE0E3CD
:107C1200EA930E94F6623F5FECCF053331F5E0E074
:107C2200E09322080E944B7401F511E01630E8F44B
:107C32001A930E94001A30E03031A8F40E94D26BED
:107C42000E945D6F71F4E32FE05DEA93E2EAF6E1F0
:107C5200FA93EA93E12FE05DEA93E0E3EA930E946C
:107C6200F6623F5FE9CF1F5FE1CF013469F4EAE2D8
:107C7200EA93E5EAF6E10E941373E1E0E093180863
:107C82000E94C27C289608950A3409F4AFDE0733B5
:107C920011F00C94BD3E0E94896C0E948E0CE1E0B2
:107CA200E0931C08E0E0F0E0E0931408F09315087C
:107CB200EFE2F6E00E948C6FE3E7F0E00E943E6F95
:107CC2000E945E67EE83FF83EE81FF810E949C6DBE
:107CD2000E94F76FB9F00E94E5100E945E67EE8382
:107CE200FF83A0911A0CA03021F00E949132E03063
:107CF20009F408C00E944173E652F84FAEE0A08337
:107D02000E942371E5E0F0E0FA93EA930E941542A3
:107D120040E050E00E947E20E03868F00E947E2021
:107D2200EF573E2F313010F0313108F004C0E32F0D
:107D32000E945070AF015A934A930E943D1E409395
:107D42001408509315080091DB05E0E0E093DB0591
:107D5200013211F00B3209F401C0B6CF0B3221F41B
:107D6200E1E0EA930E948E0C013209F0A1CFE0E03B
:107D7200E0931C08E093DB05A0912408A23011F0E7
:107D82000C941C3F093309F400DD053409F489DC45
:107D9200083309F455DB023409F4FEDB0334B1F590
:107DA20010913A0C0E94C34500E0E091390CE117B2
:107DB20011F00C3008F01DC00E94466B0E94BA6B95
:107DC2000E94096D1A930E94911D1A937CD10E9400
:107DD200E56CE0912A0C0E942B74E0912D0C0E941C
:107DE2002B740E9407700E94F46C0E94ED6F039541
:107DF200DCCF0E94600C0E94FA410E2F013221F06A
:107E0200E091390CE11709F401C0CCCF043499F4A4
:107E12000E944B7481F4A091D40BA03021F4A09164
:107E2200D20BA03031F00E9494720E94466B0E94E5
:107E3200E1510E94DA1BE0911B08E03011F40E942C
:107E4200E70C49C0E130D1F4A0912108AB3010F425
:107E5200013209F405C00E9489140E94600C0DC011
:107E6200E0E0E0931E080E9454740E941373E0E065
:107E72000E945974E2E0E0931B082DC0E23059F5EC
:107E8200013269F4E0E0E0931B080E94C345EAE294
:107E9200EA93EFE9F6E10E9413730E94E70C0B32BA
:107EA20011F00D3359F40E945474FA93EA93E1E30A
:107EB200EA930E94D462E1E00E9459740D3259F4AF
:107EC2000E945474FA93EA93E2E3EA930E94D46222
:107ED200E2E00E945974A0911808A33009F407CE79
:107EE2000E94C27C0C9469441A93E3E0E09319085F
:107EF2000E94C3450E94466B0E94466B0E949C45AD
:107F0200EBEAF6E10E94A76C0E94466B0E94A26C0B
:107F12000E949C45E3E1F6E00E948C6FE0E1F0E014
:107F22000E943E6F10E0E091CA0B1E1700F50E94FE
:107F32000D6DE117D1F0E12FE05DEA93E3EBF6E19D
:107F4200FA93EA93E0E3EA93E0E00E94696F49F46E
:107F52000E947B70ED5EF94FA1E0A083E12FE05D0E
:107F620001C0EEE2EA930E9436451F5FDCCF0E9419
:107F72003774E0E0E093C005E0931B080E94E70C31
:107F820019910895E881E03021F4EAEEF6E00E94CA
:107F92005E74A881A13021F4E4EEF6E00E945E74E2
:107FA200A881A23021F4E0EFF6E00E945E74A8817D
:107FB200A33021F4EEEFF6E00E945E74A881A430B3
:107FC20021F4E4E0F7E00E945E7429C11A930A9357
:107FD200E0E0E0937D05E0937E0510E0143190F43B
:107FE20000E0033068F4A3E01A9FF001EC57FA4F67
:107FF200DF01EE27A00FBE1FE0E2EC930F5FF1CF8F
:108002001F5FECCFECC31A9311E0E981E11780F016
:108012000E947B70E255FF4FE491AA81EA2319F096
:10802200E12FE05D01C0E0E2EA931FD51F5FEDCFD3
:1080320030C51A9311E0E981E11778F00E947B7054
:10804200E255FF4FE491AA81EA2311F0E1E301C076
:10805200E0E3EA930AD51F5FEECF1BC52A97A091F2
:108062001C0CA13038F0EA85FB856C857D850E9469
:108072001E7407C00E9463740E9467740E94637436
:10808200FCD426C12A970E9463740E9470740E94D5
:1080920079740E946374F1D41BC12A970E9463749D
:1080A2000E948C740E949374E8D41FC12A970E9484
:1080B2006374E1EDF6E10E9498740E941E730E94BF
:1080C2009374DBD412C12A970E946374E4EDF6E143
:1080D20005C02A970E946374E8EDF6E1FA93EA93E9
:1080E200EE850E94926B0E946374C7D42B9608950A
:1080F2000E94BD7C10E0E1E3E0933809E89431F896
:10810200EA930E947E62ECEDF6E10E94067200E0C4
:10811200E09182050E17E0F40E94BA6BEC57FA4F19
:10812200E081E03258F4E3E2EA930E94AF610E94F8
:10813200BA6BEC57FA4FE081E05D05C00E94BA6B62
:10814200EC57FA4FE081EA930E94AF610F5FE0CFF4
:108152000E949D749F010E94F1133A932A93E8ECC6
:10816200F0E0FA93EA930E946A670E2FA0E031FCD6
:10817200A1E0A03011F4003009F001C0ECCF31FED3
:1081820009C0E0E0E0938205E89431F8E1E00E9462
:10819200C47CF6C41F5F123008F4ADCFE0E0E09378
:1081A20082050E94C47CECC4E0918105E03021F498
:1081B200E881EA930E94535DA0918105A13069F4A0
:1081C200A0E09299A1E0A13021F4A8950E94236E2B
:1081D200F7CFE881EA930E94F75FA0918105A23070
:1081E200F1F4E0918205F0E0EC57FA4FA881A08308
:1081F200E0918205EF5FE0938205E0918305EF5FF6
:10820200E0938305A03218F4EF5FE0938305A09119
:108212008305A83320F06CDFE0E0E093830521962C
:10822200089508950E94B6730E94B67322D0EBE1BE
:10823200EA93BADFE9E6EA93B7DFA0918105A130BC
:1082420061F4E8ECF0E00E948B6DE0919A00E06945
:10825200E0939A00E9E1E0939900A0918105A230B0
:1082620021F446DFE0E0E0938305E0E0E09381055E
:108272000895EDE0EA9398DFEAE0EA9395DF089546
:108282001A9310E0E9811E1728F4EA81EA938CDF41
:108292001F5FF8CFFEC3EDE201C0EDE3EA93E8E22F
:1082A200EA93EEDFE6DF08952A97A0911C0CA13035
:1082B20038F00E9463740E9470740E94797404C042
:1082C2000E9463740E946774FE010E948C6F0FD03B
:1082D2002E9608952A970E9463740E948C740E94BD
:1082E200A174FE010E948C6F02D02C9608951A93FD
:1082F2000A9310E0EA81E03011F408E201C00A8139
:10830200AB81BC81EE27A10FBE1FAC91A03011F052
:10831200101708F007C0AB81BC810E94A6740E94AE
:10832200AB74EECFEA81E03039F0EA811E1720F417
:10833200E0E20E94AB74F9CF27C01A930A9310E0CF
:10834200EA81E03011F408E201C00A81E12FAB8139
:10835200BC810E94E473E491E03011F0101708F040
:1083620009C0E12FAB81BC810E94E473E4910E94B9
:10837200AB74ECCFEA81E03039F0EA811E1720F4C9
:10838200E0E20E94AB74F9CF198108812596089525
:10839200E091C405A091C305EA17B1F00E94B07440
:1083A2000E94FB6CEC91E093C6050E94B0740E949F
:1083B2009570E181E093C505A091C4050E94B67451
:1083C200E093C405E1E00895E0E008950E94BB74E3
:1083D200A981A0830E94BB743196A881A083A09139
:1083E200C3050E94B674E093C305C2C0E091DB05E9
:1083F20008951A93E091DB05E03059F40E94F113DD
:108402000E94297121F4A091DB05A03009F001C07E
:10841200F5CF1091DB05E0E0E093DB050E942971C6
:1084220009F011E2E12FDDC30E94BD7C0E945E676C
:108432008F010E94F113EC81FD81E00FF11FFF9388
:10844200EF930E945E67AF91BF91AE1BBF0B9D0180
:108452000024021603061CF40E94297109F001C0CF
:10846200E8CFE0E00E94C47C269608951A93E98141
:108472000E9492710E94C174E05FFC4F108117FF4D
:1084820005C0E12F0E94C874A0E0A08316FF05C0BA
:10849200E12F0E94CF74A0E0A083E981ADE0EA9FC2
:1084A200F001E05FFC4F0E94C174E15FFC4FA0E06D
:1084B200A08318815DC00E94BD7C30E0EE81ADE0FA
:1084C200EA9FF001E05FFC4F108116FF17C0E12F19
:1084D200EF730E2F0E94D67411F03A3008F009C0E3
:1084E2000E94DE74DF010E94D26B0E94E4743F5F3F
:1084F200F1CF0E94DE740E94DA73EC9317FF17C06B
:10850200E12FEF730E2F0E94D67411F0343108F070
:1085120009C00E94EA74DF010E94D26B0E94E474D7
:108522003F5FF1CF0E94EA740E94DA73EC930E94DB
:10853200C47C42C2E881F9810E94AB6CEA81FB8172
:1085420032960E94AB6CEC81FD8134960E94AB6C3A
:10855200EE81FF8136960E94AB6CE885F9853896EC
:10856200E491EA93E985FA8539960E94B76B02D0C5
:1085720022960895A0970E94BB7CEDA5FEA5A9A90D
:10858200BAA9EA0FFB1FAF01E5E0F3E0EE83FF8338
:1085920010E01431C0F5AE81BF81AC91A03049F139
:1085A200EE81FF81A381B481EFA5F8A9EA17FB0749
:1085B20001F5EE81FF81A181B281E9A9FAA9AE1785
:1085C200BF07BCF0EE81FF81A181B2814A175B0730
:1085D20084F00E94F074AE0FBF1FE9A9FAA9AE178A
:1085E200BF073CF00E94F074AE0FBF1F4A175B0733
:1085F2000CF402C01A933ADFEE81FF813D96EE83BE
:10860200FF831F5FC6CFE5E0F3E0EE83FF8310E058
:10861200143110F00C94B043AE81BF81EC91E03084
:1086220011F00C94A943EAA5EC93E9A9FAA9AE8149
:10863200BF811196ED93FC93EFA5F8A9AE81BF819E
:108642001396ED93FC93EDA5FEA5AE81BF81159621
:10865200ED93FC93EBA5AE81BF811796EC93E0916D
:108662000904A0910F04EA27AE81BF811896EC930A
:10867200E0911004AE81BF811996EC93E091110450
:10868200AE81BF811A96EC93AE81BF811B960E9488
:10869200556C1C96E0E0EC93E887E8A5F9A53097C5
:1086A20041F00E94FB740E940075E4E1EA930E948B
:1086B2005868EEA1FFA1309751F00E94FB74E8A523
:1086C200F9A5FA93EA93E4E1EA930E944468E0E0B0
:1086D200EC8F0E94FB740E942F683E2F3B30C8F043
:1086E20000E00E94EA74E081E03011F0053008F009
:1086F20002C00F5FF6CF0E94EA74E081E03049F4D5
:108702000E94EA740E940575E058AE81BF811B96F3
:10871200EC93E0E0EA8B3130C8F000E00E94DE74B6
:10872200E081E03011F0043108F002C00F5FF6CFB3
:108732000E94DE74E081E03049F40E94DE740E94FF
:108742000575E05CAE81BF811B96EC93E12F08C0FA
:10875200EE81FF813D96EE83FF831F5F59CFEFEFDE
:108762000E94C27CE39608951A930A930E941075A0
:108772003097A9F1E0916205E03061F50E94107531
:10878200049000926205E0916205E03031F4E0E08D
:10879200F0E00E945E74E0E01AC00E9415750E942B
:1087A20010750E94E87AF595E7958F01D801E0E00F
:1087B200F1E00E94607AE0938700D801E0E0F1E006
:1087C2000E94927AE09386000E941575E0E4E0939D
:1087D2008B0005C0E0916205E150E09362050991CA
:1087E200199108950E94BD7C00E025E033E010E07D
:1087F2001431B8F5D901EC91E03079F111960E946B
:10880200D97A0E941D7524F5D90113960E94D97A4E
:10881200AC81BD81EA17FB07DCF4F901018012800B
:10882200D90115960E94D97AE00DF11DAE81BF8162
:10883200AE17BF076CF4F90103801480D9011796B3
:10884200EC910E942F71AC81BD81AE17BF070CF075
:1088520004C0E12FEF5F0E2F04C0235F3F4F1F5F65
:10886200C7CF003049F0E0916305E01721F0A091F5
:108872006305A03009F401C022C0A0916405A530AF
:1088820079F40A93E1E0EA93A1DD00936305009392
:108892006505D901EC91E0936605E3E0E09361059B
:1088A200A0916405AE3119F4E4E0E0936105A09172
:1088B2006105A33018F0E5E0E093680507C0E0E049
:1088C200E0936405E09361050E9422750E94C47CD6
:1088D20028960895E0916305E03091F0A091640537
:1088E200A93220F4EA93E2E0EA9370DDA0916405F4
:1088F200AD3330F0E0916305EA93E4E0EA9366DD9C
:10890200E0E0E0936105E09364050E942275E0E0F7
:10891200E0936305E0936705089534D157DB08952A
:10892200EA81E0937F05E881E0938005E0910A0403
:10893200E061E0930A0424C10E94BB7CA0917F0500
:10894200A43120F4A0918005A33008F033C0E09157
:108952007F05F0E0ACE0B0E00E94357A8F01E09153
:108962008005F0E0A4E1B0E00E94357A9F010E9408
:108972002875ECE0F0E00E942D75F0E00E94E879A5
:108982000E94506BEE81E030A9F0E0917F05A3E0F8
:10899200EA9FF001EC57FA4FDF01E09180050E9457
:1089A200036F4C9155270E9428754A93E0E0EA93A1
:1089B2000E94604C0E94C27C27960895E0910A04AE
:1089C200E07141F0E2E0EA93B7DFE0910A04EF7E62
:1089D200E0930A0408950E943275AF3EE0E0BE07BC
:1089E20044F4A0910203B0910303AF33E1E0BE0768
:1089F2000CF039C00E9437750E94156F0E94604CBE
:108A0200A0915D05B0915E05549734F4A0915F0585
:108A1200B091600513970CF012C0E0915D05F091E2
:108A22005E05A3E0B0E00E940D7AEC57FA4FA091E8
:108A32005F05B0916005EA0FFB1FA981A083E09159
:108A42000D04ACE0EA9FF0010E9432750E94E473CB
:108A52000E944475E0915D05F0915E053196E093C8
:108A62005D05F0935E050C949E49E881EA93E091DE
:108A72001004EA93B0DF0C946D491A9310E00E943F
:108A82004975E03031F00E944975EA93EEDF1F5FCD
:108A9200F6CF1881239608951A930A9300E010E006
:108AA2000E944C75E03021F00832E0E01E070CF025
:108AB20007C00E944C75EA93D8DF0F5F1F4FF0CFBB
:108AC200198108815DC01A930A9300E010E0F80151
:108AD200AB81BC810E94537521F0EA810E945875D6
:108AE2000CF009C0F801AB81BC810E945D75BDDF4D
:108AF2000F5F1F4FECCF198108810DC30E94BD7C0F
:108B02000E9432750E94627531978F010E946775CB
:108B12000E9428750E946F7533C00E94BD7CAC8193
:108B22000E9476750E2F11270E9467750E94287584
:108B32000E946F75F0C2EA81FB81E0935D05F093BC
:108B42005E05E881F981E0935F05F0936005AA81F3
:108B5200BB81ECE0F0E00E94357A0E944475A88166
:108B6200B981E4E1F0E00E94357A06C0EA81FB8136
:108B72000E944475E881F981E0930203F0930303B4
:108B8200249608950E947E75143120F41A936EDCA7
:108B92001F5FFACF0E94466B0E94466B0E944B6B8E
:108BA200EFE3F1E00E94506B10E0153048F4A5E1CC
:108BB2001A9FF001E051FB4FA0E0A0831F5FF5CFA9
:108BC20010E0143148F4ABE01A9FF001EC5EFB4F69
:108BD200A0E0A0831F5FF5CFE0910A04EF7EE0934F
:108BE2000A04199108950E947E75143100F5ADE0D2
:108BF2001A9FF001BF01E85FFC4FDF010E94D97AA2
:108C02000F01DF01EB81FC81AE17BF075CF0E98148
:108C1200FA81E015F10534F0FB01E05FFC4FE081E1
:108C2200E03009F402C01A9321DC1F5FDECF0E94FC
:108C3200466B0E9486750E944B6BA985BA850E947D
:108C42008B750E94506B66C2A2970E94BB7CE9A5FD
:108C52000E9492718F01D8011B96EC91E03009F4C9
:108C620014C2D8011B96EC91E9A3E07859F0FE01F9
:108C72003696FA93EA93EBA10E94C874FA93EA93A8
:108C82000E941968E9A1E07459F0FE013696FA9340
:108C9200EA93EBA10E94CF74FA93EA930E941968B7
:108CA200FE0136960E949075E8A3E0910D04EB8FC9
:108CB200E0910E04EA8F0E94D96DD80111962D9190
:108CC2003C91D80113964D915C91D80115960E9462
:108CD200D97AEEA3FFA3D8011796EC91F0E0ECA3AA
:108CE200FDA3D8011896EC91EC8FE0910E04A0E15F
:108CF2000E949475EAA3FBA30E9498750E940075D6
:108D02000E940075ECA1EA930E94B24AD80119961A
:108D1200EC91EC8FAC8DAF3011F4E8E0EC8F0E9457
:108D220098750E949D755A934A930E94A4750E9459
:108D3200A8750E94AF750E94B2750E9498753A9309
:108D42002A930E94B275EEA1FFA10E94B9755A93AF
:108D52004A930E949D750E94B275A8A5A130B1F4F4
:108D62003A932A93FA0131960E94AF75FA0131962D
:108D7200FA93EA930E94A475F90131960E94BE7596
:108D8200F9013196FA93EA930E94B275A8A5A2302E
:108D9200F1F40E94A87531970E94AF75EAA5FBA570
:108DA200E40FF51F3197FA93EA930E94A475EEA19E
:108DB200FFA1E20FF31F31970E94BE75EAA5FBA542
:108DC200E20FF31F3197FA93EA930E94B275E8A576
:108DD200E03011F40C941648D8011996EC91EC8FFE
:108DE200E0910D04ACE00E94C3750E94607AED8FA1
:108DF200A8A1EA1710F40C944547E1E0E0930E04B1
:108E0200E03021F0ECA1FDA1B5970CF402C00E9464
:108E1200C975AAA1BBA1ECA1FDA1EA1BFB0BDF0155
:108E22000E947E70EAA3FBA3ABA1AA231AF4E0E09E
:108E3200EAA3EBA3A8A10E947675AEA1BFA1F0E0C0
:108E42000E94D175EE8FA8A5A13021F40E94D4759D
:108E52000E94D775A8A5A23031F40E94D4750E9451
:108E6200B9750E94E375E0E0E9A30E94E975AE0FCF
:108E7200BF1FEC91E03039F00E94E9750E945D75E8
:108E82000E94EE75F2CFD1C0E1E0E0930E04E03033
:108E920031F0ECA1FDA1E734A0E0FA070CF402C026
:108EA2000E94C975E8A1EF8FEAA1FBA1EE0FFF1F97
:108EB200ACA1BDA1AE1BBF0BE3E0F0E00E94607A63
:108EC200EAA3FBA3ABA1AA2322F4E1E0F0E0EAA328
:108ED200FBA3EF8DE150EF8FEF8DF0E0DE011696F0
:108EE200AE0FBF1FAC91A03219F0AF8DA13008F4C4
:108EF20004C0EF8DE150EF8FEFCFAF8D0E947675FA
:108F0200AE2FEEA1FFA1B0E0EA17FB0714F3EF8D3D
:108F1200E03011F4ED8DEF8FAF8DECE00E94C37560
:108F22000E94D175EE8FA8A5A13021F40E94D475BC
:108F32000E94D775A8A5A23031F40E94D4750E9470
:108F4200B9750E94E375E0E0E9A30E94E9750E9409
:108F5200537521F0EF8DA9A1AE1708F007C00E944A
:108F6200E9750E945D750E94EE75EFCFAF8DE8A1A5
:108F7200EA1BAE2FED8DEA1768F0AF8DE8A1EA1B70
:108F8200ACE0EA9FF001A0910D040E94C3750E941B
:108F9200D17501C0E0E0EE8FA8A5A130A1F40E9436
:108FA200D475E20FF31F31960E942D75AFE00E9437
:108FB2009475E40FF51FDF01ECA1FDA10E949570ED
:108FC20031960E94876DA8A5A23089F40E94D475BB
:108FD200E20FF31F0E942D75AFE00E949475E40F1B
:108FE200F51FDF01ECA1FDA10E940D74BFDD0E94FF
:108FF200E975AE0FBF1FAC91A03219F4E9A1EF5F82
:10900200E9A30E94E9750E94537539F0AF8DE9A179
:10901200EA1BAE2FED8DEA1708F407C00E94E9752E
:109022000E945D750E94EE75ECCFD8011C96EC9102
:10903200E03029F10E94D96D0E94987597DDF80100
:10904200A485A43698F4E0E0E0931004F801A48526
:10905200AA3028F0A485AA930E94644006C0D801D1
:109062001C96EC91E05DEA9300DD09C0ECE0E09330
:109072001004E2E5EA93F9DCEDE4EA93F6DCEB8D29
:10908200E0930D04EA8DE0930E040E94C27CAA963E
:1090920008951A9310E0E89427F8143170F40E94AE
:1090A200B66DE03011F00E94BD6D1F5FA895E12FF3
:1090B200E37011F40E94E813F0CFE0E0E0931004B3
:1090C2000E94E8130C94B04C1A9310E01431F8F497
:1090D2000E94C26DB1F0A85FBC4F0E94D97ADF0135
:1090E200EB81FC81EA17FB0764F4F001E85FFC4FB7
:1090F200DF010E94D97ADF01E981FA81AE17BF0749
:109102000CF002C00E94BD6D1F5FA895DFCFE0E0AA
:10911200E09310041881259608951A9310E01431F3
:1091220090F40E94C26D31F0FD01E15FFC4FE081DD
:10913200E17009F406C01A93E0910A04E170EA931F
:1091420083DD1F5FECCF0C94B04C2C970E94BB7C4C
:10915200AD89BE890E947E700E94F675EB8BFC8BF6
:10916200ED89FE890E94FB75EB89FC89E017F10706
:10917200FCF00E942E762E2F33270E9452760E94F8
:1091820059760E9460760E9465760E945276F801B6
:10919200A98DBA8D0E94486C0E946076F8010E94E7
:1091A2006F76EA8DEA930E94154B0F5F1F4FDCCF5B
:1091B20048C02C970E94BB7CAD89BE89E4E0F0E0F8
:1091C2000E94607A0E94F675EB8BFC8BED89FE891A
:1091D200EE0FFF1F0E94FB75EB89FC89E017F10778
:1091E20084F10E942E76AE2FED89FE89B0E0EA0F5F
:1091F200FB1F9F010E9452760E945976E98DFA8DDB
:10920200EE0FFF1F0E946F760E946576ED89FE8940
:10921200EE0FFF1FA98DBA8DAE1BBF0BBA93AA9397
:10922200F801A98DBA8D0E94486C0E946076F801FF
:109232000E946F76EA8DEA930E94154B0F5F1F4FD3
:10924200CBCF0E94C27C6B960895EA81F0E0EBBB23
:10925200F5BBF7E1F09365001F98E6E1E093650046
:10926200F09365001F9AE881F981EBBBF5BB1F986B
:10927200FFE1F0936500EEE1E0936500F093650095
:109282001F9A0C94234DE2E2EBBBE0E0E5BBE7E181
:10929200E09365001F98E6E1E0936500E7E1E09363
:1092A200650008951F9A0895A0910403A23021F445
:1092B200E881AEE3B3E10BC0A0910403A43021F432
:1092C200E881AEE3B3E103C0E881AEE1B3E1F0E0EF
:1092D2000E9495700E94E87A21960895E091040315
:1092E200E23011F4EEE40AC0E43039F4E0E2EA9349
:1092F200A981BA810E94627504C0E0E2EA93E98121
:10930200FA81FA93EA930E94264917C0E091040376
:10931200E23011F4EFE40AC0E43039F4E1E2EA9316
:10932200A981BA810E94737604C0E1E2EA93E981DD
:10933200FA81FA93EA930E94264922960895E091CF
:109342000403E230B9F4E4E4EA930E947876AE0FC3
:10935200BF1FFD01FE2FE0E0AF81B8850E94486C7F
:109362000E942649E5E4EA930E9486750E942649F6
:10937200E6E453C0E33089F4E7E3EA93FF81E0E0F7
:109382000F010E947876EA0FFB1F0E947D760E94F1
:1093920086750E942649E6E340C0E43049F5E7E3DA
:1093A200EA93AF81B8850E946275DF01EB81FC818F
:1093B200AE1BBF0BFD01FE2FE0E00F01AF81B885B0
:1093C2000E9462750E947D76AD81BE810E94737695
:1093D200DF01E981FA81AE1BBF0BBA93AA930E9407
:1093E2002649E6E3EA93AD81BE810E9473761CC0F2
:1093F200E0E5EA930E94DF730E942649E1E5EA93E1
:109402000E9478760E94486C0E942649E2E5EA931F
:109412000E9486750E942649E3E5EA93E981FA8172
:10942200AD81BE81EA0FFB1FFA93EA930E9426499F
:1094320028960895E0910403E33029F4E3E0EA93E7
:10944200E0E1F1E00BC0E43029F4E3E0EA93E0E28A
:10945200F1E004C0E3E0EA93E0E3F0E1FA93EA9397
:109462000E9426490895E0910403E33029F4E3E0E1
:10947200EA93E1E2F1E00BC0E43029F4E3E0EA939D
:10948200E1E1F1E004C0E3E0EA93E8E3F0E1FA931A
:10949200EA930E94264908951A930A93EFE10E94E3
:1094A2008676EBE10E948676EFE10E948676E8EF0F
:1094B200FFEFE0935F0CF093600CE491EF3F39F023
:1094C200E0915F0CF091600C049000920403ECEBCD
:1094D200F3E18F01A0910403A23019F4EEE9F3E164
:1094E2008F01A0910403A43019F4EEE5F3E18F019A
:1094F200F801E491ED3F39F4F80131960E94AB6C2A
:109502000E94BA7919C0EE3F71F4F80131960E94B7
:10951200E87ADF01E0910403F0E0EA17FB0711F0BB
:109522000D5F1F4F09C0F801E491EA93F8013196EB
:109532000E94AB6C0E9426490D5F1F4FF801E49117
:10954200EF3FB1F6EFE00E945A6BE1E0E0930E04C8
:10955200E0930D04E4E1E09313046CDF09911991A7
:1095620008950E948A76AE85AA2362F0AD85BE85F3
:10957200A03FE0E0BE0734F4AB85BC85AF33E1E049
:10958200BE070CF050C00E949276AE0FBF1FA03FE4
:10959200E0E0BE0734F0AD85BE850E946275E987C2
:1095A200FA87EF81F885AB85BC85AE0FBF1FA0346B
:1095B200E1E0BE0734F0AB85BC850E947376EF8391
:1095C200F8870E94B66C0E94B66C0E94B66C0E942C
:1095D200B66CB5DE0E94B66C0E949776498553DE62
:1095E2000BBB15BB2EE13FE100E010E0EF81F885F7
:1095F200E017F10764F050E0451730F02093650062
:10960200309365005F5FF8CF0F5F1F4FEFCF4ADEE9
:109612000E94466B0E94466B0E944B6BEFE3F1E0A7
:10962200FA93EA938CDEC9C00E948A760E949276EF
:10963200EA17FB0741F0EF81F885AB85BC85EA1795
:10964200FB0709F03EC00E949F761CF00E94A6769E
:1096520084F42D853E85ED85FE85E987FA872D8781
:109662003E872B853C85EB85FC85EF83F8872B872E
:109672003C870E94B66C0E9497760E949276EA1707
:10968200FB0749F4F0DEEB85FC85ED87FE87EF8171
:10969200F885E987FA87F7DD0BBB15BB2EE13FE1C1
:1096A2000D851E85E985FA85E017F1073CF02093C8
:1096B2006500309365000F5F1F4FF4CFF3DDBADE14
:1096C2007CC000930B0410930C040E94AD760E94A0
:1096D200B476FF93EF930E94B8760E94B476AF916E
:1096E200BF91EA17FB0780F10E94A676B4F420E04E
:1096F20030E00E94BB76E217F30774F00E94AD7669
:109702000E94C2760E94BB760E94C7760E94D076E3
:1097120058D02F5F3F4FEDCF16C020E030E00E94BF
:10972200B876E217F3077CF00E94AD760E94C2760B
:109732000E94B8760E94C776F9010E94D77641D07E
:109742002F5F3F4FECCF39C00E949F76DCF420E0C0
:1097520030E00E94DB76E217F3079CF00E94B876B5
:109762000E94C2760E94DB76D0010E94607AAF012D
:109772000E94D076FA010E94D77623D02F5F3F4F06
:10978200E8CF1BC020E030E00E94AD76E217F3077D
:10979200A4F00E94B8760E94C2760E94AD76D001F3
:1097A2000E94607AAF01F9010E94D776FA010E9405
:1097B200D77607D02F5F3F4FE7CF0E94C27C2F960C
:1097C2000895EA81FB81FA93EA9388DD0E94E276AA
:1097D2009DDDE2E2EA93E0910B04F0910C04FA932E
:1097E200EA930E942649249608950E94BB7CEC8548
:1097F200FD85309711F40C94984C00910D0410E003
:10980200E0910E041E1710F00C945F4CE885F98568
:10981200FA93EA937BDD2C853D854A855B85022E92
:10982200032A11F40C94574C37FF36C05A934A93CB
:1098320055DDE2E2EBBBE0E0E5BBE7E1E09365008A
:109842001F98F6E1F0936500E0936500EE81EBBBB3
:10985200EF81E5BBEFE1FEE1E0936500F093650087
:10986200E093650001FF04C0F0936500E09365009A
:1098720036FF11C0F0936500E093650001FF06C05A
:10988200F0936500E09365004F5F5F4F220F331F37
:109892004F5F5F4FEDCF1F9A220F331F01FF02C0B0
:1098A2004F5F5F4F4F5F5F4F0C94104CE885F98517
:1098B2003196E887F9871F5F0C94014C38C02297D4
:1098C2000E94BB7CE885EA930E945549EE83FF83A0
:1098D200E985A8E1EA9FF001E25EF84F8F0130E0EE
:1098E200383028F5F801E4915E2F0F5F1F4FF80121
:1098F200E4914E2F407F0E94E7760E94EC76EA8741
:10990200FB87F801E4914E2F440F440F440F440F9C
:109912000F5F1F4FF801E4915E2F0F5F1F4F0E94F0
:10992200E7760E94EC76EA87FB873F5FD9CF0E94F9
:10993200C27C2E9608951A93EFEF0E945671E0931F
:10994200390910E00E947B70E05CF54FE081EF3F47
:1099520031F00E947B700E94F9761F5FF3CF19915C
:1099620008951A930A930091D00BAA81A53411F499
:10997200E0E066C0AA81A23539F4A0913508A13091
:1099820019F40E94FC7609F405C00E94341BE0E041
:10999200E0933508AA81AB3411F0A33599F4E02F96
:1099A200E470E43011F414E001C013E0E02FE2703F
:1099B200E23009F41C5FE02FE170E13009F41F5F2F
:1099C200E12F3EC0AA81A13511F0A13799F4E02F11
:1099D200E470E43011F417E001C016E0E02FE27009
:1099E200E23009F41C5FE02FE170E13009F41F5FFF
:1099F200E12F26C0AA81A33421F0A13411F0A234B0
:109A020041F413E0E02FE170E13009F41F5FE12F30
:109A120017C0AA81A73741F417E0E02FE170E130C7
:109A220009F41F5FE12F0CC0AA81A03441F415E0B4
:109A3200E02FE170E13009F41F5FE12F01C0EFEF89
:109A4200198108812396089524970E94BB7C209156
:109A5200D00BA0914009A53411F00C94EF4DE0E039
:109A6200E09335080E944F71E0E0E0935D0BE091D6
:109A7200D40BE03089F5E0911008A0911108EA17A3
:109A820039F00E940277ED55F84FE081E13009F09C
:109A920023C0E7E7EA930E94AF610E940277E8558C
:109AA200F84F0E949A70FA93EA930E940877EC5555
:109AB200F84FDF010E9405730E940877E755F84FBF
:109AC2000E940D77E2E0E09335080E940277ED559F
:109AD200F84FA2E0A0832FDFE0913508E03011F0CB
:109AE2000C94EF4D0E94FC7611F40C94C94D0E9427
:109AF200291BE1E0E0933508E22FE870E83081F4B9
:109B02000E941277E8EEF3E00E94607ADF010E9481
:109B1200B17C14F4E1E301C0E0E3EA930E94AF6197
:109B2200E22FE074E03411F413E001C012E0E0919E
:109B3200250C0E949F731A930E941B62E22FE4700D
:109B4200E43049F40E941277E0E1F7E20E94927A4F
:109B5200AF0114E006C00E9412770E948772AF0123
:109B620013E0E22FE071E03111F4415050405A937A
:109B72004A931A930E941B62E22FE072E03211F4C0
:109B820014E001C013E0E091280CF091290C17C0F9
:109B920018E0E22FE470E43009F41F5FE22FE8706E
:109BA200E83009F41F5FE22FE072E03209F41F5F30
:109BB200E22FE074E03409F41F5FE0E0F0E0FA9392
:109BC200EA931A930E941B62E22FE170E13029F4BA
:109BD200E0915D0BEA930E94AF61ADDEA091400976
:109BE200A73729F4E2E0E0933508E03009F473C0C6
:109BF2000E944F710E9417770E940A721E2F0E94C4
:109C02002572AF01E1E0EA930E9456610E2FE091C6
:109C12001008A0911108EA1739F00E940277ED5559
:109C2200F84FE081E23009F053C00E940277EC5510
:109C3200F84FDF010E94D97A4E175F0711F00C949A
:109C4200654E0E940277E655F84F008011800E940F
:109C52000D6D0E94E470EA17FB0769F10E9402771A
:109C6200E655F84FDF010E94D97A0E941D770E94C3
:109C72000277E655F84FDF010E94D97AEB59F44F8B
:109C8200E0810E9425770E942C770E948E6C0E94B0
:109C92002F77E3EEF6E10E940672003029F05A9324
:109CA2004A930E94E26102C00E9435770E9439778E
:109CB2000E94996209C0003039F00E943D7720F479
:109CC2000E94FA720E945025E1E1F8E00E94447776
:109CD200E0E0E0933508A0914009A33421F40E940A
:109CE2009132E03009F40BC00E944F710E94177745
:109CF2000E9494720E94466B63D30E94DA1BA09169
:109D02004009A13411F0A23421F40E944F710E9443
:109D12001777A0914009A03421F40E949132E030DB
:109D220009F420C00E940A72E887F987E2E0EA9308
:109D32000E9456611E2F0E9448770E9408170E94B7
:109D420041730E944E77E152F84F10830E94417393
:109D5200E652F84FA7E0A0830E9423710E944F7140
:109D62000E941777A0914009AB3439F0A33529F04E
:109D7200A13519F0A13709F076C00E949132E03086
:109D820011F40C942E4F0E944F710E945577E1E41A
:109D9200F9E00E942072E22FE270E23029F4E4E05E
:109DA200EA930E94566102C0E1E0F0E0E887F98799
:109DB200A0914009A13511F0A13721F40E9425722A
:109DC2001E2F02C01091E60BE22FE470E43011F472
:109DD200E4E001C0E3E0EA930E945661AF01A09182
:109DE2004009A33511F0A13731F4E885F9850E94C5
:109DF200D479E887F9870E943D7720F0A091D40BAF
:109E0200A13011F51A935A934A93EB85FC85FA9384
:109E1200EA930E94F91B0E94B476EE83FF83AE811F
:109E2200BF810E94B17C84F40E944F71E6E6EA93FE
:109E32000E94AF61EE81FF813197EE83FF83AE8195
:109E4200BF810E94B17C94F31A935A934A93EB8593
:109E5200FC850E94DD716FDD06C00E9494720E9433
:109E6200466B0E94F91B0E94C27C2A9608950E94AA
:109E72005977E89422F80E941973E2E7EA930E9464
:109E8200AF61E0913B08EA930E94AF61EFE0EA9391
:109E92000E94AF61A0913808AA3219F41A9363D3D1
:109EA2001AC0A0913B080E947B70EB59F44FE081ED
:109EB200EA1721F4E0913B08E03349F40E94D56BA4
:109EC200AB59B44FE0913B08EC931A934CD322FC6C
:109ED20002C00E949962C0C20E945977E0913B0879
:109EE200E053AE2F0E947B70EA58F44FE081EA17EC
:109EF20041F51A9338D3A0913608A23019F40E9482
:109F0200617709F402C00E946777A0913608A330F6
:109F120019F40E94617709F402C00E946777E0E0B9
:109F2200E0933608E093630C0E947B70EA58F44F8A
:109F3200BF01E081EF5FAE2FEAE00E948F7ADB0182
:109F4200EC938AC2E881E03019F40E94357706C0AA
:109F5200E881E8500E949F730E94E2612196089571
:109F62000E94BB7C25FC28C20E94617711F40C94EC
:109F720031510E946A77E752F84F9F01D901119639
:109F8200EC91E43071F50E9470770E9473770E9421
:109F92007A77F901A681A03021F4A281B3811097CA
:109FA20009F007C0E6EEF6E10E9406720E943977D8
:109FB20015C00E942C770E947E770E942F77E9EECF
:109FC200F6E10E9406720E9482770E948877F90168
:109FD200A085B185BA93AA930E94E2610E948E770E
:109FE200EBC1E730C9F40E9470770E9473770E9438
:109FF2007A77ECEEF6E10E9406720E9482770E9466
:10A002002F77EFEEF6E10E9406720E947E770E94A1
:10A01200E2610E948E77D0C1E93089F40E947077A4
:10A022000E9473770E947A77E2EFF6E10E9406724D
:10A032000E9495770E942F770E948E77BDC1E630ED
:10A0420029F5EAE2EA930E947E62E5EFF6E10E94D8
:10A052000672D901EC910E949877E091CE0B0E9492
:10A062009877EBE4EA930E94AF610E947E770E94A8
:10A07200E261E4E5EA930E94AF610E9482770E9466
:10A08200E2610E9499620E94677796C1E530C9F445
:10A092000E94EB720E941D77D901EC910E942577F4
:10A0A2000E942C770E947E770E942F77E3EEF6E1E2
:10A0B2000E9406720E9482770E94E2610E948E775D
:10A0C2007BC1E83039F50E9470770E9473770E9455
:10A0D2007A77E8EFF6E10E940672F901A681AA9367
:10A0E2000E94F772309719F00E940C6F04C0D901D8
:10A0F2001696EC91F0E0FA93EA930E94E2610E94D4
:10A1020039770E949962D9011196E0E0EC930E949E
:10A11200677752C1E130C9F5A0911908A53029F439
:10A12200E091CE0BE65F1E2F01C011E0E12F0E94ED
:10A132009C770E947B700E94A1770E94A4770E9464
:10A142002C770E947E770E942F77EBEFF6E10E9438
:10A1520006720E9482770E948877D9011796EC9145
:10A162000E949F730E94E261A0911908A53041F4F8
:10A172000E94A877A481B581BA93AA930E945562DE
:10A182000E949D740E94AE7717C1E330B1F40E9421
:10A19200EB72F0960E94B9770E94EB720E94A1774F
:10A1A2000E94A477EEEFF6E10E9406720E94827787
:10A1B2000E94BD770E94AE77FFC0EB3069F50E9426
:10A1C200C0770E94C3770E94A477E1E0F7E10E9482
:10A1D2000672F901A681AA93B5DE0E94A877A7812B
:10A1E200AA93B0DE0E94A877A085B185BA93AA93FC
:10A1F2000E9488770E9482770E948877F901A48161
:10A20200B581BA93AA930E9488770E9495770E949B
:10A21200BD770E94AE77D0C0EC3089F40E94C0773F
:10A222000E94C3770E94A477E4E0F7E10E940672DD
:10A232000E9495770E94BD770E94AE77BDC0EE3036
:10A2420079F40E94C0770E94C3770E94A477E7E066
:10A25200F7E10E9406720E949D740E94AE77ACC024
:10A262000E94FC7661F0A0913608A03041F4A091E2
:10A27200D30BA13021F40E940D6DE13009F426C008
:10A28200A091860BA03059F0E091880BF091890BD8
:10A29200FA93EA93E8EEF3E00E949E72B9F4E1E3E6
:10A2A2000E94B977E091770BE05D0E9425770E94CA
:10A2B2000D6DEA930ED1E09336080E949D74E093EF
:10A2C200610CF093620CE0E0E093860BA0913608FB
:10A2D200A03059F0E091610CF091620CFA93EA938C
:10A2E200E4E6F0E00E949E7209F025C0A0913608D3
:10A2F200A23019F40E94617709F402C00E946777C4
:10A30200A0913608A33019F40E94617709F410C0B5
:10A31200A091630CA33030F00E946777E0E0E093F5
:10A32200630C06C00E946A77E652F84FA8E0A08349
:10A33200E0E0E0933608A091870BA130E9F5E091C7
:10A342003A0CA091390CEA1791F1EAE20E94B9772E
:10A35200E091750BE05D0E942577E0913A0CEA935B
:10A362000E94911D0E942C77E0912A0C0E949F73FB
:10A372000E942F77EAE0F7E10E9406720E940770BE
:10A38200FA93EA930E9488770E948A730E94C777A1
:10A392000E949962E0913A0CEA930E94D31BE091E9
:10A3A2003A0CEA930E94A21BE0933A0C05C0E0E04B
:10A3B200E093870B689420F80E94C27C2696089549
:10A3C2001A930A930E949132E030D9F00E944173AD
:10A3D200E752F84F8F01EC81FD81D8011296ED937F
:10A3E200FC93EA81FB81D8011896ED93FC93EE81F0
:10A3F200D8011696EC93D8011196E4E0EC930E94F2
:10A4020023711981088127960895E091420BEA93FE
:10A412000E94AF61E091430BEA930E94AF610895FD
:10A42200F4DF0E94E2760E94CA770E94CA770E94F5
:10A432002F7797C01A930E94E2601E2F103021F0EE
:10A44200E12FE150E093400BE0DFE091400BEF5F42
:10A452000E949F730E942F77199108950E94BD7CDC
:10A4620031E00E94D17728F00E941472AC91A4339B
:10A4720008F02AC030E00E941472EC91E270E69576
:10A482001E2F0E941472EC91E1700E2FA0915A0BB4
:10A492001A1729F4E1E0EA27E0935A0B31E0A09180
:10A4A2005B0B0A1729F0E1E0EA27E0935B0B31E04E
:10A4B200E0915B0BEE0FE05DA0915A0BEA0FEA937D
:10A4C2000E94AF610E940A73E32F0E94C47C24960B
:10A4D20008951A9310E00E94FC7611F40C94B05285
:10A4E2000E94291BEEE0F7E10E940672E091250C22
:10A4F2000E949F730E942F77E1E1F7E10E940672AA
:10A50200E091280CF091290C0E94C7770E941277E3
:10A51200A031E7E2BE074CF4E4E1F7E10E940672E3
:10A52200E091260CF091270C13C0E7E1F7E10E94BD
:10A532000672E9810E94216F0E941277EA0FFB1FC7
:10A542000E94C26FE091260CF091270CE051F74275
:10A55200FA93EA930E94E2610E94397711E0E12FB7
:10A5620018812296089524970E94BB7C0E94D57779
:10A57200E0E0EC930E948960E13010F40C9497556E
:10A58200E091420BEB3441F4E091430BE33219F4D6
:10A592000E94E2601E2FC7C2E435A9F4E091430B8A
:10A5A200E33221F40E94E260EE83FF83E091430BE9
:10A5B200EF3441F40E94E2601E2F1A930E94DF736F
:10A5C2000E940817B0C2E23411F00C942F54E091AB
:10A5D200430BE13251F4AA85AF3F29F40E949472F1
:10A5E2000E94466BEDDE0E94DA1BE091430BE134E0
:10A5F200E1F40E94E2601E2F113071F4A09136083E
:10A60200A13019F40E94FC7609F402C00E94341BA6
:10A61200E0E0E093860B09C0E1E0E093860B0E9444
:10A622005E67E093880BF093890BE091430BE5346E
:10A63200A9F4EAE1F7E10E9406720E94111BF39766
:10A642003CF00E94E2600E94C26F0E94DA7701C071
:10A65200E0E3EA930E94AF610E943977E091430BF5
:10A66200E63409F50E94E67719F40E94E260AF0130
:10A67200E885F9850E94116F0E2FE091E60BE0301C
:10A6820011F01091E60B003420F0A091D40BA13010
:10A6920021F40E94F2770E94F91BAA85AF3F19F4B8
:10A6A2000E94F2778DDEE091430BE23511F00C94BB
:10A6B200EC530E94E67719F40E94E260AF0130E0A9
:10A6C200A091D40BA03021F40E940D6DE13009F06D
:10A6D20027C00E949732E03011F10E94D171EC55EF
:10A6E200F84FA885B985A083B1830E94D171E65540
:10A6F200F84FDF01EA850E941F710E94D171E8556F
:10A70200F84F10830E94D171E755F84F40830E94A1
:10A71200D171ED55F84FA1E0A0830E94D77159C0C5
:10A722000E949132E23010F40C94EA530E9448776E
:10A732000E940B1D3E2F3F3F29F00E94DA6FA417A3
:10A74200B5070CF412C00E948A73E41BF50B0E9439
:10A75200E86F0E94AE7119F4E0E0E0932A0C3A939C
:10A762000E94981D689420F803C0E0E0E887E9871A
:10A772000E944173E752F84FDF01EA85F0E0EB599E
:10A78200F44FE081EC930E9441730E944E77EF51A7
:10A79200F84FDF01EA850E941F710E944173E15266
:10A7A200F84F10830E944173E652F84FA5E0A08350
:10A7B2000E942371E885F985309759F00E94487705
:10A7C200FA010E94D4790E94DD710E94F2770E9400
:10A7D200831B689422F8E091430BE335F1F50E9464
:10A7E200E260E887F9870E946A77DF01E652F84F54
:10A7F200E081E23081F4FD01EF51F84F00801180D9
:10A802000E940D6D0E94E470EA17FB0721F4A091EB
:10A812003608A23009F01FC00E946A77E552F84F4D
:10A82200DF010E94D97ADF01E885F985EA17FB0783
:10A8320079F40E946A77DF01ED51F84FE081EA93E3
:10A84200FD01E752F84FE081EA930E94502503C0D0
:10A85200E7E0E0932406689422F865C1E43411F03D
:10A862000C949754E091430BE33559F4EDE1F7E191
:10A872000E9406720E94785D0E949877E1E0E09360
:10A882003909E091430BE03511F00C9496540E9483
:10A89200F67711F40C94965420E00E94FC7740F075
:10A8A2000E941472AC91A23219F00E94007809F44D
:10A8B2003CC0E22FE03061F40E941472AC91A332EA
:10A8C20011F421E004C00E9404780E94535D2AC062
:10A8D200E13051F40E941472AC91A43211F422E0DE
:10A8E20001C020E010E01EC0E23011F0E330D1F4EC
:10A8F2000E9404780E943667EF3F99F0E12FE295BB
:10A90200E07FEF930E9404780E943667AF91EA0FCE
:10A912001E2F2F5F243021F41A930E94535D20E0F2
:10A9220001C020E00E940A73B8CFFDC0E33411F0E9
:10A932000C940755E091430BE534B9F4EAE1F7E1F1
:10A942000E9406720E94111BF3974CF00E94E26073
:10A95200E05FF84D0E94C26F0E94DA7701C0E0E327
:10A96200EA930E94AF610E943977E091430BE6348B
:10A97200D9F441E050E00E94E2600E2F0E94087874
:10A98200E13019F40E94E260AF01E091E60BE030A1
:10A9920011F01091E60B1A930E94BA6BE05FF84D2A
:10A9A2000E94BE750E94F91BE091430BE335A1F4AE
:10A9B2000E940C780E94076FE83141F4E0918A0B03
:10A9C200EA930E94B716689420F806C0E885EA93D5
:10A9D200EFEFEA930E945025E091430BE134A9F492
:10A9E200E0E2F7E10E9406720E940C78EA930E946C
:10A9F200B4170E948324E03011F0E1E301C0E0E3E8
:10AA0200EA930E94AF610E9439778DC0E63511F05A
:10AA12000C946C55E091430BE33411F00C946B559C
:10AA22000E94E2601E2F113010F40C946B55A0911D
:10AA32001908A13091F50E940878E03021F0A09128
:10AA4200A2061A1709F028C011500E94E260AF0155
:10AA52001A930E9414203E2F0E944E720E949570FB
:10AA62000F010E944E720E94FB6C0E9413780E949A
:10AA72000878E03071F00E94E260AF010E946272D9
:10AA82000E9495700F010E9462720E94FB6C0E94EC
:10AA920013781A930E946F101DC01630D8F411500B
:10AAA200A12FEAE00E943F7AA3E2EA9FF001E85573
:10AAB200F94FBF01A12FEAE00E948F7AF0E0BB01BB
:10AAC200AAE0B0E00E940D7ADB01AE0FBF1F149620
:10AAD2000E942F7028C0E93431F5E091430BE03534
:10AAE20051F40E94E2601E2FE0E0EA931A930E9462
:10AAF2008717E0932E06E091430BEC34A1F40E94F9
:10AB0200A460E09328060E940878E03021F00E94B9
:10AB1200A460E09329060E940878E03021F00E94A8
:10AB2200A460E0932A060E94436024CD0E94C27C66
:10AB32002B960895A091580BA03521F4A091590BA2
:10AB4200A03408F005C0E091590BEA930E94D41793
:10AB5200A091580BA33521F4A091590BAA3008F00B
:10AB620005C0E091590BEA930E94FF17A091580B80
:10AB7200AB3421F4A091590BA03808F005C0E09144
:10AB8200590BEA930E943B18A091580BA63521F469
:10AB9200A091590BA03108F005C0E091590BEA933E
:10ABA2000E946718A091580BA43511F40E94F21666
:10ABB200E1D60895E3EAF6E0FA93EA93E091420BD4
:10ABC200EA93E0E8F0E00E943E6F08950E941B784D
:10ABD200A0E0A083E091400BE093590BE091420B7F
:10ABE200E093580B08950E94BB7C0E948960E1307B
:10ABF20010F40C940F59E091580BA091420BEA17F4
:10AC020009F098DFE091420BE33239F5E091430B12
:10AC1200EC3431F4CFDFE4E0E09318080E942178AD
:10AC2200E091430BE435C1F4C5DFE091660CE030FE
:10AC320029F0EF77A9E0B0E00E941B7BE091670C5E
:10AC4200E03029F0EF77AAE0B0E00E941B7B0E947F
:10AC52002178E7E0E0931808DEC2E934E9F4E091F4
:10AC6200430BE434C1F40E94F677A9F010E010E03F
:10AC7200183178F4A3E2B7E00E947B70EA0FFB1F61
:10AC8200FF93EF930E94A460AF91BF91EC931F5F7B
:10AC9200EFCF0E941D0CBFC2EB34E1F5E091430BF4
:10ACA200E13211F487DF35C0E53211F443DF31C000
:10ACB200E33299F40E94277821F00E9432780E94B0
:10ACC20009180E941B78E081EB3429F4E0E0E0935C
:10ACD200350CE093360C7ADF1CC0E134D1F40E94CB
:10ACE200E2609F012093350C0E94387891F00E9417
:10ACF200E2609F01A091350CF901E270F070EA2B3D
:10AD0200E093350C0E94387821F00E94E260E093D3
:10AD1200360C81C2E33581F5E091430BE13211F447
:10AD220049DF29C0E33299F40E94277821F00E947A
:10AD320032780E94E3170E941B78E081E33529F400
:10AD4200E091400BEA930E94241A40DF14C0EE34D3
:10AD520091F40E94C27310E01A3068F4A4EBBBE0D5
:10AD6200EE27A10FBE1F0E947B70EC5BF44FE081C7
:10AD7200EC931F5FF1CF4FC2E63511F00C940957E7
:10AD8200E091430BE13211F415DF41C0E33299F453
:10AD92000E94277821F00E9432780E9447180E9470
:10ADA2001B78E081E63529F4E091400BEA930E949A
:10ADB2007A180CDF2CC0E63531F40E94E2609F0164
:10ADC2002093310C24C0E53471F40E94E2609F01AB
:10ADD2002093300C0E94387829F00E94E2609F0193
:10ADE2002093330C14C0E43591F440E050E00E940B
:10ADF200E2609F01022E032A11F042E050E00E941D
:10AE0200387819F00E94E260AF014093320C03C21D
:10AE1200E43511F00C94C357E091430BE33231F463
:10AE22000E94E2603197E093400BABC0E03511F035
:10AE32000C94C25710E00E94FC7750F00E941472EA
:10AE4200AC91AD3329F00E94007811F01E3008F069
:10AE520005C00E947B700E943E78EDCF0E947B70FD
:10AE62000E944778EDE30E944C7811F00C94C2578F
:10AE7200E4E5E093580B10E00E94A06F3496E49151
:10AE8200EF3F11F40C94C2570E94C6730E94A06F48
:10AE92000E94AB6C0E940768E03011F00C94C0571E
:10AEA2000E94A06F3496E491E03851F40E94E2606F
:10AEB200E058FF4FE093660CE0E8E093670C5FC058
:10AEC200E23839F40E94E260E058FF4FE093670CE9
:10AED20056C0E13839F40E94E260A8E0B0E00E9476
:10AEE2001B7B4DC0E03011F0E13051F40E94966FAF
:10AEF200FF93EF930E94E260AF91BF91EC933FC04A
:10AF0200E23059F40E94966FFF93EF930E94E26041
:10AF1200AF91BF91ED93FC9332C0E33051F40E94A4
:10AF2200966FFF93EF930E94C160AF91BF91EC9334
:10AF320026C0E43021F50E94A06F3596E491EA9391
:10AF42000E9490610E94966FE093640CF093650CEE
:10AF520000E00E94A06F3596E4910E1780F40E94E3
:10AF6200BA6BEC5BF44FE081A091640CB091650C7C
:10AF7200EC93A4E6BCE00E94B06D0F5FEACF1F5FC6
:10AF82007BCF49C1E03511F00C940C59E091430B91
:10AF9200E33299F40E94277821F00E9432780E94CD
:10AFA200B4170E941B78E081E03529F4E091400B50
:10AFB200EA930E94391A0ADE2EC1E13211F4FADD57
:10AFC2002AC1E134D1F40E94E2601E2F00E00D306C
:10AFD20098F40E94E873EA0FFB1F3396E491E1179D
:10AFE20049F40E94E8730E94EC73A0919B0BEA2B38
:10AFF200E0939B0B0F5FEBCF0EC1E63559F5E0E016
:10B00200E093410BAEE9BBE00E945178FF93EF93CE
:10B012000E94E260AF91BF91EC93EBE2EA930E944F
:10B022005360E03059F0A1EABBE00E945178FF93EF
:10B03200EF930E94E260AF91BF91EC930E9454782B
:10B04200A091410BA33018F40E94387809F401C092
:10B05200D9CFE1C0ED34D1F4E0E0E093410BAAEAAC
:10B06200BBE00E945178FF93EF930E94E260AF91A0
:10B07200BF91EC930E945478A091410BA33018F435
:10B082000E94387809F401C0EACFC5C0E735D1F48F
:10B09200E0E0E093410BA1EBBBE00E945178FF930B
:10B0A200EF930E94E260AF91BF91EC930E945478BB
:10B0B200A091410BA23018F40E94387809F401C023
:10B0C200EACFA9C0E434C9F5E0E0E093410B0E9465
:10B0D200E2609F01E2E0EA930E946060AF01E3E771
:10B0E2000E944C7859F40E945A78BF01D9010E94FB
:10B0F2001A71E40FF51FDB01ED93FC93E9E40E9462
:10B102004C7879F40E945A7820833183ABE9BBE012
:10B112000E9451780F010E946178EC91E160D001A8
:10B12200EC930E945478A091410BA33018F40E9432
:10B13200387809F401C0CBCF6EC0EE3499F40E9486
:10B14200C27310E01A3068F4ABE8BBE0EE27A10F3F
:10B15200BE1F0E947B70EC5BF44FE081EC931F5F9B
:10B16200F1CF59C0E33459F4E2E2EA930E9453600A
:10B172000E94E260E093960BF093970B4CC0E3358C
:10B1820089F40E94E2609F0100240216030624F45F
:10B192002B30E0E03E070CF004C0F9013197E09358
:10B1A200980B39C0E53529F40E94E260E0939A0BCE
:10B1B20032C0EF3491F40E94E2601E2FECE2EA9377
:10B1C2000E945360E12FE295E07FEF930E94E260DC
:10B1D200AF91EA0FE093990B1EC0E035E1F4E0E095
:10B1E200E093410BADEABBE00E9467780E94957044
:10B1F200FF93EF930E947061AF91BF91ED93FC9327
:10B202000E945478A091410BA23018F40E94387821
:10B2120009F401C0E7CF0E944360E7CC0E94C27CE0
:10B22200269608950E94BD7C0E948960E13010F448
:10B232000C94E45BE091420BE332A9F4E091430BFE
:10B24200E03519F4E3E2F7E109C0E83419F4E4E483
:10B25200F7E104C0E33531F4EFE5F7E1FA93EA935D
:10B262000E94C061ADC2E934C1F4E091430BE43401
:10B2720099F40E94120CC9D80E946B7810E0183120
:10B2820048F4A3E2B7E00E94A674EA930E94F06138
:10B292001F5FF5CF0E946B7893C2E43511F00C94D6
:10B2A200EA59E091430BE43229F4E8E2F0E00E942B
:10B2B2006F788EC0E33211F4BDD88AC0E03511F048
:10B2C2000C94E959A2D8A091400BA83210F00C942A
:10B2D200E9590E9473780E94AB6C0E94C061EDE351
:10B2E200EA930E94AF610E9473783496E491E03849
:10B2F20039F40E940D6D0E949F730E94E26168C042
:10B30200E23839F40E94916F0E949F730E94E261B9
:10B312005FC0E13839F40E949A730E949F730E94C1
:10B32200E26156C0E03011F0E13051F40E947378CE
:10B3320032960E94E87A0E949A700E94777848C0FA
:10B34200E23059F40E94737832960E94E87ADF0163
:10B352000E9405730E94E2613BC0E33051F40E94F7
:10B36200737832960E94E87AE081EA930E94FF6144
:10B372002FC0E43069F50E94737832960E94E87A11
:10B38200E093640CF093650C10E00E94737835969C
:10B39200E4911E1790F40E947B70EC5BF44F0F0156
:10B3A200A091640CB091650CEC91D001EC93A4E6F1
:10B3B200BCE00E94B06D1F5FE8CF0E9473783596A3
:10B3C200E491F0E00E9447780E94C6730E944C62AA
:10B3D200F7C1E33581F5E091400BEA930E94E31750
:10B3E200E091430BE43229F4EAE0F0E00E946F7846
:10B3F20021C0E33211F41ED81DC0EE34D9F40E94EC
:10B40200065210E01A3068F40E947B70EC5BF44F35
:10B412000F01A4EBBBE00E94A674D001EC931F5F66
:10B42200F1CFE0E0E0934E0B0E94C6730E944C62A3
:10B432000E943977C5C1E63511F00C945D5AE0914E
:10B44200400BEA930E944718E091430BE43229F43F
:10B45200E5E0F0E00E946F782EC0E33219F40E941A
:10B462001B5229C0E53459F40E940652E091300C77
:10B472000E949F730E947B78E091330C19C0E635DD
:10B4820029F40E940652E091310C12C0E43599F47D
:10B492000E940652E091320CE03011F0E1E301C06B
:10B4A200E0E3EA930E94AF610E948178E091320C5E
:10B4B200F0E00E94C77784C1E03511F00C94AE5BD6
:10B4C200E091400BEA930E94B417E091430BE432FF
:10B4D20029F4E0E4F0E00E946F783EC1E33219F40F
:10B4E2000E941B5239C1E13411F00C94BA5A0E94E5
:10B4F200065212E0A0919B0BECEDEA233E2F00E0F6
:10B502000D3078F40E94E8730E94EC73E31739F46B
:10B512000E94E873EA0FFB1F3396149102C00F5F7B
:10B52200EFCF0E948E6C0E942F77E091990BE03052
:10B5320089F0EAE7F7E10E9406720E94686C0E94B5
:10B542009F730E947B78E091990BEF700E949F732A
:10B552000E942F77E0919A0BE03051F0EDE7F7E18E
:10B562000E940672E0919A0B0E949F730E942F77AD
:10B57200F3C0E43479F50E948578A091410BA330A1
:10B5820040F5E091410BE03011F00E9481780E9479
:10B592006178EC91E17061F4A4EABBE00E94677803
:10B5A2000E94FB6C0E9405730E945562E3E70BC088
:10B5B200A4EABBE00E9467780E94FB6C0E940573BC
:10B5C2000E94E261E9E4EA930E94AF610E9454782A
:10B5D200D4CFBEC0ED34C9F40E948578A091410B4E
:10B5E200A33090F4E091410BE03011F00E94817899
:10B5F200AAEABBE00E948B78EC910E949F730E94A2
:10B60200E2610E945478EACFA3C0E735C9F40E94F0
:10B612008578A091410BA23090F4E091410BE0308B
:10B6220011F00E948178A1EBBBE00E948B78EC9133
:10B632000E949F730E94E2610E945478EACF88C000
:10B64200E63531F50E948578A091410BA330F8F4DC
:10B65200E091410BE03011F00E948178AEE9BBE04D
:10B662000E948B78EC910E949F730E94E261EBE250
:10B67200EA930E94AF61A1EABBE00E948B78EC9151
:10B682000E949F730E94E2610E945478DDCF60C0E5
:10B69200EE34D1F40E94065210E01A3068F40E948F
:10B6A2007B70EC5BF44F0F01ABE8BBE00E94A67429
:10B6B200D001EC931F5FF1CFE0E0E0934E0B0E94CC
:10B6C200C6730E944C6244C0E33499F40E9406524D
:10B6D2000E94C673E5E8F7E1FA93EA930E940C6FC1
:10B6E2000E941E730E94A1740E94C6730E944C6243
:10B6F2002FC0E035A9F40E940652E091AD0BF09103
:10B70200AE0BFA93EA930E946D620E948178E091F7
:10B71200AF0BF091B00BFA93EA930E946D6218C0DE
:10B72200E33531F40E940652E091980BEF5F0DC0B1
:10B73200EF3491F40E9406520E94686C0E949F733B
:10B742000E947B78E091990BEF70F0E00E9477788D
:10B75200EBE3EA930E94AF6133C0EB3489F5E091E9
:10B76200400BEA930E940918E091430BE43229F45A
:10B77200E0E8F0E00E946F7823C0E33219F40E94FF
:10B782001B521EC0E134E1F40E940652A091350C16
:10B79200E1E0EA230E949F730E947B78A091350C1E
:10B7A200E3E0EA230E949F730E947B78E091360CCB
:10B7B2000E949F730E94E261E8E8F7E10E9406722C
:10B7C2000E94436031CD0E94C47C249608951A934E
:10B7D2000E944F71E0E4F9E00E9420720E948F788B
:10B7E200E181E43471F40E948F7802800E940D6D31
:10B7F200E05DE01529F00E948F78E281EA3209F4D7
:10B8020001C05BC00E9494780E948F78E1810E94FF
:10B8120098780E948F78E2810E9498780E94147230
:10B822001C910E948F7833960E942072E12FE231A0
:10B8320039F40E94D5771397E6E0EC93D4D93DC052
:10B84200E13139F40E94D5771397E2E1EC93EADC17
:10B8520034C0EF30B1F40E94D5771397EEE0EC9349
:10B862000E942F52E13039F4A0913508A03019F02E
:10B872000E94FC7609F402C00E94341B0E949B784D
:10B882001CC0EE30D1F40E94D5771397EFE0EC9311
:10B892000E942F52E13089F4A0913508A03019F0AE
:10B8A2000E94FC7609F402C00E94341BE0E0E0939F
:10B8B2003508EFEFEA930E94B4520E94D577E0E098
:10B8C200EC936BC21A930E9419730E946E6FEAE79F
:10B8D200EA930E94AF610E94147211971C91E12FAA
:10B8E200E23131F4E6E0EA930E94AF617CD937C0DD
:10B8F200E13131F4E2E1EA930E94AF6193DC2FC0BF
:10B90200EF3099F40E94A4770E942F52E13039F46B
:10B91200A0913508A03019F00E94FC7609F402C00B
:10B922000E94341B0E949B781AC0EE30C1F4EFE0F3
:10B93200EA930E94AF610E942F52E13081F4A091FC
:10B942003508A03019F00E94FC7609F402C00E946A
:10B95200341BE0E0E0933508EA930E94B4520E945F
:10B96200D577E0E0EC93A0913808AA3211F00E945A
:10B97200996213C2EFEFE093580BE093590B0895CD
:10B98200AC81A03310F0AA3308F006C00E94A2785E
:10B99200E0530E94AA78A1C4AC81A13410F0A7346C
:10B9A20008F006C00E94A278E7530E94AA7895C4C4
:10B9B200A881B981E0E0EC9390C4AA93EA93FA9348
:10B9C200EFB7EA931A930A931BB10CB1E091A00C62
:10B9D200F0E0E259F34F0083A091A00CAF5FA09377
:10B9E200A00CA23319F4E0E0E093A00C09911991A4
:10B9F200F7C21A93E091A10CA091A00CEA17D1F31F
:10BA0200F0E0E259F34F1081A091A10CAF5FA09337
:10BA1200A10CA23319F4E0E0E093A10CBDC1A09106
:10BA2200A00CAE5CE091A10CAE1BE2E30E948F7A07
:10BA320008950A921A92FA926A937A938A939A933F
:10BA4200AA93BA93EA93FA93EFB7EA930E94AF7874
:10BA520049F0A0913909A03021F00E940C0CE1308C
:10BA620009F401C011C0E091070DF0E0EE55F34F6B
:10BA7200E081ECB9A091070DAF5FA093070DA4364A
:10BA820019F4E0E0E093070DE991EFBFF991E99134
:10BA9200B991A9919991899179916991F9901990A6
:10BAA200099018951A930E94AF7859F45D9B09C0CA
:10BAB200A0913909A13021F40E940C0CE03009F068
:10BAC20013C01091060D0E947B70EE55F34FA981B1
:10BAD200A0831F5F143609F410E0E091070DE1170F
:10BAE200E1F31093060D02C0E981ECB9A5C20E94F0
:10BAF200AF7821F40E940C0CE13009F001C01FC3A1
:10BB020054C10E94BD7C8BDFE03011F40C94845E42
:10BB120070DF1E2FA0916B0CA53618F0E0E0E093C9
:10BB22003A0930913A09E0913A09E03011F00C9467
:10BB3200EB5DA091E50BA13041F0A091E50BA230A5
:10BB420021F0A091E50BA53031F4E12FEF77E093DE
:10BB52004009EBE4CEC01A3521F4E1E0E0933A0962
:10BB6200CAC0123049F4E4E1E0933A09E0E0E0931C
:10BB72003B09E0933D09BFC0A091E50BA33069F4F6
:10BB8200173729F01A3310F4103308F402C0E7E033
:10BB920001C0E0E0E0933C0905C01A930E94B24C58
:10BBA200E0933C09A0913C09AF3F99F01093400902
:10BBB200E1E0E0933B0910933D09E0913C09E0305C
:10BBC20011F4E5E404C0EAE0E0933A09E0E0E0932E
:10BBD2003F0991C0E13069F4103039F4E2E0E093BA
:10BBE2003A09E0E0E0933F0903C0E0E0E0933A095C
:10BBF20082C0E23059F410933C0910933D09E0E011
:10BC0200E0933B09E3E0E0933A0975C0E330F1F4D5
:10BC12000E94B5780E94BB78EA0F0E94C578A9F409
:10BC2200E0913D09E03071F4E4E0E0933A09E091FB
:10BC32003B090E94B46E0E94CE780E94B578A0E0C3
:10BC4200A08303C0E0E0E0933A0955C0E43049F430
:10BC52001D3019F4EAE5E0933F09E0E0E0933A0988
:10BC62004AC0EA3079F40E94B5780E94BB78EA278C
:10BC72000E94C57831F4E0E0E0933A09E5E4E0930C
:10BC82003F0939C0E431B9F40E94B5781083E12F3D
:10BC9200A0913D09EA27E0933D09E0913B09EF5F5E
:10BCA200E0933B09E0E0E0936A0C133019F4E5E11C
:10BCB200E0933A0920C0E53111F0E63159F41A93C4
:10BCC200EAE6FCE0FA93EA93EAE3F9E0FA93EA930C
:10BCD20057DE11C0E73179F4E0E0E0933A09173119
:10BCE20031F4E0916A0CA0913D09EA1709F003C012
:10BCF200E3E4E0933F09A0913A093A1719F0E0E032
:10BD0200E0936B0C00CF0E94C47C56C4AA93BA93F2
:10BD1200EA93FA93EFB7EA931A930A9310919B006E
:10BD220000919C00E12FEC71A9F4E091D00DF0910B
:10BD3200D10DE85FF24F0083A0EDBDE00E94B06D2F
:10BD4200E83CA0E0FA0731F4E0E0F0E0E093D00D47
:10BD5200F093D10D09911991E991EFBFF991E99110
:10BD6200B991A99118951A930E94D3780E94D87814
:10BD7200D9F30E94D378E85FF24F1081A2EDBDE0C3
:10BD82000E94B06DE83CA0E0FA0731F4E0E0F0E098
:10BD9200E093D20DF093D30DE12F199108950E94F3
:10BDA200D3780E94D87809F0CAC1E0E008950E94D1
:10BDB200BD7CF5DFE03021F0A091690CA03009F0E4
:10BDC200E5C0D1DF1E2FA091DC0DA53618F0E0E012
:10BDD200E093D60D3091D60DE091D60DE03059F4B6
:10BDE200113019F4E4E0E093D60D1A3519F4EAE0C3
:10BDF200E093D60DC3C0E430C1F4E0E0E093D60D89
:10BE02001A3229F00E940D6DE05DE11769F410937A
:10BE120038081093D70DE5E0E093D60DE0E0E0930B
:10BE2200690CE1E0E093D90DA9C0E530A9F4E0E0A6
:10BE3200E093D60D0E940D6DE05DE11761F00E9466
:10BE4200DF780E94E878E091D90DEF5FE093D90D99
:10BE5200E6E0E093D60D92C0E63091F4E091D90D80
:10BE62000E94E8780E94DF78EF5FE093D90DE0E06E
:10BE7200E093DA0D133019F4E7E0E093D60D7EC0BB
:10BE8200E73011F0E83059F41A93EAEDFDE0FA9345
:10BE9200EA93E6EDFDE0FA93EA9372DD6FC0E930D2
:10BEA20081F4E0E0E093D60D173131F4E091DA0D40
:10BEB200A091D70DEA1709F003C0E4E5E093690CFD
:10BEC2005DC0EA3041F4103011F4EBE001C0E0E073
:10BED200E093D60D53C0EB3071F4E0E0E093D90D5E
:10BEE2001093D80D1093D70DECE0E093D60DE0E05F
:10BEF200E093690C43C0EC30A1F5E091D90DF0E07C
:10BF0200E05CF64F10830E94DF78EF5FE093D90D7B
:10BF1200E091D80DE150E093D80DA091D80DA0305A
:10BF220021F4A091D70DA03009F00EC0EDE0E0930E
:10BF3200D60DE091D90D0E94B46E0E94CE78E091A8
:10BF4200D90DF0E00E94CE78A091D80DA03021F456
:10BF5200A091D70DA03009F403C0E0E0E093D60D24
:10BF62000DC0ED3059F4E0E0E093D60D1D3031F410
:10BF7200EAE5E093690CEFEFE093680CE091D60DEF
:10BF8200E31719F0E0E0E093DC0D13CF0E94C47CCC
:10BF920013C3AA93EA93FA93EFB7EA93E091DE0E02
:10BFA200A091DD0EEA1791F0E0913708E03019F028
:10BFB200E89426F80AC00E94ED78F0E0E030A1E0B3
:10BFC200FA0719F4E0E0E093DE0E03C0E89425F8E6
:10BFD20026F8E091680CE03019F0E0E0E093D60D2D
:10BFE200E991EFBFF991E991A99118951A93E0911E
:10BFF200DE0EA091DD0EEA1721F4E0919B00E072C3
:10C00200C1F4E091DD0EF0E0E352F24FA981A0838A
:10C012001091DD0E1F5F0E94D56BA030E1E0BE07DC
:10C0220009F410E0E091DE0EE117E1F31093DD0E6A
:10C0320003C0E981E0939C00188122960895E0E014
:10C04200E093DE0EA091DD0EA13020F00E94ED788B
:10C05200689426F80895AA93BA93EA93EFB7EA93FD
:10C06200E091680CE03041F4E0E0E093DE0E0E94E3
:10C072000D6DEF5FE0933708E991EFBFE991B99158
:10C08200A99118950E94FC7718F00E94007809F493
:10C0920003C00E940A73F6CF0E94007811F40E9436
:10C0A2000A7308950E941472AC91E881EA1729F488
:10C0B2000E940A733197E1E060C1E0E05EC10E9434
:10C0C200BD7C00E010E0EEE20E944C78F9F420E042
:10C0D20030E0EC81D901F0E0AE17BF07BCF4D80123
:10C0E2000E94D5738F010E94D17718F00E94FB78CD
:10C0F20008F009C00E941472EC910E948C720E0F1B
:10C102001F1F0E940A732F5F3F4FE3CFF801E3C066
:10C112000E94FC7728F00E948F78E181E03208F4D7
:10C1220010C00E941472EC91E093420B0E940A73B9
:10C132000E941472EC91E093430B0E940A73E1E0B7
:10C1420008950C9498651A930A9300E010E0123057
:10C15200A8F40E9404780E943667EF3F69F0E02F4E
:10C16200E295E07FEF930E9404780E943667AF91D8
:10C17200EA0F0E2F0E940A731F5FE9CFE02F1EC045
:10C182001A930A9310E00E9414720C910B3311F06F
:10C19200003208F412C0013310F0093308F007C06E
:10C1A200E02F0E948C72E255FF4FE4911E2B0E94F9
:10C1B2000A730E9414720C91E9CFE12F099119912F
:10C1C20008950E94BD7C00E010E00E941472AC91C0
:10C1D200AD3221F40E940A7331E001C030E00E94C6
:10C1E200D17718F00E94FB7808F009C0D8010E94AC
:10C1F200D5730E94FF788F010E940A73F0CF30300E
:10C2020021F4F8010E94C47CD7C1F8010E94D479BC
:10C212000E94C47CD1C124971A93E0E0E983EA83A7
:10C22200EB83EC830E941472AC91AD3221F40E9434
:10C232000A7311E001C010E00E94D17718F00E9449
:10C24200FB7808F022C0A981BA818B819C81EAE047
:10C25200F0E060E070E00E943A7A7F936F93FF9380
:10C26200EF930E941472EC91E053AF91BF918F91C2
:10C272009F91FF27662777270E94CA79E983FA836D
:10C282006B837C830E940A73D7CF103031F4E9812B
:10C29200FA816B817C81188120C0E981FA816B81EE
:10C2A2007C810E94D879188118C00E94BD7C20E050
:10C2B20030E000E010E0EC810E9458755CF4D90196
:10C2C2000E94D5730E94FF789F010E940A730F5F3C
:10C2D2001F4FF1CFF9010E94C47C259608950E9458
:10C2E200BD7C6FDF8F0120E030E0EEE20E944C78EF
:10C2F20011F467DF9F01112322F4F9010E94D4791E
:10C302009F01A0911C0CA13030F0D8010E941A713B
:10C31200E20FF31F8F01F8010E94C47C4DC11A93F2
:10C3220010E00E94F677A1F00E94FC7758F00E947C
:10C332001472AC91A23231F00E94007819F0E981B6
:10C342001E1708F005C00E947B700E943E78ECCF59
:10C352000E947B700E9447780C94F465E8810E94E9
:10C362009878E881A0915C0BEA0FE0935C0BE8817E
:10C37200A0915D0BEA27E0935D0B219608951A9335
:10C3820010E0E12FA981BA810E94E473E491E030C8
:10C3920049F0E12FA981BA810E94E473E4910E94DD
:10C3A2000579EFCF0BC01A9310E00E944975E03077
:10C3B20029F00E9449750E940579F7CF18812396CA
:10C3C200089564970E9463740E940A79E88DF98D3A
:10C3D2000E941E730E949374E6DF66960895649726
:10C3E2000E946374E1E9F7E1FA93EA93E88D0E940F
:10C3F200926B0E946374D7DF659608951A93ECE3FB
:10C40200EA93ACDF11E0193080F40E947B70E255B0
:10C41200FF4FE491A981EA2319F0E12FE05D01C009
:10C42200E0E2EA939BDF1F5FEECFEEE3EA9396DF53
:10C432000C94F46564971A93FE013196FA93EA9389
:10C442000E940A79EA8DFB8D0E941E730E94A174DC
:10C45200FE0131960E9490751E2FED891E1720F461
:10C462000E9435771F5FF9CFFE013196FA93EA9366
:10C472009ADF18810EC064970E9463740E940A7941
:10C48200E88DF98D6A8D7B8D0E9472730E946374B0
:10C492008ADF689608950E946B780E94E27683DFB5
:10C4A2000E946B780C94F565A881B981E4E6F0E00E
:10C4B2000E94607A0E947778EEE2EA934FDFA881C9
:10C4C200B981E4E6F0E00E94927AFA93EA93E2E01C
:10C4D200EA93B0DF0C94F565A0911C0CA13020F01A
:10C4E2000E94E276E1DF07C00E94E2766ADFE6E9B7
:10C4F200F7E10E9406720C94F56525FE06C0E5E0A0
:10C50200F0E00E948B6DA895F8CFEDEDFDE0E09391
:10C512005E0BF0935F0BE1E00E945671E0935C0BBF
:10C522000E940F790E940D6D0E9498770C9470689A
:10C532001A930A93E091680CE03011F00C9467674B
:10C54200E3E0EA930BDFE0915C0BE295EF70EA9394
:10C552000E944D671E2FE0915C0BEF70EA930E94E0
:10C562004D670E2F1A93FADE0A93F8DEE7E1EA939B
:10C57200F5DEEDEDFDE00E94D5770E94FC7AEA1B24
:10C58200E093DD0E689425F80C946767EE81EA93D8
:10C59200B4DFEC81FD810E9406720E9413796BDF89
:10C5A200C7DF0C949768EB81EA93A7DF0E9476704D
:10C5B200E6DE0E940F79BCDF24960895ED81EA93AE
:10C5C2009CDFEB81FC810E940672EA81EA93C6DE5F
:10C5D200E981E03011F0EA93C1DEE881E03011F048
:10C5E2000E940F79A5DF269608950E94BB7C10E079
:10C5F200EAE9F7E1A885B985EA17FB0719F444E1EE
:10C6020050E002C048EC50E0EA85E0933809E89433
:10C6120031F8EA93E985FA85FA93EA93EA85EA938F
:10C62200EA85EA93E0E0EA93C9DF0E945E679F0130
:10C632000E94F1130E9498750E946A670E2F31FCC6
:10C6420002C0003009F001C0F3CF31FE04C0E8940B
:10C6520031F8E1E004C01F5F1230B0F2E0E00E9466
:10C66200C27C2B9608951A930A93E091400AE03017
:10C6720011F40C946767E0E0E0933909E2E0EA9391
:10C6820011DA10E003E00E947B700E941A7961F0D7
:10C692000E947B700E94F9760E947B70E05CF54FED
:10C6A200E0810E271F5FEFCFE3E0EA93FBD9E02F93
:10C6B200E295EF700E941F79E02FEF700E941F79C0
:10C6C200E7E1EA93EFD90C9467671A930A93E09132
:10C6D200400AE03011F40C9467670E94916FE030D9
:10C6E20021F0E091420AEA3209F405C00E94916FFA
:10C6F200E05DE093420AE0E0E0933909EAE5EA937B
:10C70200D1D9E0E0EA93CED910E00E947B700E947A
:10C712001A7911F01F5FF9CF1F5F012F0A93C2D957
:10C7220010E00E947B700E941A7961F00E947B7077
:10C732000E94F9760E947B70E05CF54FE0810E0F5B
:10C742001F5FEFCFE02FE195EA93ACD9EDE0EA93DA
:10C75200A9D90C9467671A930A93F894E0E0E093DE
:10C762003708E091DE0EE093DD0E7894E091400A06
:10C77200E03011F40C946767EAE5EA9337DCE0E015
:10C78200EA9334DC10E00E947B700E941A7911F067
:10C792001F5FF9CF1F5F012F0A9328DC10E00E9470
:10C7A2007B700E941A7979F00E947B70E05CF54FF1
:10C7B200E081EA931BDC0E947B70E05CF54FE08134
:10C7C2000E0F1F5FECCFE02FE195EA930FDCEDE057
:10C7D200EA930CDC0C946767E881EA938EDEEAE563
:10C7E200EA93BCDDE0914009EA93B8DD0E9414723D
:10C7F200EC91E03031F00E940478B0DD0E940A73BF
:10C80200F5CF96DE0C9470681A930E944F71E091F6
:10C812003B08EA93A3DDE4E4EA93A0DDE091390862
:10C82200EA939CDD14E00E947B70E85CF74FE081A4
:10C83200E43040F00E947B70E85CF74FE0810E9498
:10C842000579F1CFE0E0EA9389DD3FDF6BC11A930E
:10C852000A9357D9E0913F09E03011F40C94A56492
:10C86200A0913F09AA3541F4A0913B09A33020F0E1
:10C87200E0914109E43409F04BC00E94916FE0302D
:10C8820021F0E0914209EA32C1F40E940D6DE05DAF
:10C89200A0914209EA1721F0E0914209EA3221F41B
:10C8A2000E94E85B12DF08C0E3E4F9E00E94207214
:10C8B200E09142090E9425792BC00E94916FE05DB0
:10C8C200A0914209EA1721F50E940D6D1E2FE091F9
:10C8D2004309ED3421F4E0914409E33209F007C041
:10C8E200E5E4F9E00E9420726CDC1E2FCBDB0E9493
:10C8F2000D6DE11729F0E12FE05D0E94257908C056
:10C902000E940D6DE05DE09342090E94E85BDDDE6E
:10C91200A0913F09A53449F4A091E50BA33019F485
:10C922000E94E12902C00E94254DA0913F09A33433
:10C9320011F40E949229A0913F09AB3411F40E9494
:10C942008D29E0E0E0933F09A091E50BA33011F4BB
:10C952000E94E129E0E00C94676729DAA091690C52
:10C96200A43529F4A0E025FCA1E0A03009F03AC0EA
:10C97200E0913A08E03581F4E0913B08EA93E6E081
:10C98200EA930E94E741A0913B08A03820F0E09191
:10C992003B08E093650523C0E03721F4E0E0E09333
:10C9A20065051DC0EA3519F40E94635C18C0EA37B8
:10C9B20011F42ADF14C0E23519F40E94384F0FC077
:10C9C200E23719F40E946D4F0AC00E94642FE09171
:10C9D2003908A0913809EA1711F4689431F8E0E0B7
:10C9E200E093690CA091690CAA3531F40E94E85BCE
:10C9F200B2DEE0E0E093690C9AC0A0916C0CA13029
:10CA020050F0E0916C0CE150E0936C0CE03019F4C2
:10CA1200E1E0E0936D0CA0E025FCA1E0A13049F437
:10CA2200A0E026FCA1E0A03021F4A0913708A030BC
:10CA320009F001C004DBE0913708E03019F0E15061
:10CA4200E09337080895E091DC0DEF5FE093DC0D91
:10CA5200E0916B0CEF5FE0936B0CE091680CE030BF
:10CA620019F0E150E093680C0895A091E50BA13014
:10CA720041F0A091E50BA23021F0A091E50BA53089
:10CA820029F4E3E0E0939000E8E3E9B90895E09146
:10CA9200620BE0937100E0E0E0937400E2B3E360C4
:10CAA200E2BBE1B3E360E1BB85E38A95F1F7E1B371
:10CAB200EC7FE1BBE4E4E093740088EC90E0019742
:10CAC200F1F70895E2E001C0E0E0E093620BDFDFFE
:10CAD20008951A931FEFF6DF16D0E03089F4E9814A
:10CAE2000E942C7941F4EDB7FEB7FA93EA931F93B3
:10CAF2000E9431791F9118D080E991E00197F1F7F6
:10CB0200E3DFE12F70C01A9314EAE4EA0E94357958
:10CB120041F40E943A79183011F0103111F4E0E03A
:10CB220001C0E2E019910895E4E9E0937400E0E0C5
:10CB320008951A93E981E1600E943F7931F40E94DD
:10CB42003A79103411F4E0E04EC04CC01A93E981F6
:10CB52000E943F7931F40E943A79183111F4E0E0F1
:10CB620042C040C01A93E9810E943F7931F40E9489
:10CB72003A79183211F4E0E036C034C01A93E981F0
:10CB8200E03011F0E4EC01C0E4E80E94357979F478
:10CB92000E943A79E0917300AA81BB81EC9310352F
:10CBA20011F0183521F4E0E018810C94EF6AE1E00D
:10CBB20018810C94EF6A1A93E981E093740010E0F3
:10CBC200E0917400E07811F4163908F005C08BE1A9
:10CBD2008A95F1F71F5FF4CFE0917400E07811F0CD
:10CBE200E0E001C0E1E01881229608950E94BD7C38
:10CBF2003D810C8120E087DFE03011F5EE810E945B
:10CC02003E6EF1F43A93AEDFE030D1F40E94437904
:10CC1200B9F479DFE030A1F4EE810E942C7981F43D
:10CC2200EDB7FEB7FA93EA931F930E9431791F91F1
:10CC3200E03031F479DFE12F0E94C47C0C949768D4
:10CC420026DFD9CF0E94BD7C30E00E811D815BDFE3
:10CC5200E03099F4EF810E943E6E79F40E944379AC
:10CC620061F41A937FDFE03041F4EC81EA937ADFDA
:10CC7200E03019F459DFE0E002C009DFE8CF0E949A
:10CC8200C47C2896089522970E94BB7C50E02B8595
:10CC92003A85A89538DFE03011F00C94A666EE854F
:10CCA2000E943E6E11F00C94A6662A935BDFE03080
:10CCB20011F00C94A6663A9355DFE03011F00C9413
:10CCC200A66621DFE03011F00C94A666EE850E9484
:10CCD2002C79D9F5E0E0EE83EF83EC85FD85319781
:10CCE2000E941D7549F4EDB7FEB7FA93EA931F93BC
:10CCF2000E9431791F9109C0EDB7FEB7FA93EA930A
:10CD02001F93E1E0EA933ADF1F910E2FEE81FF813C
:10CD1200A885B985EA0FFB1F1083EE81FF8131964A
:10CD2200EE83FF83003039F4EC85FD85AE81BF814F
:10CD3200AE17BF0708F001C0D0CFEC85FD850E9479
:10CD42001D7519F4F1DEE0E002C0A1DEA3CF0E945E
:10CD5200C27C2F96089568970E94BB7C20E0E0E099
:10CD6200EC8FED8F31E0A895E9A1FAA1662777272C
:10CD72000E94927BEA87FB876C877D87EE8D0E94FB
:10CD82004879EE83FF8368877987AA85BB858C857E
:10CD92009D850E94687CEA8BFB8B6C8B7D8B0E944D
:10CDA200EC7AFE017296FA93EA930E94F16AEE8B94
:10CDB200FF8B688F798F0E944E790E94597BAF0159
:10CDC2000E944E79AE8DBB27882799270E94F37A5D
:10CDD2000E946179DE015A960E94597BED93FC9381
:10CDE2000AA119A190DEE030D1F5EDA10E943E6EBC
:10CDF200B1F50E94437999F51A93B4DEE03079F5E2
:10CE0200303051F14F5F5F4FEC8DFD8D3196EC8FDD
:10CE1200FD8FAC8DBD8D1197EBA1FCA1EA17FB072D
:10CE220011F430E018C0EC8DFD8D3197AF8DB8A1B3
:10CE32000E945D7597DEEE8DDA01F0E0EA17FB07DE
:10CE420051F472DEEA8DFB8DA9A1BAA1EA0FFB1F94
:10CE5200E9A3FAA389CFD4CF67DEE0E002C017DEF0
:10CE6200C1CF0E94C27CA6960895A881A03310F07B
:10CE7200AA3308F004C0E881E0530C947068A881DA
:10CE8200A13410F0A73408F004C0E881E7530C94F1
:10CE92007068EFEF0C947068A881AA3020F4E881E2
:10CEA200E05D0C947068A881AA3020F0E881E95C0A
:10CEB2000C947068E8E50C9470681A930A93F894DD
:10CEC2000091630B1091640B7894F8010991199108
:10CED20008951A930A93F1DF8F01EA81FB81AC81F5
:10CEE200BD81EA0FFB1FE01BF10BDF010E94B17C49
:10CEF2002CF4E0E0198108810C941D6BE1E01981AA
:10CF020008810C941D6B0E9466790E9466790E94CA
:10CF12006B790E946B790E947079EAE0F0E00E94DE
:10CF2200736B0E9474790E946B790E947079E2EDB2
:10CF3200F0E0FA93EA930E9466790E946B790E946C
:10CF42006B790E947079E2EDF0E00E94736B0E94AF
:10CF520074790E946B790E9470790E946B790E94A9
:10CF62006679E8ECF0E0FA93EA93ECE3F0E00E94F1
:10CF720077790E9466790E946B79E4E1F0E00E9481
:10CF82009C6D0E947779E2EDF0E00E947479E4E111
:10CF9200F0E00E949C6D0E947779EFE0E09310042C
:10CFA200E2E0E0930D04E0930E04E5E5F0E0FA938D
:10CFB200EA93EEE1F0E00E94876DEEE9F7E10E946C
:10CFC200A76C0E94D96DE0E0E093100408950895E3
:10CFD20099818881009641F0BD81AC81FB81EA8113
:10CFE20005900D920197E1F7FD81EC810C941D6B88
:10CFF200B981A881109631F0FC81EB816A8161933D
:10D002001197E9F7EB81FC8125960895E991F99151
:10D01200A991B9911D900590011421F40020D1F736
:10D02200EE2708951018E1F3E1E008F4E2500895C4
:10D03200E991F991A991B991CD0161916D9366231D
:10D04200E1F7FC010895E991F991A991B991CD0116
:10D0520005900D920020E1F7FC010895A991B99184
:10D06200EE27FF276D91662311F03196FBCF0895CD
:10D07200AA27BB27E991F9910590002011F011969A
:10D08200FBCFFD0108957991E991F991A991B991A7
:10D09200CD01772351F07A9561916D936623C9F79B
:10D0A200772319F07A956D93FBCFFC01089569916E
:10D0B200E991F991A991B991CD01662351F06A954F
:10D0C20005900D920020C9F7662319F06A950D921A
:10D0D200FBCFFC0108955D9BFECFE881ECB9219660
:10D0E20008951A930A93AC81BD810E94D97A309730
:10D0F200C1F0AA81BB810E94D97A8F01309749F091
:10D102000230E0E01E0760F0F80131978F01ED93E5
:10D11200FC93AC81BD810E94B06D3197AE81A0833A
:10D1220003C0EE81EA93D7DF19810881279608951B
:10D132002C970E94BB7C10E0E88DF98D3196E88F28
:10D14200F98F3197E4912E2FE03011F40C94596A43
:10D15200E12FE03039F4253211F411E002C00E94CF
:10D162007D79A5C1E130C1F4253219F40E947D799F
:10D172009DC112E0E0E0E98B00E02D3211F401E004
:10D1820096C12B3219F4EBE2E98B91C1203219F4EA
:10D19200E0E2E98B8CC102C0E23039F450E013E0E6
:10D1A200203311F4006883C102C0E330A1F42033BC
:10D1B20010F02A3308F009C0A52FEAE0EA9FF00137
:10D1C2005E2FE22FE0535E0F72C140E02E3211F467
:10D1D20014E06DC110C0E430A1F4203310F02A3302
:10D1E20008F009C0A42FEAE0EA9FF0014E2FE22FD7
:10D1F200E0534E0F5CC12C3619F4026015E057C1A2
:10D2020004C0E53011F00C94586AE22FE33649F479
:10D212000E948879EE89FF89A481AA930E948E795F
:10D2220045C1E33741F40E9488790E9498790E94AF
:10D2320090751E2F0CC0E037B1F40E9488790E94CD
:10D242009879FA93EA930E9439681E2F08600F7743
:10D25200403011F0411708F001C0142F40E0E0E027
:10D26200E88B30E076C0E43611F0E93611F4046060
:10D2720002C0E537A1F4EAE0E88B01FF08C0E0E074
:10D28200FAEC6AE97BE30E946A6D1AE023C0E0E1EE
:10D29200F7E260E070E00E946A6D15E01BC0E835BD
:10D2A20011F4086004C0E83711F00C94576AE0E109
:10D2B200E88B01FF08C0E0E0F0E060E070E10E946E
:10D2C2006A6D18E007C0E0E0F0E160E070E00E9403
:10D2D2006A6D14E0403011F00F7701C041E001FFA8
:10D2E20008C00E948879AE89BF8914960E94DD7AAF
:10D2F20013C002FF08C00E948879AE89BF891496C4
:10D302000E94006D09C00E948879AE89BF89149677
:10D312000E94D97A66277727EC87FD876E877F87F9
:10D3220002FF16C0AF85AA2362F4EC85FD856E85E7
:10D332007F850E94D879EC87FD876E877F87EDE233
:10D34200E98BE989E03019F01F5F4F5F01C00B7F65
:10D35200342F00FD14C0151710F4351708F00FC054
:10D3620007FF08C002FF04C00B7F2989115001C0CA
:10D3720020E301C020E20E947D795150ECCF1417C6
:10D38200B0F4006102FF0AC00B7FE989EA930E94B0
:10D392008E79503009F0515011504150E0E3EA9338
:10D3A2000E948E79503009F051504150E8CF312F10
:10D3B200E889E030D1F43030B9F003FF08C0EE81E3
:10D3C200FF813196EE83FF833197E49105C0AE81F0
:10D3D200BF81ED91AE83BF83EA930E948E79503074
:10D3E20009F051503150E7CF57C00E94A0790E94F6
:10D3F200657A2E2F2A3030F003FF02C0295C01C06B
:10D40200295A01C0205D04FD25C0213360F4A8859E
:10D41200B9858A859B85A130E0E0BE07E0E08E07F2
:10D42200E0E09E0709F40BC0431740F4531710F0D5
:10D4320000FF01C014C020E207FF0CC020E300611E
:10D4420002FF08C00B7FE989EA930E948E7950306F
:10D4520009F051500E947D79503009F051503150FD
:10D462000E94A0790E94A07AEC87FD876E877F8751
:10D47200E889A885B9858A859B85FF27662777274E
:10D482000E94657A0E946A6DE885F9856A857B85C6
:10D492000E94AD7C09F0A9CF00FF08C0503031F0E6
:10D4A2005150E0E2EA930E948E79F8CF10E044CE28
:10D4B2000E94C27C6A960895FF92F82E22971A93D0
:10D4C2000A93DE010E94C6798D01DE0116960E9442
:10D4D200C6790E94D97AEA83FB83DE0114960E9400
:10D4E200C6790E9405731A930A93FE0136960E942A
:10D4F200786B1EDEAA81BB81E0E0EC931981088182
:10D502002496FF900895A991B991EE27002460E82E
:10D51200E894162E169407941E2A1EF0A015B10543
:10D5220018F0A019B109E62BB7FBAA0FBB1F66952D
:10D5320080F708957B816A81F981E88177FB770F13
:10D5420067FD7160972F9E5781F078F0983190F4C3
:10D55200AA27BB27882708948795B795A7959A95F8
:10D56200D1F7EA23FB23682305C0E8947727EE2747
:10D57200FF2766276F77769508F4606877F9A99197
:10D58200B99189919991EA17FB076807790797FB87
:10D5920008950E9413790E94A97919F40E94B07922
:10D5A2001DC0E6F7A881B9818A819B81E0E0F0E0A5
:10D5B20060E87FE30E94617911C00E9413790E94A2
:10D5C200A97919F40E94B07909C0E6F30E94B079F2
:10D5D200A0E0B0E080E89FE30E94CC7B249608950F
:10D5E2000E94B5790E94AD7C39F4A881B9810E946C
:10D5F200426F0E94E37A20C0AA81BB818C819D8107
:10D602000E94B57C34F40E94B5790E94EC7AC1DFA5
:10D6120005C00E94B5790E94EC7ACFDFA881B9815A
:10D622000E94E37AA881B9810E94DD7AAA81BB8136
:10D632008C819D810E94617926960895E991F991E4
:10D6420030971AF4E095F095319608950E9463653B
:10D65200E0EBEA93E8E1F0E0FA93EA93E1E0F0E04C
:10D66200FA93EA93E3E2F7E0FA93EA930895E0EBA0
:10D67200EA93E0E0F0E0FA93EA930E94F7650C94F3
:10D682006565E0E2EA930C94AC66E0E0F0E0FA93C0
:10D69200EA930895EFEEF0E0FA93EA930895FA938D
:10D6A200EA93EFE0EA930C94B24AFA93EA930C9469
:10D6B2009B42E0930F04E0E0E09310040895E12F11
:10D6C200A0E4B2E0F0E00E94EC79EA0FFB1F0895BB
:10D6D200A12FB0E0ECE3F0E00E94357A3896FA939D
:10D6E200EA930895FA93EA93E2E3F0E00895FA9355
:10D6F200EA93CBCFE0911004E0930F0408950E94C7
:10D702003A0C0C944A48E32FF0E0E05BFD4FE491C1
:10D712000895EA930E94500CFE013696FA93EA931A
:10D722000895FF27662777270E94EC7A84E00E94FB
:10D732005D6A28960895FE017196FA93EA930C9415
:10D74200BB420E94BD7C0C94C345E8E0F0E0FA9332
:10D75200EA930895E4E0F0E0FA93EA930895FA93E5
:10D76200EA93E8E3F0E0FA93EA9308950E94E87AF4
:10D77200BECFE02FF0E00895A0913B0CB0913C0C9D
:10D78200BD01A3E0B0E00E940D7AE60FF71FE4911D
:10D79200E0300895E091C005EE0FEE0FEF5F3E2FEF
:10D7A2000895E32FF0E00895A12FB0E00895A0912D
:10D7B2003B0CB0913C0CBD01A3E0B0E00E940D7A9D
:10D7C200E60FF71F08950E94EA79E05AFD4F089587
:10D7D200FA93EA93E22FF0E008950E94BB7CA091B5
:10D7E20019080895E091C30BF0E00895AFE3B1E0AA
:10D7F2000E94607A089530911E08E1E0E0930D04E2
:10D80200E2E0E0930E043A930E94B417E091990B80
:10D81200E295EF70E0930F04E091990BEF70E093C3
:10D8220010040895FA93EA93E52FF0E0FA93EA934D
:10D832000895E7E3F0E0FA93EA930895E22FE450C3
:10D84200F0E0FA93EA930895EA85FB85FA93EA9366
:10D852000895E32FE058EA9318CFEBE8FBE0FA9340
:10D86200EA930C94BB423A930E94B417A0918B0B9B
:10D87200AD320895E091990BE295EF70E0930F04B9
:10D88200E091990BEF700895E52FF0E00895EA0F0B
:10D89200FB1FFA93EA930895EF5EFC4FBF01E0810C
:10D8A200E058DB01EC930895E0E0EC93AE81BF8198
:10D8B2000895E3E0F0E0FA93EA930895E52FE45047
:10D8C200F0E0FA93EA930895E550F0E00895E091CC
:10D8D200990BE295EF700895EA1BA2E5B7E0F0E03C
:10D8E2000E94EC790895F0E0EE0FFF1FEA5CFD4F15
:10D8F2000895A4E3B2E0F0E0EE0FFF1FEA0FFB1F72
:10D902000895FA93EA93E12FF0E0FA93EA930895E7
:10D912000E94C345E0E0EA930895E12FF0E0FA9314
:10D92200EA930895FA93EA93E2E0F0E0FA93EA9335
:10D932000895EBE8FBE0FA93EA93EAE0EA930C94A9
:10D942006445E1E0F0E0FA93EA930895FA93EA93EA
:10D952000C944D450E94E87AFA93EA930895ABE05D
:10D96200EA9FF001E252FA4F0895ED85FE85FA939F
:10D97200EA9308951A930A9335CF1A930A93EFE024
:10D98200EA930E94B24ADDCFE1E0E0933D0C0E94AF
:10D992005E67E0933F0CF093400C0895BD01AAE04E
:10D9A200B0E00E940D7AE60FF71F0895FA93EA930A
:10D9B200EAE0EA930C946445E1E0E0930E0465CE5C
:10D9C2000E949C450C947F45E0E2EA930C94364514
:10D9D200A3E2B7E0E881F0E0EE0FFF1FAE0FBF1F3A
:10D9E2000E94D97A0895FA93EA930C944E40E88102
:10D9F200F0E00895EE0FFF1FAE0FBF1F08950E94C3
:10DA0200D97A0E94F77908950E94EC7A0C942F40FB
:10DA1200FA93EA930C949C45A9E0B0E00E94077B3C
:10DA22000895A7E11A9FF001EF5CF94FE081089594
:10DA3200E12FEF5FEA930C946440F0E0D4CFE8E08A
:10DA4200F0E055CEEA93E6E0EA930E941A407DCEDA
:10DA5200E093620088EC90E00197F1F70895E0937B
:10DA6200610088EC90E00197F1F70895E0916D056F
:10DA7200F0916E050895E0916905F0916A050895A7
:10DA8200AE0FBF1FE3E0F0E00E94607A0895FA93C0
:10DA9200EA931A930A930C947011FA93EA933A93C5
:10DAA2002A930C947011A0917105B091720508959A
:10DAB200A0917305B09174050895A0E0B0E00E94B2
:10DAC200037B08950E94FC7AEA1BFB0B0E94F77904
:10DAD2000895E887F9876A877B870895A885B985BD
:10DAE2008A859B85EFEEF0E060E070E008950E9489
:10DAF200F7790E948A7A0895A4E0B0E00E94037B3D
:10DB02000895EC83FD836E837F830895FA93EA93ED
:10DB12000C94B745FA93EA930C94BA79A9E01A9F48
:10DB2200F001E058FC4F089537960E94E87ADF0131
:10DB32000E94D97A0895FA93EA93E8E2F0E0089510
:10DB42000A921A92FA926A937A938A939A93AA936E
:10DB5200BA93EA93FA93EFB7EA931A930895ED9181
:10DB6200FD913196FE93EE930895ADE01A9FF00178
:10DB7200EB5FFC4FE08108951A93E1E0EA930C9485
:10DB82002546ADE01A9FF001DF01EB5FFC4FE0811B
:10DB9200E0300895E2E0EA930C942546FA93EA9382
:10DBA200E4E6F0E0FA93EA930E946A67E0300895AF
:10DBB200E1E0E0930D04E0930E040895E09129085A
:10DBC200F0912A0860912B0870912C080895E09139
:10DBD2002108E150A3EAB6E0F0E00E94EC79AE0F32
:10DBE200BF1F0E94DD7A0895E12FEF5FF0E010CFB2
:10DBF200E0912208EA93E0911E08EA930E94C61976
:10DC0200A0911F0CB091200C10970895A091210CA7
:10DC1200B091220C8091230C9091240C0E94B57C2F
:10DC22000895E0911F0CF091200C0895E091210CD1
:10DC3200F091220C6091230C7091240C0895EAE07B
:10DC4200F0E068CFE2E3F0E065CF1A93E0EAEA930E
:10DC5200EA81F0E0E054F14FFA93EA930E94F7650B
:10DC62001E2F0895E0EAEA93EA81F0E0E054F14FD2
:10DC7200FA93EA931A930C942366EA930E94A76597
:10DC8200E0300895E0EAEA93EEE5F0E0FA93EA93F1
:10DC9200E0E0FFE0FA93EA93EFEBFBE00895FA93FA
:10DCA200EA93EFCCE0EAEA93E981FA81E050FE4E92
:10DCB200FA93EA930895EA81F0E0A8E2B0E00E94C4
:10DCC200357A0895E0EAEA93E2E0F0E0FA93EA9323
:10DCD2001A930A930895FA93EA930C944466FA937A
:10DCE200EA930C94F765E0EAEA93E8E2F0E0FA934B
:10DCF200EA931A930A93EBE8FBE00895EBE8FBE062
:10DD0200FA93EA930895EDE2EA93EAE0F0E0FA93F7
:10DD1200EA930E94F967E0E00895EA81F0E0ABE05F
:10DD2200B0E00E94357AE050F24F8F01AA81AA300A
:10DD32000895E0EAEA93EBE0F0E0FA93EA931A93AB
:10DD42000A93E3EBFBE00895E4EBFBE0FA93EA933A
:10DD52000895EA81F0E0EE0FFF1FE050F04F8F01CF
:10DD6200AA81A0380895E150F0E00895EA81F0E038
:10DD72000E94EC79E058F14F8F01AA81A5300895F5
:10DD8200E0E3FCE0FA93EA93E0E0EA93E3CCEDE12E
:10DD9200FCE0FA93EA93E0E0EA93D7CC0E94EC79B4
:10DDA2000E94E879DF01EA85F0E0AE0FBF1FE8E0EC
:10DDB200F0E00E94357AE050FA4E8F01E0EAEA93F1
:10DDC200C4CC1A930A93EDE1FCE085CFAE81BF810A
:10DDD200888599850E94CA79EE83FF83688779874F
:10DDE200089540931F0C5093200CEE81FF816885AB
:10DDF2007985E093210CF093220C6093230C7093AD
:10DE0200240C0895F0E0AE0FBF1F0895EA930E941C
:10DE1200B4170C94831EE091960BF091970B089522
:10DE2200FA93EA930C945317ED81EA93ED81EA9306
:10DE32000895E091AD0BF091AE0B0E94F779089531
:10DE4200F0E0A4E6B0E00E94357A0895EC81F0E0BB
:10DE5200EA0FFB1F0895E0912708F0912808089522
:10DE6200E093280CF093290C0C94171BE3EAF6E0DC
:10DE7200FA93EA93E0E0EA930895FA93EA930C9412
:10DE8200F967E0E0F0E060E070E00895E0932908CF
:10DE9200F0932A0860932B0870932C080895E09160
:10DEA200980BA3EAB6E0F0E00E94EC790895AE0F79
:10DEB200BF1F0E94DD7A0895ED5EF94FE081E130E7
:10DEC2000895FA93EA93E0912208E05DEA930895B7
:10DED200EA930E94F662E1300895ECE3F8E0E09301
:10DEE200600BF093610B0895E12FA3EAB6E0F0E036
:10DEF2000E94EC7908950E94E967A881AF5FEAE089
:10DF02000E943F7AE05D0895A881AF5FEAE00E9437
:10DF12008F7AE05D0895FA93EA93E0E0EA93089538
:10DF2200AAE0B0E00E94077B0895E12FF0E00E9492
:10DF3200EA79E854FF4F32960E94E87A0895E12F79
:10DF4200F0E00E94EA79E854FF4F08953696E49192
:10DF5200D901EC930895E0EAEA93E5E0F0E0FA9360
:10DF6200EA930895EA930E94081BFA93EA93E5E282
:10DF7200FCE00895FA93EA93EFEFEA93E5E0F0E02C
:10DF82007CCFE093260CF093270C08950E94FC7A34
:10DF9200EA1BFB0B0895EAE2FCE0ECCFA0912B0C0C
:10DFA200B0912C0C0895E0E0E093390CE0933A0C28
:10DFB2000895A0912D0CB0912E0C0895E0912D0C96
:10DFC200F0912E0CAC81BD81EA0FFB1F0895E09306
:10DFD2002D0CF0932E0C08951A930E94A21B1E2F53
:10DFE2000895E0932B0CF0932C0C0895FA93EA9386
:10DFF2000E946A67E0300895ABE01A9FF001E45294
:10E00200FA4F08951A930E94911DD3CFE0912B0CE1
:10E01200F0912C0C0895EA930E94911D0E942E1DEE
:10E02200E0300895EB81EA930E94C91BFA93EA93C8
:10E03200EAE2FCE00895E0E0E093500CE0934F0C3C
:10E0420008951A930A93E0911208ABE0EA9FF00157
:10E05200E752F84F8F01D80111960895E0E0F0E001
:10E06200ED93FC930895EA81D801EC93E2E1F8E0A4
:10E07200FA93EA930E948532198108810895E12F6B
:10E08200ACE8B0E0F0E0EE0FFF1FEA0FFB1F0E94CA
:10E09200E87A0895E150ADE0EA9FF0010895ACE816
:10E0A200B0E0F0E0EE0FFF1FEA0FFB1F0E94E87ADC
:10E0B2000895A0911608B0911708EA2BFB2BE09364
:10E0C2001608F09317080895E150A7E1EA9FF001BE
:10E0D2000895A7E10A9FF001E15DF94FAF010895AC
:10E0E200ED55F94FE081E0300895E981FA81FA9324
:10E0F200EA930895E12FF0E00895E2E0F0E00E9453
:10E10200607A0895ABE9BBE0E0911A080895AEE9A0
:10E11200BBE0E0911A0876CEA1EABBE0E0911A08D2
:10E1220071CEA3E2B7E0B0CBEE0FFF1FEA0FFB1FE9
:10E132000895E081F0E00895A7E11A9FF001E15D02
:10E14200F94FEE83FF83AE81BF810895EE81FF8197
:10E15200A481AA930C94D91E0D901C90AE81BF810C
:10E162001296EC91F0E0E00DF11DDB01ED93FC93D2
:10E172000895ED91FD913197FE93EE9308950E94DB
:10E182007E20EF770E2EAA85BB851296EC91E015C4
:10E192000895A3E20A9FF001E855F94F0895E0912E
:10E1A2001208ABE0EA9FF001E752F84FEC87FD87D7
:10E1B200AC85BD85119608951296EC91AC85BD850E
:10E1C2001696EC930895D001F0E00895A885B985DC
:10E1D20018960E94D97A0895AC85BD85EC93E2E148
:10E1E200F8E0FA93EA930C948532E885F985A281E6
:10E1F200AA930895AA85BB85EC91EA93E3E0EA939A
:10E202000C94E741AA85BB85E0E0EC93E2E0E09361
:10E2120024060895BF0100801180AE81BF8112964D
:10E22200EC910895DB01ED93FC93AE81BF811296D0
:10E232003BCBE4E6F0E00E94357A0895F0E0ED93FE
:10E24200FC930895E2E1F8E0FA93EA930C948532A4
:10E25200E0911908A0911808EA170895F0E0E00D7E
:10E26200F11D0895A4EABBE045CFAEE9BBE0EE277D
:10E27200A10FBE1FEC910895A1EABBE0EE27A10F0A
:10E28200BE1FEC910895BD01AAE0B0E00E940D7A94
:10E29200DB010895E081EA930C94535DE0E4FAE037
:10E2A200E0935E0BF0935F0B0895EA930E94AF61D7
:10E2B200E0E00895EA930E94AF610C943463AEE902
:10E2C200BBE0EE27A00FBE1FEC910895A1EABBE0D0
:10E2D200EE27A00FBE1FEC910895ABE9BBE0EE273D
:10E2E200A00FBE1FEC91E1700895A4EABBE041CA01
:10E2F200A1EBBBE0EE27A00FBE1FEC910895AAEAA6
:10E30200BBE0EE27A00FBE1FEC910895EA81ADE0BD
:10E31200EA9FF001E15FFC4FA0E0A083EA81EA936B
:10E322000895ADE0EA9FF001EB5FFC4F0895ABE08A
:10E332000A9FF001E452FA4F0895ABE00A9FF00100
:10E34200EE51FA4F0895FA93EA930C941234FA9329
:10E35200EA930E945C423A931DCCE0912D0CF0911D
:10E362002E0C30970895AFEFBFEFA083B1830895CD
:10E372000E945E67E093550CF093560C0895FA9351
:10E38200EA93E0E0F0E80895E0911208ABE0EA9F3A
:10E39200F001E752F84FFA93EA930E94EE2752CF28
:10E3A200E0911008ABE0EA9FF0010895E0E1F8E0A7
:10E3B200FA93EA930C948532FA93EA930C94E1511E
:10E3C200E88DABE0EA9FF0010895FA93EA93D1C990
:10E3D200E0E1EA93E0912506EA930E9487171E2F57
:10E3E200089539DDFA93EA930895FA93EA930C9427
:10E3F2005C1DE0932506E0E0E093520CE1E3E0933C
:10E40200530C0E942D290C94FA24FA93EA930C944B
:10E41200C061E1E4F9E0E093600BF093610BE3E0AB
:10E42200EA930C945661A091600BB091610B089530
:10E432000E945E67E0934A0CF0934B0C0895E093C0
:10E44200600BF093610B0895E3E0EA930C9456613C
:10E45200E0932708F09328080895E0E0F0E0E093C5
:10E462002508F0932608E2E0E0930E040895E09177
:10E4720013042ACAE0912508F0912608B4CAE09153
:10E482005D05F0915E0531970895FA93EA930C9435
:10E492009144EF5CEA930C943645A3EEB6E081C951
:10E4A200A4EABBE0E0911A08F0E03ECE0E94D97ADD
:10E4B200D001ED93FC9326CEF0E0EA0FFB1F0F0193
:10E4C20021CEA3E2B7E06DC9E7E0E0931808EA9332
:10E4D200E0E0EA93DAC8EA930E94C33F0E94FA415D
:10E4E2001E2F0895EAE2EA93E1EBF5E114CD0E94D2
:10E4F200E22AE1E0EA930C94CA2A1F771A930C9459
:10E50200B417A0912508B09126080895E8EEF3E02B
:10E512000E94927A0895E053F0E00895A0E024FC6E
:10E52200A1E0A0300895E0E0EA93AFC8E09133089B
:10E53200F0913408FA93EA930895FA93EA930E94C9
:10E542006A67E13008950E945E67E0933308F093B2
:10E5520034080895E0E0E0934F0C0895D2DFEA1703
:10E56200FB070895E0931808E0E0E093300808956F
:10E572000E94D4620E944B2CE093240808950E94CA
:10E58200B4170C94C345E0911908EA93E0E0EA93CA
:10E592000E94F52B0C94A0270E94FA411E2F1A9379
:10E5A2000E947E2C103808951A93E091C605EA93D2
:10E5B2000895E0918A0BEA930E94C116E030089513
:10E5C2000E945E67E093570CF093580C0895FA93FB
:10E5D200EA93F6C9D90118960E94D97A0895E4E619
:10E5E200F0E060E070E00E948A7A08950E94B41719
:10E5F20012CC0A93E091C605EA930895E0912F08A0
:10E60200EA930A930C94E5180E94D97AFA93EA9352
:10E612000895A0E6BBE0A3CAE0913C08E053E09372
:10E6220022080895FA93EA93E0E3EA930C94D46201
:10E63200E0913908EA930C947E620E94F7790E9475
:10E64200EC7A08950E943C62EBE3EA930C94AF618A
:10E65200E89423F8E0E0F0E0FBDEE0E0E0931E085F
:10E662000A93E1E0EA930C94F52BE89423F8E0E0B6
:10E67200F0E0EEDEE0E0E0931E08EA930C94CA2A92
:10E68200E0911208ABE0EA9FF0010895A881B981F8
:10E69200EC91EF5FEC930895ABE00A9FF001E35237
:10E6A200FA4F0895A083ABE00A9FF0010895ABE012
:10E6B2000A9FF001E152FA4F0895E8EDF5E1FA936D
:10E6C200EA93EA85ABE0EA9FF0010895AC81BD814F
:10E6D200EE27A00FBE1F0895E02FAC81BD81F0E0B0
:10E6E20008950E94EC7A84E00E945D6A289608955B
:10E6F200EE27A30FBE1FEC91D001EC930895A2E583
:10E70200B7E00C94D26B0E94EC79EA0FFB1FAF01C9
:10E712000895E0912D0CF0912E0C0895E32FA09115
:10E722001E08EA0F0895ADE02A9FF001E35FFC4F57
:10E732000895A8E0B0E00E94077B0895F0E0FA9304
:10E74200EA9308950E946B410C943A41F0E00E94D2
:10E75200EC7908950E94EC7A0E9455410C943A415A
:10E762000E946B41EDEFF5E1D6CB0E943A410C9449
:10E772003A4120E030E0E12FE05DEA93E0E0F6E1AB
:10E78200A0CBEAE0EA930C949061E4E4FBE0FA9314
:10E79200EA93089510915D0500915F0508950E9426
:10E7A200FA413E2F0C94DF44EAE0F0E00E94357A11
:10E7B2000895DF01EE27A30FBE1F0895EF81F885AC
:10E7C200FA93EA930895F0E0EA0FFB1F0895E02F11
:10E7D200A0E0B2E0BBCFEA0FFB1F3296E4910895AE
:10E7E200FA93EA93E0911C0CEA930E945937E132C2
:10E7F2000895EA930E94FF36E1320895E6E0F0E0E0
:10E802000C94786B0E949C45ABE9BBE0EE27A10F0C
:10E81200BE1FEC91E1700895EE0FFF1F0C94486C3F
:10E82200EA930E945937E13208950E94600C0C94D9
:10E83200466BEAE3EA930C9436450E94EC7A0C9418
:10E842004340E3E7EA930C943645EA23EA930E94B5
:10E852006A40BAC8EA930E946A40B6C8DF0132969B
:10E8620079C80E94EA79E854FF4F0895E2E4F6E09D
:10E87200E0933B0CF0933C0C08950E944A19E0E0AF
:10E88200E09321080E9489140E94600CE1E0E09369
:10E892001B0808950E94C3450E94010F0E94FA417D
:10E8A2000E2F0D330895EAE2EA93E8EAF6E10895BD
:10E8B200EA930E94D9140C94600CE093C105F09382
:10E8C200C2050895FE01FA93EA930895E0ECF6E199
:10E8D200FA93EA93EE85FF856889798902CFE4ECA1
:10E8E200F6E1FA93EA93AE85BF858889998977CE56
:10E8F2000E94EC7AAA89BB898C899D89E4E6F0E0C2
:10E9020060E070E00E94A47A0E94EC7A88E00E94A3
:10E912005D6A2C960895EDECF6E1FA93EA93EE85A2
:10E92200FF858BCE84E00E945D6A2896CBCFFA9356
:10E93200EA93EE85FF8508950E9499620C945E67C2
:10E9420084E00E945D6A28960895EE27A10FBE1FFB
:10E95200EC910895EA930E94D5401F5F0895E091DB
:10E96200C405A7ECB5E0F0E00895AF5FEAE00E94CD
:10E972008F7A0895E091C305A7ECB5E0F0E0D4CB1F
:10E98200A0E0A083E981ADE0EA9FF0010895EF7372
:10E99200A5E1EA9FF001E051FB4F0895EF73ABE070
:10E9A200EA9FF001EC5EFB4F0895AC81BD81EE273A
:10E9B200A30FBE1FAC91A0300895ABE00A9FF001F7
:10E9C200EC5EFB4F0895EA0FFB1F0F01AC81BD8186
:10E9D2008FCEA5E10A9FF001E051FB4F0895EE8131
:10E9E200FF8101801280AE81BF8115960E94D97A83
:10E9F200D0010895FE013896FA93EA930895EAA5A4
:10EA0200FBA5FA93EA930895FA93EA93FE013A96E4
:10EA1200FA93EA930E94196830E0E02F0895E0919A
:10EA2200C105F091C2050895A1ECB5E0ED91FD910B
:10EA32003296FE93EE930895AE81BF81EA17FB07EB
:10EA42000895E0E0E0936505E093660508951A9362
:10EA52000A933A932A930895FA93EA93E0910E0463
:10EA62000895A0910003B09101030895E09100037D
:10EA7200F0910103FA93EA93E0910203F091030308
:10EA8200FA93EA930895E0930003F0930103089543
:10EA9200A981BA815ACFF801AA81BB81EA0FFB1F73
:10EAA200E4910895AE0FBF1FAC91A0300895D80134
:10EAB200F0E0AE17BF070895AE0FBF1FEC91EA93C7
:10EAC2000895EFEEF0E0EA1BFB0B0895A0910E040F
:10EAD200E4E1EA9FF0012E2F3327C8CFEFE0EA935B
:10EAE2000E94B24A0E94C47C0895ECE0EA9FF001C1
:10EAF200A0910D04EA9FF00108951A93E1E0E093DA
:10EB02000E04E0930D0410E00895ED81FE81FA9366
:10EB1200EA930895EF81F885EA1BFB0B0895FA93B7
:10EB2200EA930C942F68EA9FF001F0E008953A937B
:10EB32002A935A934A930895EAA5FBA5E20FF31F7D
:10EB4200FA93EA930895ECA1EA930C94154B3A9345
:10EB52002A93EEA1FFA1E40FF51F0895FA93EA9319
:10EB6200EBCFEAA5FBA5E40FF51FFA93EA93EBCFEF
:10EB7200E20FF31FFA93EA930895FA93EA935A93F2
:10EB82004A930895EA9FF001AEA1BFA1F0E0089573
:10EB9200E2E0E0930E04E0E2F0E0EAA3FBA30895D2
:10EBA200AE1BBF0BAACAEE8DF0E00895E20FF31F71
:10EBB2003196FA93EA93ECA1FDA1E40FF51F319689
:10EBC2000C94876DECA1FDA1E40FF51F0C94876DE9
:10EBD200E9A1F0E0DE0116960895ED8DEA930E9418
:10EBE200EC44E9A1EF5FE9A30895ED8BFE8BAB89BD
:10EBF200BC8983CAA98DBA8DEA0FFB1FE98FFA8FF0
:10EC0200EB89FC89AF89B88DEA0FFB1FEF8BF88F78
:10EC1200ED89FE89AD89BE890E94357A0E94F77915
:10EC22000E94927BEE87FF87688B798BEB89FC8948
:10EC3200AB89BC890E94357A0E94F7790E94927B47
:10EC4200AE85BF85888999890E94687CEA87FB879F
:10EC52006C877D8700E010E00895F8010E94F77943
:10EC62000E94927BEE83FF8368877987AE81BF81A2
:10EC7200888599850E941A7CAA85BB858C859D858D
:10EC82000E941A7CAE85BF85888999890E94F67A8E
:10EC92000E94C57B0E945B7BAF015A934A930C94FE
:10ECA200846AE98DFA8DE21BF30BFA93EA930895D5
:10ECB200E98DFA8DE01BF10BFA93EA930895F901BD
:10ECC200AD8DBE8D0C94486CED8DFE8DE01BF10B6D
:10ECD200FA93EA93EA8DEA930C94154BAD8DBE8DAF
:10ECE2000C94486CEFE3F1E0EA1BFB0B0895EB8117
:10ECF200FC81AF81B8850895E00DF11DFA93EA9386
:10ED02000E942649E5E3EA930895E09365000C9496
:10ED1200236E0E94BB7CEE81EA930E9455498F01CB
:10ED22000895E985FA85AD85BE8508950E946F49EB
:10ED3200EB85FC85FA93EA930C948749ED85FE8571
:10ED4200A985BA85AE17BF070895EB85FC85AF810B
:10ED5200B885AE17BF070895AD85BE85E985FA85EA
:10ED6200EA1BFB0B0895FA93EA930C941F6BAB8595
:10ED7200BC85D0CEAF81B885EB85FC85EA1BFB0B49
:10ED82000895D9010E94357A0F010895D0010E9499
:10ED9200607AAF01FA01AD85BE850C94486CED85B1
:10EDA200FE85E21BF30BFA93EA930895AD85BE85C7
:10EDB2000C94486CA985BA85ED85FE85EA1BFB0B90
:10EDC2000895E881F981FA93EA9308955A934A9350
:10EDD200EE85FF85ACCDFA93EA93EC85FD85FA9337
:10EDE200EA930E94F64BE0910E04AA85BB85EBCC18
:10EDF200E05CF54F4FCAE091380CA091370CEA174E
:10EE02000895E0911108ABE0EA9FF0010895E3E074
:10EE1200EA930E941B62F5CFE081E05DEA930C94D5
:10EE2200AF61A091260CB091270C0895E2E5EA9318
:10EE32000E94AF610C949C4CF096EA930E947E6211
:10EE4200E2E7EA930C94AF61EA930E94AF61EEE0CD
:10EE5200EA930C94AF61E0EEF6E1D7CA0E94E26158
:10EE6200EBE3EA930C94AF61E0E3EA930C94AF61B5
:10EE7200EBE3EA930C94AF615A934A930E945317BF
:10EE82000E2F00340895FA93EA930C9485321A9364
:10EE9200E985FA85FA93EA930895E552F84FA88531
:10EEA200B985A083B183ECCBE2E5EA930C94AF6120
:10EEB2001A93E0913908E0531E2FEDE3F8E0BFCA40
:10EEC200E0911208A0911308EA170895E3E1F8E02F
:10EED200DACFE0911308ABE0EA9FF0010895A09128
:10EEE200750B43CDE093750BEAE2EA930E947E62D2
:10EEF200DBCFE091750BE05AA7CFD9011696EC91C2
:10EF02001DCCF901A281B381BA93AA9308950E94FC
:10EF1200E261EAE3EA930C94AF61D9011196E0E071
:10EF2200EC930E949962D2CFD901EC9107CCE05DBB
:10EF3200EA930C94AF61E05DEA930E947E62B4CFE3
:10EF4200EA58F44F69CFEEE0EA930C94AF61EAE33A
:10EF5200EA930E94AF61F9010895E093610CF09386
:10EF6200620CE2E0E0933608D9011196EC93089521
:10EF7200EA930E947E6298CF0E94E261DDCCE0912A
:10EF82001A0CD9CFE0911A0CF0E0DACFFA93EA9397
:10EF920065CF0E94E261ECE2EA930E94AF6111CF79
:10EFA20042DAAC91A0330895A0915E0BB0915F0B51
:10EFB2000895EE81FF81E093280CF093290C1093C1
:10EFC200250C0E94171BE1E3089541E050E00E94E6
:10EFD200E260E887F987EAE3EA930E945360E1304E
:10EFE20008951A93E985FA85C8CDE2E2EA930E9470
:10EFF2005360E030089517DAAC91A032089513DA25
:10F00200AC91AB3308950FDAEC91EA930895EAE3F9
:10F01200EA930C9453600E94E2603197E887F98783
:10F02200E88508950E94D97AE40FF51FD001ED9387
:10F03200FC930895E091400BF0E0ED55F94F0895EF
:10F04200E0E0E093660CE093670C08950E94E260B2
:10F052003197E093400BE091590BA091400BEA17D6
:10F0620008950E949B55E091400BEA930895ECE2CB
:10F07200EA930E945360E0300895EC5BF44F0F0175
:10F08200D2D9EC91D001EC931F5FC3CAEC5BF44F71
:10F09200A0E0A0830895EA930E945360E1300895AE
:10F0A200E091410B90CBE091410BEF5FE093410B7C
:10F0B2000895A4EABBE0E091410BF0E00C94957056
:10F0C200ABE9BBE0E091410B0C94036FE091410B83
:10F0D200F0E00895E2E2EA930C94AF61FA93EA93C6
:10F0E2000C941152E091400BF0E0BBCBFA93EA93FF
:10F0F2000C94E2610E94E261ECE2EA930C94AF614B
:10F10200ECE2EA930C94AF610E940652E0E0E093D5
:10F11200410B0895E091410B0C94036FE091600B59
:10F12200F091610B0895AEE5BBE00C94B06D3CDF4D
:10F13200EC93F9CFE0E0EA930E946A52E09335083B
:10F142000895AA81BB81EC91E295E07FAE2FEC811C
:10F152000895EA0FAA81BB81EC9398CAE091070D4A
:10F16200A091060DEA170895E0913B09F0E0E05CFA
:10F17200F64F08951083E0913B09EF5FE0933B095E
:10F18200E12FA0913D090895E0933D09E0913C09EA
:10F19200E150E0933C09E0300895E05CF64FA0E0D6
:10F1A200A0830895E091D20DF091D30D0895A0911E
:10F1B200D00DB091D10DEA17FB070895E12FA09170
:10F1C200D70DEA0FE093D70DE091D90D0895F0E045
:10F1D200E85CF74F10830895E091DE0EF0E0E35211
:10F1E200F24FE081E0939C00E091DE0EEF5FE0934E
:10F1F200DE0E089518D9AC91AA3308950F0113D9E0
:10F20200EC91E0530C942F71EA930E94AF611F5F5F
:10F212000895EEE8F7E1FA93EA930895E881EA9314
:10F222000C94AF61E881F9816A817B810E94EC7A5A
:10F232000895E05CF54FE081E0300895EA930E9482
:10F242004D67EA930C94535DEA930E94ED63EAE5FD
:10F25200E0933E090895EA930E949A65E03008958A
:10F26200E0E0EA930C94BF65EA930E94DC65E0302B
:10F272000895E0917100E87F1E2F0895E0937300D6
:10F28200E4E8F2CF0A930E94B365E0300895FF27C5
:10F29200662777270E94927B0895EE8DAE85BF8503
:10F2A20088899989F4DF0E941A7CA9A1BAA18827CA
:10F2B20099270E94F37A0E94F67A0E94C57B0895EC
:10F2C2000E94F67A0E94C57B0895EAE0F0E0FA9384
:10F2D200EA930895E4E1F0E0FA93EA930895ECE00A
:10F2E200EA930C94A648FA93EA93F4CFFA93EA933A
:10F2F200ECE0EA930C94B24A2A93ED89FE89FA93E0
:10F30200EA93FE017596FA93EA930C947268EE8979
:10F31200FF893497EE8BFF8B0895ED89FE89FA936E
:10F32200EA93FE017596FA93EA930C947268AE8999
:10F33200BF8914960E94D97AEE83FF830895E885E7
:10F34200F9856A857B85AC85BD858E859F85089507
:10F352000E949B6AE883F9836A837B830895E8812C
:10F36200F9816A817B810895EA81FB816C817D81CB
:10F372000895E991F991309639F080EA9FE001977A
:10F38200F1F7A8953197C9F708950024AF0DB01D84
:10F392000895EA0FFB1F681F791F0895EA1BFB0BF4
:10F3A200680B790B0895F195E195F0400895F09579
:10F3B20060957095E195FF4F6F4F7F4F0895EE2353
:10F3C2000E2EEA2F19F0EE0F0A94E9F70895EE0FC8
:10F3D200FF1FEE0FFF1FEE0FFF1FEE0FFF1F08951F
:10F3E200FE2FFF0FFF0B6F2F7F2F08956F2F660FDA
:10F3F200660B762F0895BA2FBB0FBB0B8B2F9B2F5B
:10F4020008958B2F880F880B982F0895EA17FB0712
:10F41200E1E00CF0EE270895FA9FF02DEB9FF00D3E
:10F42200EA9FE02DF10D08957A9F702D6B9F700D6C
:10F43200F89F700DE99F700D6A9F602D710DFB9F03
:10F44200600D711DE89F600D711D8827FA9FF02DD8
:10F45200610D781FEB9FF00D611D781FEA9FE02D73
:10F46200F10D681F781F089582D0D6DF0EF49BDF5E
:10F4720008958BD0D9DF0EF49ADF0895002498E026
:10F48200AA0F001C0E1A10F40E0E01C0A1609A956C
:10F49200B9F7EA2FA02D08950024112490E1AA0FB4
:10F4A200BB1F001C111C0E1A1F0A18F40E0E1F1E81
:10F4B20001C0A1609A9599F7FD01D001089557D036
:10F4C200EBDF0EF470DF08953F934F935F930024B8
:10F4D20011244427552730E2AA0FBB1F881F991F0A
:10F4E200001C111C441F551F0E1A1F0A460B570BF6
:10F4F20028F40E0E1F1E461F571F01C0A1603A9529
:10F5020059F7FD01BC01D001CA015F914F913F91B2
:10F5120008953BD0D9DF0EF44ADF0895AFDFEA2F1A
:10F522000895E894B7FF04C0A095B0951196689429
:10F53200F7FD39DFB1DFFD010EF435DF0895C4DFD9
:10F54200FD01BC010895E89497FF09C0A095B0950C
:10F5520080959095AF5FBF4F8F4F9F4F689477FD17
:10F5620026DFB2DFFD01BC010EF421DF0895E8942D
:10F57200F7FF02C018DF6894B7FF06C0A095B095E8
:10F58200119600F8039400FA0895E89477FF02C0F8
:10F592000EDF689497FF0BC00024A095B09580956C
:10F5A20090951196801D901D00F8039400FA08951D
:10F5B200ED91FC9111970895ED91FD916D917C91E2
:10F5C20013970895ED93FD936D937C9308950590A1
:10F5D200F491E02D08957A936A93FA93EA93089549
:10F5E200689401C0E89401D09DD0182E862F612D19
:10F5F200192E972F712D1B2EBF2FF12D1A2EAE2FE4
:10F60200E12D0895119602D0FE2F1197E199FECFB8
:10F61200FF93FFB7F894AEBBBFBBE09AEDB3FFBF59
:10F62200FF91089507D01196EF93EF2F03D0EF913A
:10F6320011970895E19B02C0A895FCCF9FB7F8945B
:10F64200AEBBBFBBE09A8DB3E81719F0EDBBE29AEF
:10F65200E19A9FBF0895552342F4503811F4E0FF18
:10F6620004C03196691F791F6BF050E8572711F4D7
:10F672005F93CDC05F3F31F0660F000C57956795E1
:10F68200752F08955F9300200AF0CDC0C6C050E8E0
:10F69200192E1522880F991F9527550F879550E827
:10F6A200072E0522660F771F7527550F6795089558
:10F6B200689401C0E8945F93F2DF703818F07F3FDE
:10F6C20008F4A5C056E1571BAAF4519558300EF420
:10F6D200593030F0EFEFFFEF6FEF7FE777F91AC0A5
:10F6E20077275523B9F0EE0FFF1F661F771F5A9534
:10F6F200D1F710C07727583028F0EF2FF62F672F59
:10F702005850F9CF552331F076956795F795E795DF
:10F712005A95D1F700200AF44ADE5F910895689461
:10F7220001C0E894309760407040B1F0002426F0A8
:10F73200772312F400943BDE172E7EE1112032F083
:10F742007A95EE0FFF1F661F111CF9CFEF2FF62FD0
:10F75200612D5F938ADF5F9108954F93AF01FD01A1
:10F76200DA01AB01BC01CA01402D012C142E4F91CC
:10F772000895EA0FFB1F681F0895E095F0956095C4
:10F78200EF5FFF4F6F4F08955F9381DF903871F104
:10F7920050E8152604C05F937ADF903839F170384B
:10F7A20021F1572F591B13F112F4D7DFFACF583139
:10F7B20018F0AA27BB278827583028F0AB2FB82F7C
:10F7C20088275850F9CF552329F08695B795A795E4
:10F7D2005A95D9F7502D512562F0CBDF38F4679551
:10F7E200F795E795739513F41EC0B7DF3EDF5F917F
:10F7F2000895EA1BFB0B680B51F010F40094BDDF77
:10F802006623A2F3EE0FFF1F661F7A95CBF7EE2752
:10F81200FF27662777275F910895EFEFFFEF6FE7E6
:10F822007FEF5F910895EFEFFFEF6FE77FE75F9163
:10F8320008955F932CDF703851F3903841F301241F
:10F842000894791F23F41CF300203AF3ECCF0F92B3
:10F852001F932F933F934F93112722279927689F36
:10F86200A0018F9F302D410D591F6B9F300D411DFF
:10F87200591F8E9F27D0BF9F25D06A9F23D0BE9F3E
:10F882001DD0AF9F1BD0AE9F110D291F391F491FDD
:10F89200591FE32FF42F652F522F4F913F912F9134
:10F8A2001F910F9066232AF0550FEE1FFF1F661F50
:10F8B20002C073954BF2CFDE5F910895100D211DAA
:10F8C200391F02C0200D311D491F591F08955F9332
:10F8D200DEDE703821F411200AF49FCFA4CF9038D5
:10F8E20009F495CF01240894970B1BF4D4F300205C
:10F8F200F3CF792F1F932F933F934F931124112707
:10F90200222733274427552790E2AE17BF078607E1
:10F91200410730F0AE1BBF0B860B410B089401C0B0
:10F922008894551F221F331F111CAA1FBB1F881F3B
:10F93200441F9A9551F7F901612D4F913F912F91F3
:10F942001F91662332F0550FEE1FFF1F661F7A9537
:10F9520043F281DE5F9108953097604070400895D0
:10F9620000240A160B06089500240A160B06080640
:10F97200090608955A934A933A932A931A930A933B
:10F9820008955D814C813B812A8119810881089506
:00000001FF
